:100000000C9461130C9492130C9492130C9492130D
:100010000C9492130C9492130C9492130C949213CC
:100020000C9492130C9492130C9492130C949213BC
:100030000C9492130C941D750C9492130C949213BF
:100040000C9492130C949C450C9492130C94921360
:100050000C9492130C9492130C945F7D0C9422B622
:100060000C9492130C948A440C9492130C94921353
:100070000C9492130C9492130C9492130C9492136C
:100080000C9492130C9492130C9492130C9492135C
:100090000C9492130C9492130C9492130C9492134C
:1000A0000C9492130C9492130C9492130C9492133C
:1000B0000C9492130C9492130C9492130C9492132C
:1000C0000C9492130C9492130C9492130C9492131C
:1000D0000C9492130C9492130C9429450C94EA44BA
:1000E0000C949213192D362D672D842D992DC22D28
:1000F0002F2E952E3E2F863394338D33B433B83361
:10010000D2333738E733333465348C34B5340A3579
:100110001B352C353D354E355F353738423737384E
:100120004D37BD37C337E3373BB23EB22DB231B2A4
:1001300037B275B242B246B24CB250B254B25AB2B1
:100140005EB262B275B268B26CB270B23EB543B51F
:1001500048B552B55CB5D5B566B56EB576B580B562
:100160008AB594B5A3B5ADB5D5B5B7B5C1B5CBB561
:10017000084AD73B3BCE016E84BCBFFDC12F3D6C0E
:1001800074319ABD56833DDA3D00C77F11BED9E474
:10019000BB4C3E916BAAAABE000000803F05A84C54
:1001A000CDB2D44EB93836A9020C50B99186880820
:1001B0003CA6AAAA2ABE000000803F004E414E493C
:1001C0004E495459494E46CDCCCC3D0AD7233C1715
:1001D000B7D13877CC2B329595E6241FB14F0A0062
:1001E0000020410000C84200401C4620BCBE4CCA52
:1001F0001B0E5AAEC59D74434F4D4D554E4943415C
:1002000054494F4E0044525952554E004552524F98
:10021000525300494E464F004543484F0047322F46
:1002200047332062616420706172616D657465722C
:10023000730A00206F6620004D424C20473239205F
:10024000706F696E74200059206F7574206F66207E
:1002500072616E67652028312D35292E0A005820DD
:100260006F7574206F662072616E67652028312D6E
:1002700035292E0A004D6573682070726F62696EB1
:100280006720646F6E652E0A005374617274206D6E
:100290006573682070726F62696E67207769746831
:1002A0002022473239205331222066697273742E1E
:1002B0000A004732380A47323920533200537461FA
:1002C00074653A20004D65736820626564206C6532
:1002D00076656C696E6720686173206E6F2064615B
:1002E00074612E0A0053206F7574206F662072614E
:1002F0006E67652028302D35292E0A004D657368FC
:1003000020706F696E742063616E6E6F7420626519
:10031000207265736F6C7665640A00456E642066B2
:10032000696C65206C6973740A00426567696E20A8
:1003300066696C65206C6973740A00286E6F2066AC
:10034000696C6529005344207072696E74696E6728
:10035000206279746520004E6F74205344207072BF
:10036000696E74696E670A0043757272656E7420F7
:1003700066696C653A200046696C652064656C6549
:100380007465643A0044656C6574696F6E206661DB
:10039000696C65642C2046696C653A200025697398
:1003A0000025696D20256973002569682025696D20
:1003B0002025697300256964202569682025696DF9
:1003C00020256973002569792025696420256968DD
:1003D0002025696D20256973005072696E74207440
:1003E000696D653A2000180213020C020502F7013C
:1003F0006F66660044454255473A004B494C4C45B0
:10040000442E20004D3131332053006F6B002C20DF
:10041000002C2000544845524D414C5F50524F54DF
:10042000454354494F4E004155544F5245504F5249
:10043000545F53445F53544154555300454D455206
:1004400047454E43595F5041525345520043415333
:10045000455F4C494748545F4252494748544E45CE
:10046000535300544F47474C455F4C4947485453FA
:1004700000534F4654574152455F504F5745520025
:100480004255494C445F50455243454E54004C45FB
:1004900056454C494E475F44415441005A5F5052C3
:1004A0004F4245004155544F4C4556454C00505223
:1004B000494E545F4A4F420050524F4752455353A2
:1004C000004155544F5245504F52545F54454D5082
:1004D00000564F4C554D45545249430045455052E6
:1004E0004F4D0053455249414C5F584F4E5F584F56
:1004F0004646004649524D574152455F4E414D4593
:100500003A4D61726C696E20312E312E39202847A8
:1005100069746875622920534F555243455F434FB4
:1005200044455F55524C3A68747470733A2F2F6784
:1005300069746875622E636F6D2F4D61726C696EA0
:100540004669726D776172652F4D61726C696E20BC
:1005500050524F544F434F4C5F56455253494F4EA4
:100560003A312E30204D414348494E455F54595051
:10057000453A3344205072696E7465722045585470
:1005800052554445525F434F554E543A31205555CC
:1005900049443A63656465326132662D34316132B3
:1005A0002D343734382D396231322D633535633689
:1005B000326633363766660A002F2F20002054003B
:1005C000205200416363656C65726174696F6E3AB5
:1005D0002050005741524E494E4721204C6F772002
:1005E0005A204A65726B206D6179206C65616420C8
:1005F000746F20756E77616E7465642070617573B9
:1006000065732E0A0020466C6F773A200000013691
:100610003726032BFFFFFF3C3D382AFFFFFFFF2E4D
:10062000303E12FFFFFFFFFFFFFF0809FF2C071AF4
:100630001C18FFFFFF08440A2C4324221E20643AA2
:100640000020693A0020703A00496E76616C696456
:100650002065787472756465720A0043290A006126
:10066000626C656420286D696E2074656D70200071
:10067000436F6C6420657874727564657320617271
:1006800065200020643A0020693A0020703A004E4C
:100690006F2063617365206C696768740A00454563
:1006A00050524F4D204F4B0A00205A004475616C48
:1006B00020456E6473746F702041646A7573746D45
:1006C000656E7420286D6D293A20003F4B207661BD
:1006D0006C7565206F7574206F662072616E67653A
:1006E0002028302D3130292E0A00416476616E6356
:1006F00065204B3D004163746976652045787472CE
:10070000756465723A2000496E76616C6964206593
:10071000787472756465720A0043616E6E6F74203E
:10072000656E746572207375626469723A20004761
:1007300039310A4731205A2D302E30320A473930AC
:10074000005370656369616C204D656E753A205A7F
:1007500020446F776E20302E310A004739310A4726
:1007600031205A2D302E30320A473930005370650F
:100770006369616C204D656E753A205A20446F772D
:100780006E20302E30320A004739310A4731205A64
:100790002B302E30320A473930005370656369615F
:1007A0006C204D656E753A205A20557020302E30E1
:1007B000320A004739310A4731205A2B302E310A8C
:1007C000473930005370656369616C204D656E7503
:1007D0003A205A20557020302E310A0047323920F5
:1007E0005332005370656369616C204D656E753AD4
:1007F000204E657874204D65736820506F696E7463
:100800000A00473239205331005370656369616CC7
:10081000204D656E753A205374617274204D657376
:1008200068204C6576656C696E670A004D3134301E
:1008300020533630005370656369616C204D656EDE
:10084000753A2050726568656174204265640A00DB
:100850004D353031005370656369616C204D656EB4
:10086000753A205265616420454550524F4D0A004B
:100870004D353030005370656369616C204D656E95
:10088000753A205361766520454550524F4D0A0018
:100890004D33303320452D3120533830204338201C
:1008A0005531005370656369616C204D656E753A12
:1008B000204175746F2054756E6520486F746265B1
:1008C00064205069640A004D333033204530205392
:1008D00032333020433820553100537065636961ED
:1008E0006C204D656E753A204175746F2054756E9D
:1008F0006520486F74656E64205049440A003C537B
:1009000070656369616C5F4D656E753E003C537048
:10091000656369616C5F4D656E753E002F002F0049
:100920002F002F2E2E0A002F2E2E002F2E2E003CB1
:100930005370656369616C5F4D656E753E0A003C7E
:100940005370656369616C204D656E753E003C5364
:1009500070656369616C204D656E753E003C526543
:10096000616420454550524F4D3E003C52656164E4
:1009700020454550524F4D3E003C4175746F205408
:10098000756E6520486F74626564205049443E006E
:100990003C4175746F2054756E6520486F746265B4
:1009A00064205049443E003C4175746F2054756E7C
:1009B0006520486F74656E64205049443E003C4198
:1009C00075746F2054756E6520486F74656E642071
:1009D0005049443E003C457869743E003C45786986
:1009E000743E003C5361766520454550524F4D3E64
:1009F000003C5361766520454550524F4D3E003CCA
:100A00004E657874204D65736820506F696E743E32
:100A1000003C4E657874204D65736820506F696E98
:100A2000743E003C5374617274204D657368204CB1
:100A30006576656C696E673E003C53746172742024
:100A40004D657368204C6576656C696E673E003C49
:100A500050726568656174206265643E003C507246
:100A60006568656174206265643E003C5A20446F8D
:100A7000776E20302E313E003C5A20446F776E2036
:100A8000302E313E003C5A20446F776E20302E309D
:100A9000323E003C5A20446F776E20302E30323E7A
:100AA000003C5A20557020302E30323E003C5A20F7
:100AB000557020302E30323E003C5A205570203088
:100AC0002E313E003C5A20557020302E313E0056CB
:100AD000313136004A333320004D3530300A4D3441
:100AE00032302053310A4731205A313020463234D7
:100AF000300A4731205830205930204636303030C7
:100B0000004A3232004A3232004731205A352046FC
:100B10003234300A473120583139302059323020B0
:100B200046363030300A4731205A30204632343091
:100B3000004731205A3520463234300A4731205898
:100B400031393020593139302046363030300A477B
:100B500031205A302046323430004731205A352077
:100B6000463234300A47312058313930205932303A
:100B70002046363030300A4731205A302046323451
:100B800030004739310A4731205A3130204632345B
:100B9000300A4739300A4732380A4732390A473172
:100BA00020583230205932302046363030300A4713
:100BB00031205A302046323430004A3032004A3137
:100BC00032004731205A3130004F4B004731205A14
:100BD00031300047393000473120452569463530EE
:100BE0003000473120452D302E31462569004731F0
:100BF0002045302E31462569004731205A25694667
:100C00002569004731205A2D302E3146256900478D
:100C100031205A302E314625690047312059256947
:100C200046256900473120592D302E31462569006F
:100C300047312059302E314625690047312058254B
:100C40006946256900473120582D302E31462569E7
:100C50000047312058302E31462569004739310090
:100C600047323800473238205A004732382059007E
:100C70004732382058004132305620004731205A40
:100C80003130004A3034004A3231004A3230004BB1
:100C9000494C4C45442E20004A303400454E440017
:100CA000464E20004A3032003939393A3939390054
:100CB0004D0048004137562000413656202D2D2D3D
:100CC000004A30320041365620005A3A2000593A44
:100CD0002000583A2000413556004134562000414A
:100CE0003356200041325620004131562000413019
:100CF0005620004D3834004A3136004A313800471A
:100D000039310A4731205A313020463234300A47CF
:100D10003930004A3134004A3030004A3031004A1C
:100D2000313000656E7175657565696E67202200EA
:100D30004B494C4C45442E20005072696E746572CC
:100D40002073746F707065642064756520746F2003
:100D50006572726F72732E20466978207468652000
:100D60006572726F7220616E6420757365204D39F3
:100D7000393920746F20726573746172742E202863
:100D800054656D7065726174757265206973207247
:100D9000657365742E2053657420697420616674D0
:100DA00065722072657374617274696E67290A00D6
:100DB0004E6F20436865636B73756D207769746847
:100DC000206C696E65206E756D6265722C204C61B9
:100DD0007374204C696E653A20004E6F204368653D
:100DE000636B73756D2077697468206C696E65201C
:100DF0006E756D6265722C204C617374204C696E47
:100E0000653A2000636865636B73756D206D697367
:100E10006D617463682C204C617374204C696E653D
:100E20003A20004C696E65204E756D6265722069CE
:100E300073206E6F74204C617374204C696E652052
:100E40004E756D6265722B312C204C617374204C91
:100E5000696E653A20004D313130004D3331005319
:100E6000442072656164206572726F720A00446F7B
:100E70006E65207072696E74696E672066696C6554
:100E80000A0024F4D43050C38E20C2A24017828BB3
:100E90007011127A910D816CD90AA861E108C758C6
:100EA0006607615143061E4B5D05C145A7041A4103
:100EB0001104093D9803713931034036DB02653373
:100EC0009102D4305402802E1D02632CEE01752A4B
:100ED000C501B028A001102781018F2564012B24B2
:100EE0004B01E0223401AC211F018D200D01801F38
:100EF000FC00841EED00971DDF00B81CD200E61B2D
:100F0000C600201BBC00641AB200B219A8000A195E
:100F1000A0006A189900D117910040178B00B516F0
:100F2000840031167E00B31579003A157300C7149A
:100F30006F0058146A00EE136600881363002513CF
:100F40005E00C7125B006C12570015125400C111ED
:100F5000510070114F0021114B00D61049008D1027
:100F600047004610440002104200C00F4000800FAE
:100F70003E00420F3C00060F3B00CB0E3800930EA4
:100F800037005C0E3500270E3400F30D3200C10D22
:100F90003100900D3000600D2E00320D2D00050D3A
:100FA0002C00D90C2B00AE0C2900850C29005C0C00
:100FB0002700350C27000E0C2600E80B2400C40B7C
:100FC0002400A00B23007D0B23005A0B2100390BBA
:100FD0002100180B2000F80A1F00D90A1E00BB0AC6
:100FE0001E009D0A1D00800A1D00630A1C00470A9E
:100FF0001B002C0A1B00110A1A00F7091A00DD0950
:101000001900C4091900AB091900920917007B09DE
:101010001800630917004C0916003609160020094C
:1010200016000A091500F5081500E0081400CC08A0
:101030001400B8081400A4081400900813007D08D8
:1010400012006B08130058081200460812003408FA
:101050001100230811001208110001081100F00707
:101060001000E0071000D0071000C0071000B00704
:101070000F00A107100091070E0083070F007407EF
:101080000F0065070E0057070E0049070E003B07CB
:101090000D002E070E0020070D0013070D00060798
:1010A0000D00F9060C00ED060D00E0060C00D4065C
:1010B0000C00C8060C00BC060C00B0060C00A40610
:1010C0000B0099060C008D060B0082060B007706BC
:1010D0000B006C060B0061060A0057060B004C065D
:1010E0000A0042060A0038060A002E060A002406F4
:1010F0000A001A060A001006090007060A00FD0584
:101100000900F4050900EB050900E2050900D9050D
:101110000900D0050900C7050900BE050900B5058D
:101120000800AD050800A50509009C050800940508
:1011300008008C050800840508007C05080074057B
:1011400008006C050700650508005D0507005605E9
:1011500008004E0507004705070040050800380550
:101160000700310507002A050700230507001C05B5
:101170000600160507000F05070008050600020512
:101180000700FB040600F5040700EE040600E8046F
:101190000600E2040700DB040600D5040600CF04C5
:1011A0000600C9040600C3040600BD040600B70417
:1011B0000600B1040500AC040600A6040600A00465
:1011C00005009B04060095040500900406008A04AF
:1011D000050085040500800406007A0405007504F6
:1011E0000500700405006B04050066040500610439
:1011F00005005C04050057040500520405004D0479
:10120000050048040500430405003E0404003A04B8
:10121000050035040500300404002C0405002704F3
:101220000400230405001E0404001A04040016042C
:101230000500110404000D04040009040500040461
:10124000040000040400FC030400F8030400F40399
:101250000400F0030400EC030400E8030400E403CA
:101260000400E0030400DC030400D8030400D403FA
:101270000400D0030400CC030400C8030300C5032A
:10128000030024F404D9201BC40C5C0E9804C40988
:101290005F0265077101F405F900FB04B30048041F
:1012A0008700C10369005803550003034500BE02CF
:1012B0003A008402310053022A0029022500040268
:1012C0002000E4011C00C8011900AF0117009801BB
:1012D000140084011300710110006101100051011C
:1012E0000E0043010D0036010B002B010B00200105
:1012F0000B00150109000C01090003010800FB00A7
:101300000800F3000800EB000700E4000600DE0020
:101310000600D8000600D2000600CC000500C70079
:101320000500C2000500BD000400B9000400B500BE
:101330000400B1000400AD000400A9000400A500F1
:101340000300A20003009F0004009B00030098001C
:1013500003009500020093000300900003008D003D
:1013600002008B0003008800020086000200840057
:101370000300810002007F0002007D0002007B006C
:10138000020079000200770001007600020074007C
:10139000020072000100710002006F0002006D0087
:1013A00001006C0002006A00010069000200670091
:1013B0000100660001006500010064000200620097
:1013C000010061000100600001005F0002005D009B
:1013D00001005C0001005B0001005A00010059009F
:1013E000010058000100570001005600010055009F
:1013F000010054000100530000005300010052009E
:10140000010051000100500001004F0001004E009A
:1014100000004E0001004D0001004C0001004B0097
:1014200000004B0001004A00010049000100480093
:10143000000048000100470001004600000046008F
:101440000100450000004500010044000100430088
:101450000000430001004200000042000100410082
:10146000000041000100400001003F0000003F007B
:1014700001003E0000003E0001003D0000003D0074
:1014800001003C0000003C0000003C0001003B006B
:1014900000003B0001003A0000003A000100390062
:1014A000000039000100380000003800000038005A
:1014B0000100370000003700010036000000360050
:1014C0000000360001003500000035000000350046
:1014D000010034000000340000003400010033003B
:1014E0000000330000003300010032000000320031
:1014F0000000320001003100000031000000310026
:1015000001003000000030000000300001002F001A
:1015100000002F0000002F0000002F0001002E000F
:1015200000002E0000002E0001002D0000002D0004
:1015300000002D0000002D0001002C0000002C00F8
:1015400000002C0000002C0001002B0000002B00EC
:1015500000002B0000002B0001002A0000002A00E0
:1015600000002A0000002A000100290000002900D4
:1015700000002900000029000000290001002800C7
:1015800000002800000028000000280000002800BB
:1015900001002700000027000000270000002700AE
:1015A00000002700010026000000260000002600A1
:1015B0000000260000002600010025000000250094
:1015C0000000250000002500000025000000250087
:1015D000010024000000240000002400000024007A
:1015E000000024000100230000002300000023006D
:1015F000000023000000230000002300000023005F
:101600000100220000002200000022000000220051
:101610000000220000002200010021000000210043
:101620000000210000002100000021000000210036
:101630000000210001002000000020000000200028
:10164000000020000000200000002000000020001A
:101650000000200001001F0000001F0000001F000C
:1016600000001F0000001F0000001F0000001F00FE
:1016700001001E0000001E0000001E0000001E00F1
:101680000000C23100001C260000F4190000D80F31
:101690000000EB080000C0040000750200004001DB
:1016A0000000526573656E643A20006F6B00207411
:1016B0006F6F206C6F6E6720657874727573696FD9
:1016C0006E2070726576656E7465640A0020636FC3
:1016D0006C6420657874727573696F6E20707265C2
:1016E00076656E7465640A00627573793A2070617C
:1016F0007573656420666F7220696E7075740A0078
:10170000627573793A2070617573656420666F72D3
:1017100020757365720A00627573793A2070726F72
:1017200063657373696E670A004A3135004B494C33
:101730004C45442E20004B494C4C20636175736529
:1017400064206279204B494C4C20627574746F6E32
:101750002F70696E0A004B494C4C45442E20004BBB
:10176000494C4C2063617573656420627920746F05
:101770006F206D75636820696E616374697665209A
:1017800074696D65202D2063757272656E742063B7
:101790006F6D6D616E643A20004A3131005072699C
:1017A0006E7465722068616C7465642E206B696C60
:1017B0006C28292063616C6C6564210A000000A01C
:1017C000C000000000000000005761726E696E6783
:1017D0003A20486F6D696E672042756D70204469CC
:1017E0007669736F72203C20310A00020204000007
:1017F000A0400000A0400000004000005C4300004A
:10180000574300004E43FFFFFF20746F6F206C6F43
:101810006E6720657874727573696F6E207072657B
:1018200076656E7465640A0020636F6C6420657869
:1018300074727573696F6E2070726576656E74650B
:10184000640A00454550524F4D20646174617369CC
:101850007A65206572726F722E0A00290A00206272
:10186000797465733B2063726320005365747469F7
:101870006E67732053746F726564202800290A0014
:101880002062797465733B20637263200020737457
:101890006F7265642073657474696E677320726516
:1018A00074726965766564202800202863616C6322
:1018B000756C6174656429210A0020213D20004572
:1018C0004550524F4D20435243206D69736D6174F2
:1018D0006368202D202873746F72656429200020AE
:1018E00053697A653A2000496E6465783A20002091
:1018F0004D61726C696E3D563535290A00284545A3
:1019000050524F4D3D00454550524F4D2076657227
:1019100073696F6E206D69736D6174636820000276
:101920004A3135004A3132004A3137002020506CAC
:10193000616E6E6572427566666572427974657332
:101940003A20002046726565204D656D6F72793AC8
:101950002000436F6D70696C65643A204E6F76208D
:10196000313920323031380A00207C2041757468CA
:101970006F723A2028646176696472616D69726F72
:101980002C20666F7220416E7963756269632069ED
:1019900033204D656761290A00323031392D3131EC
:1019A0002D313500204C617374205570646174656D
:1019B000643A2000312E312E390A004D61726C6973
:1019C0006E0020536F66747761726520526573658F
:1019D000740A00205761746368646F6720526573EE
:1019E00065740A002042726F776E206F7574205202
:1019F000657365740A002045787465726E616C20A9
:101A000052657365740A00506F77657255700A00ED
:101A100073746172740A004D3234004D32332025E4
:101A200073006175746F25692E67006572726F723D
:101A30002077726974696E6720746F2066696C65BF
:101A40000A00205A3A0020593A0020583A00656EA0
:101A50006473746F7073206869743A2000446F6E09
:101A60006520736176696E672066696C652E0A0071
:101A70004D3239006F70656E206661696C65642C4B
:101A80002046696C653A200043616E6E6F74206F6A
:101A900070656E2073756264697220004A3035008B
:101AA0004A3233004739310A4731205A2D3130202C
:101AB000463234300A47393000534420636172643F
:101AC000206F6B0A006F70656E526F6F74206661D5
:101AD000696C65640A00766F6C756D652E696E6958
:101AE00074206661696C65640A004572726F723AAF
:101AF00000534420696E6974206661696C0A006550
:101B000063686F3A001000C90210012C01400122E5
:101B10000170011801B0010E01F00104015002FA38
:101B200000B002F0003003E600D003DC009004D2E5
:101B3000007005C800A006BE000008B400B009AAE5
:101B400000D00BA000600E960060118C0000158282
:101B50000020197800C01D6E00A0226400B0275A32
:101B600000902C500000314600E0343C0010383228
:101B700000903A2800603C1E00A03D1400803E0A00
:101B800000203F00002CFFFFFFFFFF0001010101CB
:101B9000016265640A002C2073797374656D20738B
:101BA000746F7070656421204865617465725F4967
:101BB000443A20004265642068656174696E67205C
:101BC0006661696C65640048656174696E6720666A
:101BD00061696C65640045312048656174696E67B0
:101BE000206661696C65640048656174696E672090
:101BF0006661696C65640070012C0190012701B079
:101C0000012201C0011D01F0011801100213013071
:101C1000020E016002090190020401C002FF0000EF
:101C200003FA004003F5008003F000D003EB00202E
:101C300004E6007004E100E004DC004005D700C0C9
:101C400005D2004006CD00D006C8008007C3003092
:101C500008BE00F008B900C009B400B00AAF00B077
:101C60000BAA00D00CA500000EA000500F9B00C0D6
:101C70001096005012910000148C00C0158700B01F
:101C8000178200B0197D00D01B7800001E73004041
:101C9000206E0090226900F024640040275F0090CD
:101CA000295A00E02B5500102E500020304B001018
:101CB000324600E033410090353C00103737007069
:101CC000383200A0392D00B03A2800A03B23006034
:101CD0003C1E00103D1900903D1400103E0F007096
:101CE0003E0A00C03E0500003F0000403FFBFF8071
:101CF0003FF6FFC03FF1FF453120544845524D416A
:101D00004C2052554E4157415900424544205448B9
:101D100045524D414C2052554E415741590054684F
:101D200065726D616C2052756E6177617900453125
:101D3000204572723A204D415854454D500045722D
:101D4000723A204D415854454D5020424544004D73
:101D5000415854454D5020747269676765726564D7
:101D6000004531204572723A204D494E54454D5040
:101D7000004572723A204D494E54454D502042451F
:101D800044004D494E54454D502074726967676553
:101D9000726564004D383420582059205A2045007F
:101DA000202F002042403A0020403A003A00436190
:101DB000703A00205A00205900580020204D6178C8
:101DC0003A2000205A00205900580020204D696E0A
:101DD0003A20004F6E20004F666600536F667420F5
:101DE000656E6473746F70733A20004B6420002337
:101DF000646566696E652044454641554C545F00F4
:101E00004B69200023646566696E65204445464140
:101E1000554C545F004B70200023646566696E6505
:101E20002044454641554C545F005049442041757B
:101E3000746F74756E652066696E69736865642178
:101E40002050757420746865206C617374204B7029
:101E50002C204B6920616E64204B6420636F6E738D
:101E600074616E74732066726F6D2062656C6F773B
:101E700020696E746F20436F6E6669677572617456
:101E8000696F6E2E680A00504944204175746F7462
:101E9000756E65206661696C6564212074696D6585
:101EA0006F75740A00453120544845524D414C200D
:101EB00052554E41574159004245442054484552DD
:101EC0004D414C2052554E4157415900546865725E
:101ED0006D616C2052756E617761790045312048E3
:101EE000656174696E67206661696C65640042654E
:101EF000642068656174696E67206661696C6564F9
:101F00000048656174696E67206661696C6564008C
:101F1000504944204175746F74756E65206661691F
:101F20006C6564212054656D7065726174757265AD
:101F300020746F6F20686967680A00204B643A203C
:101F400000204B693A2000204B703A20000A2043C1
:101F50006C617373696320504944200A00205475F2
:101F60003A2000204B753A2000206D61783A20001D
:101F7000206D696E3A200020643A20002062696179
:101F8000733A2000504944204175746F74756E6532
:101F9000206661696C656421204261642065787403
:101FA0007275646572206E756D6265720A005049C3
:101FB00044204175746F74756E652073746172741A
:101FC0000A004F66660A00466164652048656967D5
:101FD00068742000426564204C6576656C696E67A4
:101FE00020004661696C656420746F20656E6162D3
:101FF0006C6520426564204C6576656C696E670A85
:10200000004D65736820426564204C6576656C20E0
:10201000646174613A0A004D65736820706F696E7F
:10202000742063616E6E6F74206265207265736FD9
:102030006C7665640A004D34323120696E636F72CC
:102040007265637420706172616D6574657220756C
:10205000736167650A002066697273740A005A002A
:1020600059005800486F6D652000546F6F206661FD
:10207000722066726F6D207265666572656E63654B
:1020800020706F696E740A007C3C3E5E2B3D3F2FD2
:102090005B5D3B2C2A225C0020496E76616C696492
:1020A00020657874727564657220000000A0C0001D
:1020B00000000000000000000057430000574300EC
:1020C000004E43486F6D696E67206661696C656498
:1020D00000206E6F7420656E74657265642E0A0050
:1020E00050726F7465637465642050696E0A004AAB
:1020F0003036004A3034004A30370020573A004A20
:102100003038004A30390020573A00205A3A00202F
:10211000593A0020436F756E7420583A0020453AB2
:1021200000205A3A0020593A00583A004861726437
:10213000636F6465642044656661756C74205365E3
:102140007474696E6773204C6F616465640A00B8CB
:102150000B0000B80B00003C00000010270000003E
:1021600000FA430000FA430000C040000070420043
:1021700000A0420000A0420000C843E17AD2422001
:10218000286D6D290020204D393030204B004C69DE
:102190006E65617220416476616E63653A0A002063
:1021A000440020490020204D33303420500020448A
:1021B0000020490020204D33303120500050494448
:1021C0002073657474696E67733A0A00205A0020A0
:1021D000204D36363600456E6473746F702061642E
:1021E0006A7573746D656E743A0A00205A0020593E
:1021F000002020473239205333205800205A002035
:10220000204D3432302053004D65736820426564A0
:10221000204C6576656C696E673A0A00205A00208A
:10222000590020204D323036205800486F6D65200F
:102230006F66667365743A0A00204500205A0020D4
:10224000590020580020540020530020204D3230E7
:102250003520510020453C6D61785F655F6A65728D
:102260006B3E0020583C6D61785F785F6A65726BE9
:102270003E20593C6D61785F795F6A65726B3E20E4
:102280005A3C6D61785F7A5F6A65726B3E004164AB
:1022900076616E6365643A20513C6D696E5F73656B
:1022A000676D656E745F74696D655F75733E20530D
:1022B0003C6D696E5F66656564726174653E20544D
:1022C0003C6D696E5F74726176656C5F66656564AE
:1022D000726174653E0020540020520020204D326F
:1022E0003034205000416363656C65726174696FBE
:1022F0006E2028756E6974732F7332293A20503C12
:102300007072696E745F616363656C3E20523C72EB
:102310006574726163745F616363656C3E20543CF5
:1023200074726176656C5F616363656C3E0A002060
:102330004500205A0020590020204D3230312058CD
:10234000004D6178696D756D20416363656C6572E0
:102350006174696F6E2028756E6974732F733229EA
:102360003A0A00204500205A0020590020204D3212
:1023700030332058004D6178696D756D2066656554
:102380006472617465732028756E6974732F732984
:102390003A0A00204500205A0020590020204D39DB
:1023A0003220580053746570732070657220756E0A
:1023B00069743A0A0020204D3230302044300A003F
:1023C00020204D3230302044002044697361626C1B
:1023D00065640A0046696C616D656E74207365748E
:1023E00074696E67733A0020204732312020202024
:1023F0003B00545249474745524544006F70656E53
:10240000003A20007A325F6D696E007A5F6D696E06
:1024100000795F6D696E00785F6D696E005265705E
:102420006F7274696E6720656E6473746F70207369
:1024300074617475730A000A4D6561737572656421
:1024400020706F696E74733A0A005A206F66667363
:1024500065743A20004E756D20582C593A20352C61
:10246000350A004572726F722077726974696E67FF
:1024700020746F20454550524F4D210A0000002125
:1024800000240027002A002D003000330001010045
:1024900000040107010A0100002200250028002B8A
:1024A000002E003100340002010000050108010B7C
:1024B00001000020002300260029002C002F0032FC
:1024C00000000100000301060109010505050507DB
:1024D0000508080808020202020A0A08080404049F
:1024E00004010101010101010103030303030303CB
:1024F00003040707070C0C0C0C0C0C0C0C0202025A
:102500000206060606060606060B0B0B0B0B0B0B4C
:102510000B010210202008081020401020408002EB
:102520000102010804020101020408102040808019
:10253000402010080402018004020180402010089D
:102540000402010804020101020408102040800175
:102550000204081020408000000A0B02090C0D0E36
:102560000807030401000000000000000000000054
:10257000000000000000000000000000000000005B
:102580000000001211100000000000000000000018
:1025900000000000000000000000000000556E6B0D
:1025A0006E6F776E20636F6D6D616E643A202200EE
:1025B0000000484200004842000080400000000047
:1025C00057726974696E6720746F2066696C653A2A
:1025D00020006F70656E206661696C65642C204612
:1025E000696C653A20006F70656E206661696C6584
:1025F000642C2046696C653A200046696C6520733E
:10260000656C65637465640A002053697A653A20D5
:102610000046696C65206F70656E65643A20002025
:1026200066696C653A2000646F696E670066726562
:102630007368004E6F772000454E44205355425238
:102640004F5554494E450A002220706F73002220D6
:10265000706172656E743A2200535542524F555460
:10266000494E452043414C4C207461726765743A71
:1026700022004B494C4C45442E2000747279696EFF
:102680006720746F2063616C6C207375622D6763C3
:102690006F64652066696C6573207769746820745F
:1026A0006F6F206D616E79206C6576656C732E207E
:1026B0004D4158206C6576656C2069733A00A8C25C
:1026C000E8BC11241FBECFEFD1E2DEBFCDBF00E0DA
:1026D0000CBF14E0A0E0B2E0E4EEF0EA01E00BBFD2
:1026E00002C007900D92AC30B107D9F727E1ACE0FA
:1026F000B4E001C01D92AB32B207E1F713E1C0E6CE
:10270000D3E100E006C021970109802FFE010E945D
:10271000CACFCF35D10780E00807A9F70E9409BDCD
:102720000C9461D00C9400002F923F924F925F92D4
:102730006F927F928F929F92AF92BF92CF92DF92D1
:10274000EF92FF920F931F93CF93DF93CDB7DEB736
:10275000CB56D1090FB6F894DEBF0FBECDBF91E0C6
:1027600090932B0B8091E0168D3411F40C94581D2E
:10277000843511F40C943F2A873411F00C948B2A81
:102780002090DE163090DF162CE12216310409F479
:102790003EC6A4F444E0241631044CF452E025165D
:1027A00031040CF046C037FE3DC00C94541D64E06B
:1027B0002616310409F4ECC50C94541D7AE527164D
:1027C000310411F40C948D1C6CF49DE12916310434
:1027D00009F422C6AAE22A16310411F40C94021C50
:1027E0000C94541DBBE52B16310411F40C94911C70
:1027F000ECE52E16310411F00C94541D9FE4292EA3
:1028000092E0392E29E3E22E2BE0F22E69E274E009
:1028100079AF68AF3CE0C32E34E0D32E00E010E087
:102820000C94D01C8091410281110C94922A0C943A
:102830008D2A80914102882311F40C948D2A0E94E4
:102840000E9B82E50E945C40882309F450C10E94DF
:10285000DC3F4B015C0120E030E0A9010E9488C808
:10286000882309F474C12091290430912A044091ED
:102870002B0450912C0428AF39AF4AAF5BAF409185
:102880002D0450912E0460912F04709130044CAFB0
:102890005DAF6EAF7FAF6091460B7091470B80913B
:1028A000480B9091490B2C966CAF7DAF8EAF9FAFCC
:1028B0002C9780914A0B90914B0BA0914C0BB091AF
:1028C0004D0B28968CAF9DAFAEAFBFAF28972C961F
:1028D0002CAD3DAD4EAD5FAD2C9768AD79AD8AADF9
:1028E0009BAD0E9488C881110FC028962CAD3DADCC
:1028F0004EAD5FAD28976CAD7DAD8EAD9FAD0E94A6
:1029000088C8882309F423C111E092E02916310414
:1029100009F010E020E030E0A901C501B4010E94F7
:1029200088C8881F8827881F181759F020E030E0D2
:1029300040E85FEB64962CAF3DAF4EAF5FAF64975E
:102940000AC040E050E060E87FE364964CAF5DAFC2
:102950006EAF7FAF649728AD39AD4AAD5BAD2C96B5
:102960006CAD7DAD8EAD9FAD2C970E94B1CC6096C5
:102970006CAF7DAF8EAF9FAF60972CAD3DAD4EADD0
:102980005FAD28966CAD7DAD8EAD9FAD28970E9452
:10299000B1CC6B017C0160962CAD3DAD4EAD5FAD11
:1029A0006097CA01B9010E94EDC82B013C01A70143
:1029B0009601C701B6010E94EDC89B01AC01C3019D
:1029C000B2010E94B2CC0E941DCF24966CAF7DAFA5
:1029D0008EAF9FAF249720E030E040E05FE30E949D
:1029E000EDC82B013C01A5019401C501B4010E9471
:1029F000EDC84B015C01A3019201C301B2010E9429
:102A0000EDC89B01AC01C501B4010E94B1CC0E948C
:102A10001DCF64962CAD3DAD4EAD5FAD64970E9469
:102A2000EDC84B015C01C701B601905824962CAD4E
:102A30003DAD4EAD5FAD24970E948ECDA5019401B2
:102A40000E94EDC86B017C012C962CAD3DAD4EADC6
:102A50005FAD2C9768AD79AD8AAD9BAD0E94B2CCCD
:102A600020E030E040E05FE30E94EDC89B01AC0154
:102A7000C701B6010E94B2CC28AD39AD4AAD5BADFD
:102A80000E94B1CC6B017C0128962CAD3DAD4EADC2
:102A90005FAD28976CAD7DAD8EAD9FAD0E94B2CC81
:102AA00020E030E040E05FE30E94EDC82B013C01F4
:102AB00024962CAD3DAD4EAD5FAD249760966CADC8
:102AC0007DAD8EAD9FAD60970E948ECDA501940126
:102AD0000E94EDC89B01AC01C301B2010E94B2CCBF
:102AE0002CAD3DAD4EAD5FAD0E94B1CC14C089E4BC
:102AF0000E945C40882329F00E94DC3F6B017C012E
:102B000003C0C12CD12C76018AE40E945C4088234A
:102B100009F10E94DC3F2C966CAF7DAF8EAF9FAF6A
:102B20002C9720E030E0A901C701B6010E9488C8B7
:102B300081111FC020E030E0A9012C966CAD7DAD65
:102B40008EAD9FAD2C970E9488C8811112C0EAEE0D
:102B5000FAE10AC420E030E0A901C701B6010E94F1
:102B600088C88823A1F32C961CAE1DAE1EAE1FAEE6
:102B70002C97C701B601905868AF79AF8AAF9BAF69
:102B80002C968CAD9DADAEADBFAD2C97B0588CAF33
:102B90009DAFAEAFBFAF28AD39AD4AAD5BADCA0199
:102BA000B9010E94EDC84B015C012CAD3DAD4EADAD
:102BB0005FADCA01B9010E94EDC89B01AC01C5011E
:102BC000B4010E94B2CC0E941DCFA0966CAF7DAF25
:102BD0008EAF9FAFA0972091290430912A04409195
:102BE0002B0450912C0428962CAF3DAF4EAF5FAF15
:102BF0002897A701960128966CAD7DAD8EAD9FAD4F
:102C000028970E94B2CC64966CAF7DAF8EAF9FAF19
:102C1000649740912D0450912E0460912F0470917F
:102C2000300460964CAF5DAF6EAF7FAF60972C966F
:102C30002CAD3DAD4EAD5FAD2C9760966CAD7DADCE
:102C40008EAD9FAD60970E94B2CCA4966CAF7DAF65
:102C50008EAF9FAFA4976091460B7091470B809108
:102C6000480B9091490B68966CAF7DAF8EAF9FAFCC
:102C7000689764962CAD3DAD4EAD5FAD64970E94F4
:102C8000B1CC6B017C0180914A0B90914B0BA091D0
:102C90004C0BB0914D0B6C968CAF9DAFAEAFBFAFF0
:102CA0006C97A4962CAD3DAD4EAD5FADA497BC0125
:102CB000CD010E94B1CC4B015C01209131043091D7
:102CC00032044091330450913404A8962CAF3DAFA8
:102CD0004EAF5FAFA89760914E0B70914F0B8091F4
:102CE000500B9091510B0E94B1CC24966CAF7DAFEC
:102CF0008EAF9FAF2497A701960168AD79AD8AADDD
:102D00009BAD0E94EDC82B013C01A50194016CAD67
:102D10007DAD8EAD9FAD0E94EDC89B01AC01C3019E
:102D2000B2010E94B2CC2B013C01A501940168AD17
:102D300079AD8AAD9BAD0E94EDC84B015C01A70146
:102D400096016CAD7DAD8EAD9FAD0E94EDC89B012F
:102D5000AC01C501B4010E94B1CCA30192010E9453
:102D600025CD6B017C0120E030E0A9010E9488C8DC
:102D700087FF0AC02BED3FE049EC50E4C701B601E4
:102D80000E94B2CC6B017C0132E02316310451F475
:102D90002BED3FE049EC50E4C701B6010E94B1CCF5
:102DA0006B017C0120E030E0A901C701B6010E945F
:102DB00088C8811128C068962CAD3DAD4EAD5FAD81
:102DC000689728966CAD7DAD8EAD9FAD28970E941B
:102DD00088C8811118C06C962CAD3DAD4EAD5FAD6D
:102DE0006C9760966CAD7DAD8EAD9FAD60970E9487
:102DF00088C8811108C01BEDC12E1FE0D12E19EC2F
:102E0000E12E10E4F12EA7019601A0966CAD7DADE8
:102E10008EAD9FADA0970E94EDC84B015C0120E0F4
:102E200030E0A90124966CAD7DAD8EAD9FAD2497A9
:102E30000E9488C88823E9F0A5019401C501B40166
:102E40000E94EDC84B015C0124962CAD3DAD4EAD0A
:102E50005FAD2497CA01B9010E94EDC89B01AC0186
:102E6000C501B4010E94B2CC0E941DCF4B015C0190
:102E70000DC020E030E0A901C501B4010E94D8CE08
:102E800087FF04C0B7FAB094B7F8B0942FE632E1E8
:102E900043E85AE3C501B4010E9488C887FF02C015
:102EA0000C948D2AC501B4010E9427CE0E94FBCD4F
:102EB0002E967FAF6EAF2E97672B31F441E050E036
:102EC0002E965FAF4EAF2E9740903504509036044B
:102ED00060903704709038042E96AEADBFAD2E973B
:102EE000BD0180E090E00E948CC84B015C019B0119
:102EF000AC01C701B6010E948ECD28966CAF7DAFA4
:102F00008EAF9FAF2897A501940124966CAD7DAD3F
:102F10008EAD9FAD24970E948ECDA0966CAF7DAFF5
:102F20008EAF9FAFA097A30192016091520B709159
:102F3000530B8091540B9091550B0E94B1CCA5017D
:102F400094010E948ECDAC966CAF7DAF8EAF9FAFDB
:102F5000AC9728962CAD3DAD4EAD5FAD2897CA011C
:102F6000B9010E94EDC820E030E040E05FE30E943C
:102F7000EDC89B01AC0160E070E080E89FE30E9437
:102F8000B1CC68966CAF7DAF8EAF9FAF6897A896B7
:102F90002CAD3DAD4EAD5FADA89729873A874B87E5
:102FA0005C874D865E866F86788A6091020270919A
:102FB0000302072E000C880B990B0E948EC82091EB
:102FC0004B0230914C0240914D0250914E020E94B2
:102FD000EDC82AE037ED43E25CE30E94EDC86CAB3C
:102FE0007DAB8EAB9FAB0E9416B69B01AC01285304
:102FF0003F4F4F4F5F4F6C962CAF3DAF4EAF5FAF23
:103000006C9748AC59AC6AAC7BAC22242394312C2D
:1030100039E121963FAF21972E964EAD5FAD2E97A9
:103020004215530509F44DC10E949A820E9416B6BA
:10303000DC01CB016C962CAD3DAD4EAD5FAD6C9718
:10304000821B930BA40BB50BB7FD10C00E9416B6E4
:103050009B01AC0128533F4F4F4F5F4F6C962CAFF5
:103060003DAF4EAF5FAF6C970E94B95121963FAD17
:103070002197315021963FAF2197332309F445C062
:103080002CAD3DAD4EAD5FAD68966CAD7DAD8EADFA
:103090009FAD68970E94EDC86B017C019201A3016E
:1030A00028966CAD7DAD8EAD9FAD28970E94EDC882
:1030B000A70196010E94B2CC7B018C019201A30171
:1030C00068966CAD7DAD8EAD9FAD68970E94EDC8E2
:1030D0004B015C012CAD3DAD4EAD5FAD28966CADA6
:1030E0007DAD8EAD9FAD28970E94EDC89B01AC01D0
:1030F000C501B4010E94B1CC2B013C01C701D8012C
:103100008CAF9DAFAEAFBFAF55C0B10180E090E0D6
:103110000E948CC828962CAD3DAD4EAD5FAD289772
:103120000E94EDC84B015C010E948BCD6B017C01BC
:10313000C501B4010E9413CF4B015C01A7019601A8
:1031400068AD79AD8AAD9BAD0E94EDC82B013C0105
:103150002C962CAD3DAD4EAD5FAD2C97C501B401A5
:103160000E94EDC8A30192010E94B2CC2B013C0148
:10317000A501940168AD79AD8AAD9BAD0E94EDC803
:103180004B015C012C962CAD3DAD4EAD5FAD2C9747
:10319000C701B6010E94EDC89B01AC01C501B40195
:1031A0000E94B1CC6CAF7DAF8EAF9FAF49E121964D
:1031B0004FAF21979201A30164966CAD7DAD8EADAA
:1031C0009FAD64970E94B2CC69837A838B839C8382
:1031D0002CAD3DAD4EAD5FADA4966CAD7DAD8EAD6D
:1031E0009FADA4970E94B2CC6D837E838F83988716
:1031F000A0962CAD3DAD4EAD5FADA09769857A85AB
:103200008B859C850E94B2CC69877A878B879C8747
:10321000AC962CAD3DAD4EAD5FADAC976D857E856A
:103220008F8598890E94B2CC6D877E878F87988B17
:1032300080912102882321F0CE0101960E94844FC3
:10324000E0902A0B1CA61DA61EA61FA689819A81A6
:10325000AB81BC8188A399A3AAA3BBA38D819E81C6
:10326000AF81B8858CA39DA3AEA3BFA389859A85A2
:10327000AB85BC8588A799A7AAA7BBA7AE01485D67
:103280005F4FBE016C5D7F4FCE0180960E94E8AA21
:10329000BE01645D7F4F6B018E010C5C1F4F9E0170
:1032A000235F3F4FAE01485D5F4F68507109CE010B
:1032B00080960E94B559882321F07FEF271A370A9C
:1032C000ABCEE0902A0B18AA19AA1AAA1BAA8091C1
:1032D000460B9091470BA091480BB091490B88A3E6
:1032E00099A3AAA3BBA380914A0B90914B0BA091E9
:1032F0004C0BB0914D0B8CA39DA3AEA3BFA38091AB
:103300004E0B90914F0BA091500BB091510B88A791
:1033100099A7AAA7BBA7AE01485D5F4FBE016C5D30
:103320007F4FCE0180960E94E8AACE01C0966C0124
:103330008E010C5C1F4F22E53BE0AE01485D5F4F04
:10334000BE016C5D7F4F40970E94B55980E1E6E475
:10335000FBE0A9E2B4E001900D928A95E1F70C94AC
:103360008D2A0E947840F80184918F010F5F1F4FD2
:103370008111F7CFEDE1F2E084918F010F5F1F4FD4
:10338000882311F40C948D2A0E947840F801F4CF20
:1033900080E50E945C40882379F080911804909128
:1033A0001904009749F04AE050E060E070E00E94A4
:1033B00007C76B017C0103C0C12CD12C760183E5CA
:1033C0000E945C40882361F00E94DC3F20E030E0F6
:1033D0004AE754E40E94EDC80E94FBCD6B017C01DA
:1033E0000E94D8690E9416B6C60ED71EE81EF91EA6
:1033F0000E9416B6DC01CB018C199D09AE09BF09EC
:10340000B7FD02C00C948D2A0E94B951F1CF80E023
:103410000E94AE9C0C948D2A83E50E945C40882318
:1034200021F10E94BC3F182F863070F0E5EEF2E0EB
:1034300084918F010F5F1F4F882311F40C948D2A04
:103440000E947840F801F4CF833009F44AC130F487
:10345000813091F1823009F43FC008C0843009F412
:103460009FC1853009F4ACC101C010E00E94619C8D
:10347000811103C0E5ECF2E013C08091A716882308
:1034800019F06BE073E002C06FE073E08DEB92E047
:103490000E94024F8AE00E9478400E9422AB96C1AF
:1034A00084917F019FEFE91AF90A882309F48EC1FC
:1034B0000E947840F701F4CF0E94D5AB1092010230
:1034C0001092000282EB92E09093680D8093670D5A
:1034D0000E94A4400C948D2A8091000290910102D8
:1034E00097FF0EC0E9E8F2E084918F010F5F1F4F54
:1034F000882311F40C948D2A0E947840F801F4CFAF
:103500000097A1F48091210280931F0419821A82EE
:103510001B821C8218A219A21AA21BA2BE016F5FF5
:103520007F4FCE0180960E9481B327C0815065E015
:103530000E947ACF80FF03C024E0291B922FA5E0D0
:103540009A02F0011124E80FF11D87FDFA95EE0FA4
:10355000FF1FEE0FFF1FE15DF94E80913104909146
:103560003204A0913304B091340480839183A28308
:10357000B38380911F048093210280910002909177
:103580000102893191050CF067C0109221029C0163
:103590002F5F3F4F309301022093000265E00E94AD
:1035A0007ACF80FF03C024E0291B922F4091310481
:1035B00050913204609133047091340448A359A3AC
:1035C0006AA37BA319821A821B821C82B4E08B023D
:1035D00090011124F901E355F04F4F012081318111
:1035E00042815381F4E09F02C0011124BC016F535A
:1035F000704F5B01DB016D917D918D919C91FE017E
:1036000031966F01E12CF12C00EA10E40E94B1B276
:1036100019821A821B821C82B601CE0180960E94FA
:1036200081B3F50180819181A281B38180932904C6
:1036300090932A04A0932B04B0932C04F40180816E
:103640009181A281B38180932D0490932E04A09345
:103650002F04B0933004BCC080E090E0A0EAB0E456
:103660008093310490933204A0933304B0933404D4
:103670000E949B9D0E94D8698FEF9FEF909301025B
:1036800080930002E5E7F2E084918F010F5F1F4F06
:10369000882321F00E947840F801F6CF83E992E078
:1036A0009A83898304E610E019A308A3BE016F5F23
:1036B0007F4FCE0180960E9434B48AEB92E09A83C9
:1036C000898319A308A3BE016F5F7F4FCE01809647
:1036D0000E9434B481E00E94AE9C81E00E948E9CE6
:1036E00077C088E50E945C408823A1F00E94AC3F2F
:1036F0001FEF160F1530A8F0EEE5F2E084918F0170
:103700000F5F1F4F882311F40C948D2A0E9478407C
:10371000F801F4CF88E50E9478400E9479C40C94A7
:103720008D2A89E50E945C408823A1F00E94AC3F6D
:103730000FEF060F0530A8F0E7E4F2E084918F0167
:103740000F5F1F4F882311F40C948D2A0E9478403C
:10375000F801F4CF89E50E9478400E9479C40C9466
:103760008D2A8AE50E945C40882399F00E94DC3F04
:1037700025E0129FF0011124E00FF11DEE0FFF1F55
:10378000EE0FFF1FE15DF94E6083718382839383A7
:1037900035C08AE50E9478400E9479C40C948D2A35
:1037A0008AE50E945C408823A1F30E94DC3F60937D
:1037B0002B1670932C1680932D1690932E161EC0E8
:1037C00080E00E948E9C0E94D5AB18C01230B1F4EC
:1037D00060910002709101026931710514F069E194
:1037E00070E088E392E00E94E94E69E170E083E3D3
:1037F00092E00E94E94E8AE00E9478400E94699817
:103800000C948D2A80914102882311F40C948D2A06
:1038100089E40E945C40E82E882321F00E94AC3F9E
:10382000062F01C000E08AE40E945C40F82E882345
:1038300021F00E94AC3F162F01C010E0EE2011F0E5
:10384000053020F4FF2081F0153070F0ECEFF2E04D
:1038500084918F010F5F1F4F882311F40C948D2AE0
:103860000E947840F801F4CF0E946E40EE2091F063
:1038700034E00302F0011124EF53F04F8081918175
:10388000A281B3818093460B9093470BA093480B82
:10389000B093490BFF2091F044E01402F001112491
:1038A000E355F04F80819181A281B38180934A0BCF
:1038B00090934B0BA0934C0BB0934D0B80E50E9463
:1038C0005C40882319F00E94CD3F03C080E50E9430
:1038D000134086E40E945C408823D9F00E94DC3FBC
:1038E0006B017C0120E030E0A9010E94D8CE1816BF
:1038F00084F420E030E040E752E4C701B6010E94C2
:103900008ECD60934B0270934C0280934D02909346
:103910004E020E9479550C948D2A10921E040C942C
:103920008D2A90931E040C948D2A0E94DC3F2B015B
:103930003C01133049F0F6012081318142815381ED
:103940000E94B1CC2B013C01A8ADB9AD2D913D91A8
:103950004D915C91C301B2010E94B1CC4B015C015D
:103960002DEB37E346E855EB0E94D8CE87FD20C00B
:103970002DEB37E346E855E3C501B4010E9488C842
:103980001816B4F01F5FB4E0EB0EF11CE8ADF9AD12
:103990003496F9AFE8AFF4E0CF0ED11C143039F112
:1039A000D1018D911D010E945C40882359F3BDCF48
:1039B000133051F44092350450923604609237042B
:1039C0007092380401E0DECFA5019401F701608117
:1039D0007181828193810E94B2CCD7016D937D93D6
:1039E0008D939C931397812F0E94F29DCBCF002340
:1039F00009F404CFC0903504D0903604E090370429
:103A0000F090380420E030E0A901C701B6010E941F
:103A1000B2CC209121173091221740912317509159
:103A200024170E94EDC80E94E3CE6093A90F709303
:103A3000AA0F8093AB0F9093AC0FC092990FD092C6
:103A40009A0FE0929B0FF0929C0F9091770F8091CC
:103A5000780F981719F00E947A69D0CE0E94D86921
:103A600080916F00982F927081FF05C080916F0048
:103A70008D7F80936F004091A90F5091AA0F6091A4
:103A8000AB0F7091AC0F40939D1550939E156093B2
:103A90009F157093A015992309F4B0CE80916F0003
:103AA000826080936F00AACE0E9468B40C948D2A25
:103AB0008091DE169091DF168637910509F4AAC72A
:103AC0000CF0CEC08D34910509F4D1C40CF05AC06D
:103AD0008A31910509F43DC264F58531910509F4F7
:103AE000F6C1C4F48231910509F432C684319105DE
:103AF00009F4ADC1419711F00C943C2A5F988A9863
:103B00004798809108018170809306014798129828
:103B10000C948D2A8731910509F4E3C10CF4DBC1C3
:103B20008831910509F4F3C1499709F4FBC10C945C
:103B30003C2A8F31910509F49AC384F48C319105A4
:103B400009F4ADC20CF413C28D31910511F40C943B
:103B50008D2A4E9709F4ADC20C943C2A8A32910505
:103B600009F438C42CF4809709F435C30C943C2A2A
:103B70008B34910509F462C48C34910509F462C454
:103B80000C943C2A8B36910509F4B4C50CF042C064
:103B90008535910509F40BC6FCF48235910509F4CD
:103BA000D0C584F48135910511F00C943C2A0E9413
:103BB000DA7F0E9493A610923A041092390400E032
:103BC00010E0A8C58335910509F4BEC5843591057B
:103BD00009F4BEC50C943C2A8836910509F44BC4FF
:103BE0007CF48C35910511F00C943C2AFFE4CF2E27
:103BF000F2E0DF2EA5E1EA2EA7E1FA2E10E0F0C5F3
:103C00008936910509F4FAC48A36910509F456C536
:103C10000C943C2A8037910509F4BFC484F48D3696
:103C2000910509F42BC50CF4B5C48E36910509F441
:103C30004BC48F36910509F45AC40C943C2A823740
:103C4000910509F44DC60CF4AFC48337910509F40E
:103C5000FBC08537910511F40C948D2A0C943C2AF5
:103C60008E3221E0920711F40C9478280CF06EC08B
:103C70008B3C910509F48CC7ACF58C38910509F49F
:103C800000C58CF48837910509F413C70CF40EC7EE
:103C90008937910511F00C943C2A1092D40B1092A4
:103CA000D30B0C948D2A8E3B910509F404C534F492
:103CB0008B39910509F4BDC40C943C2A883C9105CC
:103CC00009F4FDC6893C910511F00C943C2A7FE46F
:103CD000E72E72E0F72E05EF16E1E5E0CE2EE7E1E4
:103CE000DE2E3DC78C3D910511F40C940C27A4F4F5
:103CF0008D3C910509F4DDC70CF466C78E3C910537
:103D000011F40C94E626833D910511F00C943C2AA5
:103D10000E94CF8F0C948D2A823E910511F40C9451
:103D200086273CF48D3D910511F40C9419270C94D1
:103D30003C2A8C3241E0940711F40C94AF278D3269
:103D4000914011F40C94D8270C943C2A853F61E0F3
:103D5000960711F40C946529E4F58A39A1E09A07D5
:103D600009F41FC4BCF48033E1E09E0711F40C9405
:103D7000CF2814F40C94CC28833621E0920709F460
:103D80005FC08039914011F00C943C2A0E94D869A0
:103D90000C948D2A853A41E0940711F40C94622921
:103DA0004CF4843A914011F00C943C2A0E946A88A9
:103DB0000C948D2A8C3A71E0970711F40C94092722
:103DC000843F914011F00C943C2A0E941F700C9487
:103DD0008D2A8A39B2E09B0711F40C94A429B4F41B
:103DE000873FF1E09F0711F40C946B2914F40C94B5
:103DF0006829883F31E0930711F40C9477298C30BF
:103E0000924011F40C949B290C943C2A8B3853E07B
:103E1000950711F40C948D2A3CF48438934011F4E6
:103E20000C94D1290C943C2A803AA3E09A0709F417
:103E300011C2873E934011F40C94292A0C943C2A19
:103E4000EAEEFAE10C944F29E3EFF4E088C5EAE2E8
:103E5000F3E084918F010F5F1F4F882321F00E94B0
:103E60007840F801F6CF1092731286E290E10E943A
:103E700046938BE1E6E2F0E1DE01159601900D92AA
:103E80008A95E1F780912410909125109C838B8373
:103E900085EE92E09A83898340E050E0BE016F5F37
:103EA0007F4F80E090E00E945479CE0101960E94FD
:103EB0004F51EBE1F3E084918F010F5F1F4F882397
:103EC00011F40C948D2A0E947840F801F4CF0E94DE
:103ED00023770C948D2A1092F50F1092F60F0C9404
:103EE0008D2AE091DC16F091DD168081882329F07F
:103EF000803209F410823196F8CF40E061E0809181
:103F0000DC169091DD160E947EB60C948D2A80916D
:103F1000F60F882319F081E08093F50F0E94A37FAC
:103F20000C948D2A1092F50F8091A515813011F017
:103F30000C948D2A82E08093A5150E9416B660939A
:103F4000A1157093A2158093A3159093A4150C94BA
:103F50008D2A8091F60F882311F40C948D2A83E525
:103F60000E945C4081110C94972A0C948D2A83E462
:103F70000E941340882309F450C0E8E6F3E08491DE
:103F80008F010F5F1F4F882321F00E947840F801B6
:103F9000F6CF8091C111811103C0EBE3F3E012C0B1
:103FA000BE016F5F7F4F8EEB91E10E940E928E01FA
:103FB0000F5F1F4FF80181918F01882349F10E9403
:103FC0007840F8CF84918F010F5F1F4F882301F154
:103FD0000E947840F801F6CFB6EECB2EB3E0DB2E90
:103FE000E12CF12C20E08091BD0B90E00E2C02C062
:103FF000959587950A94E2F780FDA9C29FEFE91A8B
:10400000F90AA2E0CA0ED11CB5E0EB16F10459F78B
:104010008AE00E9478400C948D2A8091F60F8823C4
:1040200039F08091F50F882319F0E5E4F3E003C03F
:10403000E7E5F3E028C084918F010F5F1F4F8823CD
:1040400021F00E947840F801F6CF60916F127091D4
:10405000701280917112909172124AE00E94944302
:104060008FE20E94784060916B1270916C12809187
:104070006D1290916E124AE00E9494438AE00E9471
:1040800078400C948D2A84918F010F5F1F4F8823F5
:1040900011F40C948D2A0E947840F801F4CF40E08E
:1040A00060E08091DC169091DD160E947EB60C9443
:1040B0008D2A8091F60F882311F40C948D2A8EEBB3
:1040C00091E10E945FB08EEB91E10E94E991109224
:1040D000F40F1092F30F8091F60F882311F40C94D3
:1040E0008D2A0091DC161091DD160E944779B801E7
:1040F000CE0180960E945B7B8C01892B11F40C947D
:104100008D2A68A179A16115710511F06C5F7F4F4F
:1041100019821C8222E0A801CE0101960E947C97A0
:10412000811102C0F12C14C0CE0101960E94B57815
:104130008823C1F361E0CE0101960E94F2910097BD
:1041400089F325EEDC012C931C820E9408AEF82E28
:10415000CE0101960E946840F11003C0E5E8F3E04B
:1041600022C0E7E7F3E084917F01BFEFEB1AFB0A7F
:10417000882321F00E947840F701F5CFF801819162
:104180008F01882319F00E947840F8CF8AE00E94BE
:10419000784010926F121092701210927112109259
:1041A00072120C948D2A84917F012FEFE21AF20A89
:1041B000882321F00E947840F701F5CFD8018D9136
:1041C0008D01882319F00E947840F8CF8EE20E947A
:1041D00078400C948D2A8091F50F81110E94D86946
:1041E0008091F60F882311F40C948D2A80E50E94AB
:1041F0005C40882319F00E94CD3F03C080E50E94F7
:104200001340182F482F61E08091DC169091DD1645
:104210000E947EB683E50E945C40882381F00E9464
:10422000AC3FAB01BC0140936F125093701260938E
:104230007112709372128EEB91E10E94FF90809147
:10424000F60F882319F081E08093F50F11110C947B
:104250008D2A64CE8091DC169091DD1621E02093AA
:10426000F40F40E060E00E947EB60C948D2A0E941C
:10427000547F7B018C0120E831E541E050E00E9451
:1042800076CCC9016DE671E00E9487CF4B015C01DD
:10429000C801B70120E13EE040E050E00E9476CC4A
:1042A000CA01B90128E130E040E050E00E9476CC3C
:1042B000762E672EC62ED72E8CE3282E312C412C3D
:1042C000512CC801B701A20191010E9476CCF62EB3
:1042D000E72ECA01B901A20191010E9476CCCB015F
:1042E0008E010F5F1F4F81149104D1F0EF92FF9266
:1042F0007F936F936F927F92BF92AF929F928F92B4
:1043000085EC93E09F938F931F930F930E945AC85D
:104310000FB6F894DEBF0FBECDBFEFEFFAE145C098
:10432000A114B10489F0EF92FF927F936F936F9283
:104330007F92BF92AF9285EB93E09F938F931F93F1
:104340000F930E945AC8E4CFCD2879F0EF92FF92E4
:104350007F936F936F927F9289EA93E09F938F93FD
:104360001F930F930E945AC8D3CF892B69F0EF9205
:10437000FF927F936F9381EA93E09F938F931F93B4
:104380000F930E945AC8C4CFEF92FF928DE993E039
:104390009F938F931F930F930E945AC80F900F9073
:1043A0000F900F900F900F90B8CF84917F017FEF07
:1043B000E71AF70A882321F00E947840F701F5CF29
:1043C000B80189ED93E00E94024F8AE00E94784094
:1043D0000C948D2A83E50E945C40882311F40C9490
:1043E0008D2A0E94BC3FE82E80E50E945C40882315
:1043F00039F00E94BC3F182F87FF03C00C948D2A10
:104400001DE089E40E945C40882341F00E94CD3F7A
:1044100081110C94052BEDE0F6E00BC089E40E94BD
:104420001340F6CF319686E0ED33F80711F40C9483
:10443000052B84911813F6CF0C94DA2A0E94A37FDF
:104440000C948D2A8091A515813011F00C948D2A41
:1044500082E08093A5150E9416B66093A115709313
:10446000A2158093A3159093A4150C948D2A0E94F5
:10447000C57F0C948D2A88E690E00E94329E8111BF
:104480000C948D2A8091BD0B83FF02C00C948D2A61
:1044900083E50E945C40882399F00E94DC3F0E94E3
:1044A000F6CDCB010E94BC750E94DC3F20E030E0DD
:1044B00044EB52E40E9488C8181614F00E94C57F8D
:1044C0000E944D4F0C948D2A8EE40E945C408823FC
:1044D00011F40C948D2A0E94AC3F6093BA1670932D
:1044E000BB168093BC169093BD160C948D2A83E561
:1044F0000E941340882359F083E50E945C40882382
:1045000019F00E94BC3F01C080E08093BD0BEFEF2B
:10451000FAE184918F010F5F1F4F811103C0E4EF17
:10452000F3E004C00E947840F801F3CF84918F013A
:104530000F5F1F4F882321F00E947840F801F6CFCB
:104540008091BD0B811148CDE0EFF3E018C0BB2492
:10455000B394B20E222319F08CE20E947840F60147
:1045600085919491FC0184918F010F5F1F4F8823E7
:1045700021F00E947840F801F6CF2B2D3FCD849199
:104580008F010F5F1F4F882309F442CD0E947840AE
:10459000F801F5CF10924002C0C78BEF93E00E9464
:1045A00072510E94318AB9C783E50E945C40811133
:1045B00003C0EFEFFAE10BC00E94BC3F8D3318F44B
:1045C00080932202AAC78CE380932202A6C784911B
:1045D0008F010F5F1F4F882321F00E947840F80160
:1045E000F6CF4091220250E060E070E084E094E079
:1045F0000E94AF4E8AE00E9478408FC789E690E023
:104600000E94329E811111C0EBE0F4E084918F0191
:104610000F5F1F4F882321F00E947840F801F6CFEA
:104620000E94DC7C8AE00E94784010922B0B0C9454
:104630001A2B83E50E945C40882309F46EC70E9410
:10464000BC3F182F8D3308F01CE31093380B0E94E9
:1046500016B66B017C01212F30E0A8EEB3E00E947A
:10466000A2CCC60ED71EE81EF91EC092340BD09203
:10467000350BE092360BF092370B4FC70E94749EB9
:104680004CC78091BD0B83FD48C783E50E945C4009
:10469000882309F442C70E94DC3F0E94F6CD6E36A3
:1046A000710514F06EE670E070933C0460933B0477
:1046B0000E94967D32C70E9433992FC780E50E94E1
:1046C0005C40811106C083E50E945C40882359F05C
:1046D00005C00E94BC3F811120C7F5CF0E94AC3FAE
:1046E0006F3F710510F06FEF70E070933A046093C4
:1046F000390413C780E50E945C40811105C0109207
:104700003A041092390409C70E94AC3F672B09F0A4
:1047100004C7F5CF62E370E080E090E00E94DEB570
:104720000E949A820F5F1F4F0331110599F762E3D0
:1047300070E080E090E00E94DEB50E949A8294D7FB
:10474000ECC610921D04E9C681E080931D04E5C605
:1047500083E50E945C40882399F00E94DC3F20E0C2
:1047600030E04AE754E40E94EDC80E94FBCD60931C
:104770002302709324028093250290932602CDC6D3
:1047800088E50E9413408111E3C689E50E94134029
:104790008111DEC68AE50E9413408111D9C685E4E5
:1047A0000E9413408111D4C60E9493A6B6C683E529
:1047B0000E941340882309F4B0C60E94DC3F20E029
:1047C00030E04AE754E40E94EDC80E94FBCD6093BC
:1047D000300B7093310B8093320B9093330B9DC64B
:1047E000F60181916F010E941340882309F46EC085
:1047F000133009F063C00E94DC3F4B015C0120E0F4
:1048000030E040EA51E40E9488C887FF4EC0A5010D
:104810009401609121177091221780912317909134
:1048200024170E948ECD2B013C019B01AC016091AD
:104830008C0B70918D0B80918E0B90918F0B0E9441
:10484000EDC860938C0B70938D0B80938E0B9093BF
:104850008F0BA30192016091AC0B7091AD0B809115
:10486000AE0B9091AF0B0E94EDC86093AC0B7093B0
:10487000AD0B8093AE0B9093AF0B6091F1167091DE
:10488000F2168091F3169091F4160E948CC8A30141
:1048900092010E94EDC80E94FBCD6093F1167093C7
:1048A000F2168093F3169093F4168092211790924B
:1048B0002217A0922317B092241708C00E94DC3F51
:1048C000D7016D937D938D939C9313971F5FB4E0F5
:1048D000EB0EF11C143009F083CF0E9477BC1DC68B
:1048E0000E94D86983E50E945C40882311F40C94EF
:1048F000FE1B0E94AC3F6230710511F00C94FE1B50
:104900000E9455598BE50E94784060911E0B709172
:104910001F0B8091200B9091210B42E00E941944C3
:104920004091220B5091230B6091240B7091250B29
:1049300081E194E00E94CC4E4091260B5091270BD0
:104940006091280B7091290B8EE094E00E94CC4E70
:104950008DE50E9478408AE00E947840DEC584910F
:104960008F010F5F1F4F882321F00E947840F801CC
:10497000F6CF60E083EE94E00E94AD9061E08CEDB4
:1049800094E00E94AD9061E081ED94E00E94AD90D2
:1049900061E081EC94E00E94AD9060E088EB94E0EF
:1049A0000E94AD9061E08EEA94E00E94AD9060E0DC
:1049B00084EA94E00E94AD9060E08CE994E00E946B
:1049C000AD9061E08EE894E00E94AD9060E080E8F8
:1049D00094E00E94AD9060E081E794E00E94AD9089
:1049E00060E083E694E00E94AD9060E08DE494E0A6
:1049F0000E94AD9060E08CE394E00E94AD9060E096
:104A000087E294E00E94AD9061E084E194E00E942E
:104A1000AD9083C50091DC161091DD1683E0D12C9A
:104A200040E08150E1F0F8019081292F2B7F213463
:104A3000C1F721812133A9F7913421F0953421F474
:104A400041E002C0DD24D39498012E5F3F4F8901DD
:104A50002F5F3F4FD8019C919032C9F3E2CF44239E
:104A600069F0EFEFFAE184917F01BFEFEB1AFB0AE7
:104A7000882321F00E947840F701F5CFDD2069F00E
:104A8000E9EBF5E084917F012FEFE21AF20A882327
:104A900021F00E947840F701F5CFD8018D918D016A
:104AA000882309F4B5CA0E947840F7CF0E946DAC04
:104AB00034C581E08093D40B8093D30B2EC588EC52
:104AC00090E00E94329E811128C584E40E94134028
:104AD000882309F441C00E94DC3F6B017C0111E096
:104AE00020E030E0A9010E9488C8811101C010E0D7
:104AF0001093931620E030E0A901C701B6010E948F
:104B000088C8882349F10E94DC3FE091C815B4E0D1
:104B1000EB9FF0011124E856F94E60837183828384
:104B2000938320E030E0A901609198167091991666
:104B300080919A1690919B160E9488C881110CC092
:104B400080E090E0A0EEBFE38093981690939916D2
:104B5000A0939A16B0939B160E94D1A6DEC4F701CB
:104B600081917F010E941340882351F00E94DC3F15
:104B70000E94FBCDD8016D937D938D939C931397E9
:104B80000C5F1F4FC016D10651F70E9406BBC5C46B
:104B90006FE4E62E62E0F62E00EA1BE0F701819159
:104BA0007F010E941340882341F00E94DC3FD8011E
:104BB0006D937D938D939C9313970C5F1F4FBBE078
:104BC000003B1B0759F7A9C483E50E945C4088237A
:104BD000A1F00E94DC3F6093980B7093990B809337
:104BE0009A0B90939B0B6093940B7093950B80930F
:104BF000960B9093970B10E001C011E080E50E94A6
:104C00005C40882359F00E94DC3F6093980B7093BE
:104C1000990B80939A0B90939B0B10E082E50E9476
:104C20005C40882359F00E94DC3F60939C0B70939A
:104C30009D0B80939E0B90939F0B10E084E50E9448
:104C40005C40882359F00E94DC3F6093940B709382
:104C5000950B8093960B9093970B5FC4112309F4E7
:104C60005CC44091980B5091990B60919A0B709194
:104C70009B0B83EC95E00E94CC4E40919C0B509195
:104C80009D0B60919E0B70919F0B80EC95E00E94B4
:104C9000CC4E4091940B5091950B6091960B709176
:104CA000970B8DEB95E00E94CC4E8AE00E947840F5
:104CB00034C481E50E9413408823C1F08091180418
:104CC00090911904009739F04AE050E060E070E0FC
:104CD0000E9407C703C060E070E0CB016093B00B97
:104CE0007093B10B8093B20B9093B30B83E50E944A
:104CF0001340882351F00E94DC3F6093B80B7093FF
:104D0000B90B8093BA0B9093BB0B84E50E941340C0
:104D1000882351F00E94DC3F6093B40B7093B50B75
:104D20008093B60B9093B70B88E50E9413408823BD
:104D300051F00E94DC3F6093800B7093810B809355
:104D4000820B9093830B89E50E941340882351F0D6
:104D50000E94DC3F6093840B7093850B8093860BDD
:104D60009093870B8AE50E9413408823F1F00E94FC
:104D7000DC3F6093880B7093890B80938A0B909330
:104D80008B0B2DEC3CEC4CEC5DE30E9488C81816B4
:104D900064F0E3EDF5E084918F010F5F1F4F8823EE
:104DA00021F00E947840F801F6CF85E40E9413407C
:104DB000882309F4B2C30E94DC3F60938C0B70938C
:104DC0008D0B80938E0B90938F0BA7C34FE4C42E53
:104DD00042E0D42E55EDE52E5BE0F52E10E0F60115
:104DE00081916F010E941340882359F00E94DC3F9B
:104DF000D7016D937D938D939C931397812F0E9480
:104E0000F29D1F5FB4E0EB0EF11C133041F70C94E0
:104E1000FE1B0E94268681C383E50E945C40882396
:104E200009F47BC30E94AC3F7093030260930202BB
:104E300074C38DED90E00E94329E81116EC383E5B4
:104E40000E945C40811103C0EFEFFAE139C000918C
:104E5000C81510E00E94AC3F000F111FF801E75B7E
:104E6000FD4F718360838091C81590E07C01EE0C4A
:104E7000FF1CEE0CFF1C87010D5C1D4F880F991F56
:104E8000FC01E75BFD4F60817181072E000C880BF0
:104E9000990B0E948EC82AE037ED43E25CE30E9442
:104EA000EDC8F701EC56F94E2081318142815381E2
:104EB0000E94EDC8F80160837183828393832DC3C0
:104EC00084918F010F5F1F4F882321F00E9478404B
:104ED000F801F6CF85E40E9478408091C815805D86
:104EE0000E947840E091C815F0E0EE0FFF1FE75BED
:104EF000FD4F6081718185E096E00E94E94E85E278
:104F00000E9478408AE00E94784007C380E50E94B2
:104F10001340882309F401C30E94AC3F6B017C015C
:104F200083E50E945C40882321F00E94AC3F8B0106
:104F300002C00FEF1FEFC8010196039708F0EDC202
:104F4000D7FCEBC28C2DEDE0F6E09491891709F4C3
:104F500031C3319626E0ED33F207B9F72EC383E56E
:104F60000E945C40882319F00E94AC3F02C064E0BC
:104F700071E079A368A380E50E945C40882339F042
:104F80000E94AC3F693833E1730730F402C068EE29
:104F900073E07A83698304C088E893E19A83898304
:104FA000BE01605E7F4FCE0101960E9434B4B5C24F
:104FB00085E40E945C40811110C080E50E9413408E
:104FC000882391F00E94DC3F6093B6157093B7156B
:104FD0008093B8159093B91507C00E94BC3F8823F1
:104FE00061F3EAEEFAE171C089E40E94134088237C
:104FF00081F00E94DC3F2CEA35EC47E25EE30E9440
:10500000EDC86093B2157093B3158093B415909367
:10501000B51584E40E941340882381F00E94DC3F90
:105020002CEA35EC47E25EE30E948ECD6093BA1520
:105030007093BB158093BC159093BD15EFEFFAE10B
:1050400084918F010F5F1F4F882321F00E947840C9
:10505000F801F6CF4091B6155091B7156091B8158B
:105060007091B91585E496E00E94CC4E2CEA35EC9F
:1050700047E25EE36091B2157091B3158091B4156B
:105080009091B5150E948ECDAB01BC0181E496E0F4
:105090000E94CC4E2CEA35EC47E25EE36091BA15F3
:1050A0007091BB158091BC159091BD150E94EDC803
:1050B000AB01BC018DE396E00E94CC4E8AE00E94D9
:1050C00078402BC20E947840F80184918F010F5FD5
:1050D0001F4F8111F7CFE9E4F6E084918F010F5F54
:1050E0001F4F882309F419C20E947840F801F5CFB8
:1050F00083E50E941340182F882371F00E94DC3F43
:105100000E94F6CD709338026093370221E0672B3E
:1051100009F020E02093BC0B80E50E941340882317
:1051200059F02091370230913802232B11F00E9460
:10513000CD3F8093BC0BF1C11111EFC1EFEFFAE14C
:1051400084918F010F5F1F4F882321F00E947840C8
:10515000F801F6CF8091BC0B882319F063E173E06E
:1051600002C066E173E080E796E00E94024F609122
:105170003702709138028FE596E00E94E94EEBE528
:10518000F6E084918F010F5F1F4F882309F4C5C19A
:105190000E947840F801F5CF0E946E8ABEC180E57A
:1051A0000E941340882351F00E94DC3F6093AE15AB
:1051B0007093AF158093B0159093B11589E40E9458
:1051C0001340882381F00E94DC3F2CEA35EC47E253
:1051D0005EE30E94EDC86093AA157093AB158093AF
:1051E000AC159093AD1584E40E941340882381F0A0
:1051F0000E94DC3F2CEA35EC47E25EE30E948ECD54
:105200006093A6157093A7158093A8159093A91580
:10521000EFEFFAE184918F010F5F1F4F882321F098
:105220000E947840F801F6CF4091AE155091AF152D
:105230006091B0157091B1158BE896E00E94CC4E4C
:105240002CEA35EC47E25EE36091AA157091AB154C
:105250008091AC159091AD150E948ECDAB01BC0133
:1052600087E896E00E94CC4E2CEA35EC47E25EE3FC
:105270006091A6157091A7158091A8159091A91518
:105280000E94EDC8AB01BC0183E896E00E94CC4EC1
:105290008AE00E94784041C10E947840F8018491E0
:1052A0008F010F5F1F4F8111F7CFEFE8F6E0849178
:1052B0008F010F5F1F4F882309F42FC10E94784090
:1052C000F801F5CF0E947F8728C10E94137025C185
:1052D0000E9405A522C183E50E941340882321F086
:1052E0000E94CD3F91E089270E9471A016C181E004
:1052F0008093C40B0E94096A1092C40B882309F49E
:105300000CC1EFEFFAE184918F010F5F1F4F811104
:1053100003C0EEE9F6E004C00E947840F801F3CF44
:1053200084918F010F5F1F4F882309F4F6C00E94FC
:105330007840F801F5CF8091F50F882309F4EDC08E
:1053400081E08093F80FE9C08AE50E945C408111FA
:1053500003C0ECEAF6E00BC00E94DC3F6093271626
:10536000709328168093291690932A16D6C084919C
:105370008F010F5F1F4F882321F00E947840F801B2
:10538000F6CF4091271650912816609129167091FA
:105390002A1689EA96E00E94CC4E8AE00E94784064
:1053A000BCC08BE40E945C40811103C0EFEFFAE1C6
:1053B00036C08BE40E945C408823C1F00E94DC3F31
:1053C0006B017C0120E030E0A9010E94D8CE87FD6E
:1053D0000AC020E030E040E251E4C701B6010E947B
:1053E00088C8181634F4EBECF6E00EC0C12CD12CB2
:1053F00076010E94D869C092900BD092910BE092F6
:10540000920BF092930B89C084918F010F5F1F4F15
:10541000882309F482C00E947840F801F5CF849176
:105420008F010F5F1F4F882321F00E947840F80101
:10543000F6CF4091900B5091910B6091920B70912F
:10544000930B8AEE96E00E94CC4E8AE00E94784050
:1054500064C081E08093410283E50E945C40882320
:1054600039F00E94CD3F811158C00E948E5955C01D
:1054700083E50E941340F7CF0E9468B44EC0F090BD
:10548000DE160E94D8691091A71680E00E948E9CBB
:10549000FF2029F1EFEFFAE184918F010F5F1F4F99
:1054A000882321F00E947840F801F6CF84E50E941D
:1054B00078406F2D70E080E090E04AE00E949443D5
:1054C00080E20E947840E7E0F7E084918F010F5F6F
:1054D0001F4F882311F10E947840F801F6CF1092F7
:1054E0002A0B812F0E948E9CEFEFFAE184918F01AD
:1054F0000F5F1F4F882321F00E947840F801F6CFFC
:1055000060912A0B70E085EF96E00E94E94E8AE0F8
:105510000E94784002C00E9468B410922B0B0E9437
:10552000715988C00E940E9B0E947955F6CF0E9447
:10553000AC3FAB01BC0140936F125093701260936B
:105540007112709372128EEB91E10E94FF90E5CF81
:105550000E94D86988E50E941340882331F05F9A41
:10556000809128048E7F8093280489E50E9413404F
:10557000882339F08A9A479A809128048D7F8093F6
:1055800028048AE50E941340882361F08091080175
:105590008095817080930601479A809128048B7FC3
:1055A0008093280485E40E941340882309F4B5CF32
:1055B000129AB3CF0E945EC4B0CF0E94D869BC2CAF
:1055C00060E08C2D0E94DBB40F3F4FEF140759F4BD
:1055D0008C2D0E9485B431E020E0892B09F030E069
:1055E000032F122F05C00130110561F401E010E016
:1055F0008B2D0E9485B48017910709F48ECF0E94ED
:10560000B951F6CF00E010E0F3CF61E0812F0E94A6
:10561000DBB46E2D812F0E94ADB4F12CB701812F28
:105620000E9417B5193009F078CFF0923A04E09251
:10563000390473CFC559DF4F0FB6F894DEBF0FBEE4
:10564000CDBFDF91CF911F910F91FF90EF90DF9031
:10565000CF90BF90AF909F908F907F906F905F9012
:105660004F903F902F9008952F923F924F925F92CC
:105670006F927F928F929F92AF92BF92CF92DF9262
:10568000EF92FF920F931F93CF93DF93CDB7DEB7C7
:105690006F970FB6F894DEBF0FBECDBFC090430426
:1056A000D0904404E0904504F090460420E030E0BF
:1056B00040EA50E4C701B6010E9488C887FD19C1BD
:1056C00020E030E041E953E4C701B6010E94D8CEA2
:1056D00018160CF40EC1109212141092111480912D
:1056E000090140911014042E000C550B817021E02B
:1056F000822790E04817590709F433C080910901C7
:10570000817028272093101481111BC00E942377D9
:10571000E7E1FDE084918F01882351F0082E000C11
:10572000990B0E941E770F5F1F4FF8018491F4CFF1
:105730008DE090E00E941E778AE090E00E941E7744
:1057400010C0EBE1FDE084918F01882389F3082EDE
:10575000000C990B0E941E770F5F1F4FF801849178
:10576000F4CF80910314833009F44CC02CF48823C7
:1057700051F08130D9F072C0843009F43EC08530D8
:1057800009F44DC06BC08091F50F882309F466C001
:1057900081E0809303140E9416B6609307147093FF
:1057A00008148093091490930A1458C08091F50F3F
:1057B000811154C08091C111882321F082E080932F
:1057C00003144CC010920314E3E1FDE084918F01B7
:1057D000882351F0082E000C990B0E941E770F5F52
:1057E0001F4FF8018491F4CF8DE090E00E941E7766
:1057F0008AE090E00E941E7731C080915014882387
:10580000E9F22CC08091F50F811128C08091770FAB
:105810009091780F891B8F7009F496C01FC08091FA
:10582000F50F81111BC08091770F9091780F891B24
:105830008F7009F4ABC012C08DE090E00E941E771B
:105840008AE090E00E941E771092031483EF9CE0A0
:105850009093680D8093670D0E94A4408091F81387
:105860009091F91303974CF577E2272E79E0372EC4
:10587000E0E68E2EEAEE9E2EA12CB12C8EE595E16F
:105880000E94853B18161906C4F48091F813909174
:10589000F913049794F48EE595E10E94493B8093B7
:1058A000FE13E091FF13F09100148A3019F08D304F
:1058B00009F07DC0309709F083C08091F813909172
:1058C000F913009711F40C94BA3A01979093F913D5
:1058D0008093F8138091FA139091FB13019664E082
:1058E00070E00E949BCF9093FB138093FA130C946B
:1058F000BA3A80911114909112148136FAEE9F07F2
:10590000E8F01092121410921114EFE1FDE084916E
:105910008F01882351F0082E000C990B0E941E77EE
:105920000F5F1F4FF8018491F4CF8DE090E00E944B
:105930001E778AE090E00E941E77D1CE0196909368
:10594000121480931114CBCE8FEF9CE09093680DCE
:105950008093670D0E94A44080915014882311F019
:1059600082E001C084E080930314EBEFFCE08491BB
:105970008F01882309F438CF082E000C990B0E9460
:105980001E770F5F1F4FF8018491F3CFE7EFFCE024
:1059900084918F01882309F44FCF082E000C990BB6
:1059A0000E941E770F5F1F4FF8018491F3CF8A3357
:1059B00009F480CFEF35F10514F40C9453387ACF05
:1059C0008091FC139091FD1320E6289F7001299F80
:1059D000F00C1124870108581D4EE00FF11F1082B2
:1059E00061E470E0C8010E941ED0009711F40C948D
:1059F00037389093021480930114801B910B8E0D05
:105A00009F1D60E070E087589D4E0E9489C40E94EF
:105A1000F6CDCB01770FAA0BBB0B8232910510F0AC
:105A20000C943738FC018827EE58FF4F8F4F0C94A9
:105A3000CACFEEEEFCE084918F01882351F0082E4E
:105A4000000C990B0E941E770F5F1F4FF801849185
:105A5000F4CF20E030E040E05FE3609143047091D8
:105A6000440480914504909146041EC0E9EEFCE098
:105A700084918F01882351F0082E000C990B0E940D
:105A80001E770F5F1F4FF8018491F4CF609141049E
:105A900070914204072E000C880B990B0E948EC84F
:105AA00020E030E040E05FE30E94B2CC0E94F6CDFF
:105AB000CB010E94B4440E94B6B88DE090E00E94F1
:105AC0001E778AE090E00E941E770C943738E4EE4F
:105AD000FCE084918F01882351F0082E000C990B73
:105AE0000E941E770F5F1F4FF8018491F4CF20E0D2
:105AF00030E040E05FE360913D0470913E048091AE
:105B00003F0490914004D0CFEFEDFCE084918F01F1
:105B1000882351F0082E000C990B0E941E770F5F0E
:105B20001F4FF8018491F4CF60913B0470913C04C5
:105B3000B1CF2091390430913A0444E6429FC0012C
:105B4000439F900D11246FEF70E00E949BCF8B015B
:105B50006536710510F004E610E0EAEDFCE0849192
:105B60007F01882359F0082E000C990B0E941E77A4
:105B7000FFEFEF1AFF0AF7018491F3CFB80180E03D
:105B800090E040C7E6EDFCE084918F01882351F05E
:105B9000082E000C990B0E941E770F5F1F4FF80113
:105BA0008491F4CF80E290E00E941E77E2EDFCE069
:105BB00084918F01882351F0082E000C990B0E94CC
:105BC0001E770F5F1F4FF8018491F4CF6091290475
:105BD00070912A0480912B0490912C040E94B7B8F4
:105BE00080E290E00E941E77EEECFCE084918F0151
:105BF000882351F0082E000C990B0E941E770F5F2E
:105C00001F4FF8018491F4CF60912D0470912E0400
:105C100080912F04909130040E94B7B880E290E008
:105C20000E941E77EAECFCE084918F01882351F0FA
:105C3000082E000C990B0E941E770F5F1F4FF80172
:105C40008491F4CF609131047091320480913304D7
:105C5000909134040E94B7B880E290E0A0C5809192
:105C6000F50F882309F450C0E5ECFCE084918F0126
:105C7000882351F0082E000C990B0E941E770F5FAD
:105C80001F4FF8018491F4CF8091F60F882359F1CA
:105C90008091C111882329F180916B1290916C122F
:105CA000A0916D12B0916E120097A105B105C1F0DF
:105CB000BC01CD016D597F4F8F4F9F4F24E630E0DF
:105CC00040E050E00E9476CC60916F1270917012AB
:105CD00080917112909172120E9476CC822F01C035
:105CE00080E090E0E6CEE1ECFCE084918F01882337
:105CF00009F4E3CE082E000C990B0E941E770F5F6B
:105D00001F4FF8018491F3CFE9EBFCE084918F0100
:105D1000882309F4D2CE082E000C990B0E941E771E
:105D20000F5F1F4FF8018491F3CFE4EBFCE0849107
:105D30008F01882351F0082E000C990B0E941E77CA
:105D40000F5F1F4FF8018491F4CF80910714909159
:105D50000814A0910914B0910A14892B8A2B8B2B5B
:105D600009F477C00E9416B6A50194010E9476CC72
:105D700069017A01609107147091081480910914E7
:105D800090910A14A50194010E9476CC8601021B11
:105D9000130BC8016CE370E00E9487CFCB019927F9
:105DA000EAE0F0E0BF010E949BCF282FCB01BF01AA
:105DB0000E949BCF805D80932004205D209321046E
:105DC0001092220480E294E00E94B6B880E290E053
:105DD0000E941E77E2EBFCE084917F01882359F05A
:105DE000082E000C990B0E941E77FFEFEF1AFF0A96
:105DF000F7018491F3CF80E290E00E941E77C80102
:105E00006CE370E00E9487CF6AE070E00E949BCF55
:105E1000605D60932004805D8093210410922204D1
:105E200080E294E00E94B6B880E290E00E941E7783
:105E3000E0EBFCE084918F01882309F43ECE082E2C
:105E4000000C990B0E941E770F5F1F4FF801849181
:105E5000F3CF80E290E00E941E77E8EAFCE08491B4
:105E60008F01882309F429CE082E000C990B0E947B
:105E70001E770F5F1F4FF8018491F3CF10923114FA
:105E80008091090180FF11C0E4EAFCE084918F0158
:105E9000882309F412CE082E000C990B0E941E775D
:105EA0000F5F1F4FF8018491F3CF83E50E9452B832
:105EB000882341F00E946DB80E94FBCD70930614B8
:105EC00060930514E0EAFCE084918F01882351F08F
:105ED000082E000C990B0E941E770F5F1F4FF801D0
:105EE0008491F4CF8DE090E00E941E778AE090E0EC
:105EF0000E941E7780914F14882309F442C280913A
:105F00000514909106148430910509F4C8C08830B6
:105F1000910509F47DC1892B09F0E7C3E4ECFAE0AF
:105F200084918F01882351F0082E000C990B0E9458
:105F30001E770F5F1F4FF8018491F4CF8DE090E042
:105F40000E941E778AE090E00E941E77E9EBFAE05B
:105F500084918F01882351F0082E000C990B0E9428
:105F60001E770F5F1F4FF8018491F4CF8DE090E012
:105F70000E941E778AE090E00E941E77EDEAFAE028
:105F800084918F01882351F0082E000C990B0E94F8
:105F90001E770F5F1F4FF8018491F4CF8DE090E0E2
:105FA0000E941E778AE090E00E941E77E1EAFAE004
:105FB00084918F01882351F0082E000C990B0E94C8
:105FC0001E770F5F1F4FF8018491F4CF8DE090E0B2
:105FD0000E941E778AE090E00E941E77E3E9FAE0D3
:105FE00084918F01882351F0082E000C990B0E9498
:105FF0001E770F5F1F4FF8018491F4CF8DE090E082
:106000000E941E778AE090E00E941E77E5E8FAE0A1
:1060100084918F01882351F0082E000C990B0E9467
:106020001E770F5F1F4FF8018491F4CF8DE090E051
:106030000E941E778AE090E00E941E77E8E7FAE06F
:1060400084918F01882351F0082E000C990B0E9437
:106050001E770F5F1F4FF8018491F4CF8DE090E021
:106060000E941E778AE090E00E941E77EBE6FAE03D
:1060700084918F01882351F0082E000C990B0E9407
:106080001E770F5F1F4FF8018491F4CF8DE090E0F1
:106090000E941E778AE090E00E941E7726C3EDE5FD
:1060A000FAE084918F01882351F0082E000C990B9F
:1060B0000E941E770F5F1F4FF8018491F4CF8DE08F
:1060C00090E00E941E778AE090E00E941E77EFE445
:1060D000FAE084918F01882351F0082E000C990B6F
:1060E0000E941E770F5F1F4FF8018491F4CF8DE05F
:1060F00090E00E941E778AE090E00E941E77E9E31C
:10610000FAE084918F01882351F0082E000C990B3E
:106110000E941E770F5F1F4FF8018491F4CF8DE02E
:1061200090E00E941E778AE090E00E941E77E3E2F2
:10613000FAE084918F01882351F0082E000C990B0E
:106140000E941E770F5F1F4FF8018491F4CF8DE0FE
:1061500090E00E941E778AE090E00E941E77E1E1C5
:10616000FAE084918F01882351F0082E000C990BDE
:106170000E941E770F5F1F4FF8018491F4CF8DE0CE
:1061800090E00E941E778AE090E00E941E77EFEF79
:10619000F9E084918F01882351F0082E000C990BAF
:1061A0000E941E770F5F1F4FF8018491F4CF8DE09E
:1061B00090E00E941E778AE090E00E941E77E1EF57
:1061C000F9E084918F01882351F0082E000C990B7F
:1061D0000E941E770F5F1F4FF8018491F4CF8DE06E
:1061E00090E00E941E778AE090E00E941E77E3EE26
:1061F000F9E084918F01882309F448CF082E000C20
:10620000990B0E941E770F5F1F4FF8018491F3CF07
:10621000ECEDF9E084918F01882351F0082E000CF9
:10622000990B0E941E770F5F1F4FF8018491F4CFE6
:106230008DE090E00E941E778AE090E00E941E7739
:10624000E5EDF9E084918F01882351F0082E000CD0
:10625000990B0E941E770F5F1F4FF8018491F4CFB6
:106260008DE090E00E941E778AE090E00E941E7709
:10627000EEEBF9E084918F01882351F0082E000C99
:10628000990B0E941E770F5F1F4FF8018491F4CF86
:106290008DE090E00E941E778AE090E00E941E77D9
:1062A000E7EAF9E084918F01882351F0082E000C71
:1062B000990B0E941E770F5F1F4FF8018491F4CF56
:1062C0008DE090E00E941E778AE090E00E941E77A9
:1062D000E0E9F9E084918F01882351F0082E000C49
:1062E000990B0E941E770F5F1F4FF8018491F4CF26
:1062F0008DE090E00E941E778AE090E00E941E7779
:10630000E9E7F9E084918F01882351F0082E000C11
:10631000990B0E941E770F5F1F4FF8018491F4CFF5
:106320008DE090E00E941E778AE090E00E941E7748
:10633000EBE6F9E084918F01882351F0082E000CE0
:10634000990B0E941E770F5F1F4FF8018491F4CFC5
:106350008DE090E00E941E778AE090E00E941E7718
:10636000EDE5F9E084918F01882309F48FCE082EA2
:10637000000C990B0E941E770F5F1F4FF80184914C
:10638000F3CF8091F60F882309F486C181E08093D2
:106390007312109275121092741285E490E10E94AB
:1063A00046938BE1E5E4F0E1DE01159601900D9254
:1063B0008A95E1F780914310909144109C838B83E0
:1063C00085EE92E09A83898340E050E0BE016F5FE2
:1063D0007F4F80E090E00E945479CE0101960E94A8
:1063E0004F51C0907412D090751200910514109105
:1063F0000614C601801B910B049720F06801F3E09E
:10640000CF0ED11C5EE4452E59E0552E6FE3662E6B
:1064100069E0762EC016D10608F467C10115110592
:1064200009F0A1C069EF7FE085E490E10E940E923F
:106430006AE173E089EF9FE00E9429D0892B09F07F
:106440004AC0F20184914EE4E42E49E0F42E882300
:1064500059F0082E000C990B0E941E77FFEFEF1ADF
:10646000FF0AF7018491F3CF8DE090E00E941E7740
:106470008AE090E00E941E77F30184913FE3E32ECF
:1064800039E0F32E882359F0082E000C990B0E9456
:106490001E77FFEFEF1AFF0AF7018491F3CF8DE02B
:1064A00090E00E941E778AE090E00E941E774AE00A
:1064B00060E070E0CB010E949443EFE2F9E0849148
:1064C0007F012FEFE21AF20A882309F4E2C00E944A
:1064D0007840F701F4CFEBE2F9E084917F01882363
:1064E00059F0082E000C990B0E941E77FFEFEF1A4F
:1064F000FF0AF7018491F3CF8DE090E00E941E77B0
:106500008AE090E00E941E77F101849127E2E22E5A
:1065100029E0F22E882359F0082E000C990B0E94D6
:106520001E77FFEFEF1AFF0AF7018491F3CF8DE09A
:1065300090E00E941E778AE090E00E941E774AE079
:1065400060E070E0CB010E949443E2E2F9E08491C4
:106550007F012FEFE21AF20A882309F49AC00E9401
:106560007840F701F4CF60E070E0C80101970E9425
:106570001A7B8091F70F882309F45FC0E0E2F9E00D
:1065800084917F01882359F0082E000C990B0E94FA
:106590001E77FFEFEF1AFF0AF7018491F3CF89EF1F
:1065A0009FE00E94B6B88DE090E00E941E778AE0DE
:1065B00090E00E941E77EEE1F9E084917F0188234C
:1065C00059F0082E000C990B0E941E77FFEFEF1A6E
:1065D000FF0AF7018491F3CF86E090E10E94B6B8FC
:1065E0008DE090E00E941E778AE090E00E941E7786
:1065F000C801A0E0B0E04AE0BC01CD010E94944394
:10660000ECE1F9E084917F012FEFE21AF20A88238E
:1066100021F00E947840F701F5CF96E0E92E90E155
:10662000F92EF70181917F01882319F00E947840AB
:10663000F8CF8AE00E9478402CC089EF9FE00E944A
:10664000B6B88DE090E00E941E778AE090E00E944C
:106650001E7786E090E10E94B6B88DE090E00E943F
:106660001E778AE090E00E941E77C801A0E0B0E0AB
:106670004AE0BC01CD010E94944386E0E82E80E10F
:10668000F82EF70181917F01882399F20E947840CA
:10669000F8CF0F5F1F4FBECEEDE0F9E084918F0180
:1066A000882351F0082E000C990B0E941E770F5F73
:1066B0001F4FF8018491F4CF8DE090E00E941E7787
:1066C0008AE090E00E941E77EEEFF8E084918F015F
:1066D000882309F4DBCC082E000C990B0E941E774E
:1066E0000F5F1F4FF8018491F3CFECE9FCE0849138
:1066F0008F01882309F4E1C9082E000C990B0E9430
:106700001E770F5F1F4FF8018491F3CF8091F50F33
:10671000882339F00E948678AAC48091F50F8823D7
:10672000E9F00E949BB2A3C480910314823019F057
:10673000833609F09CC40E946578E8E9FCE0849106
:106740008F01882309F4B9C9082E000C990B0E9407
:106750001E770F5F1F4FF8018491F3CF80910314D0
:10676000833609F084C4DDCF8FE89CE00E9472512B
:106770008091770F9091780F891B8F7009F077C403
:1067800080910314823009F472C4833609F0A3C4E3
:106790006EC48DE090E00E941E778AE090E00E9437
:1067A0001E778BC98091770F9091780F891B8F701E
:1067B00009F05DC480910314823009F458C4833613
:1067C00009F455C48091C1118111D9C450C483E525
:1067D0000E9452B8811126C083E40E9452B88823D7
:1067E00009F445C48091770F9091780F891B8F70C1
:1067F00009F03DC420E030E040E251E46091310412
:106800007091320480913304909134040E9488C8BE
:1068100087FF08C08CE79CE09093680D8093670D1C
:106820000E94A4400E946DB820E030E0A9010E94BF
:1068300088C887FD10C00E946DB820E030E849E8A4
:1068400053E40E94D8CE18164CF00E946DB80E94F6
:10685000FBCDCB0105C080E090E002C083E191E078
:106860000E94BC7504C483E50E9452B8882309F4D1
:10687000FEC30E946DB820E030E0A9010E9488C8E4
:1068800087FD11C00E946DB820E030E046E153E47E
:106890000E94D8CE18164CF00E946DB80E94FBCD15
:1068A000362F272F04C030E001C036E920E0832FC7
:1068B000922F8E36910514F08EE690E090933C0472
:1068C00080933B040E94967DD2C383E50E9452B818
:1068D0008823D9F00E946DB820E030E04FE753E400
:1068E0000E94EDC820E030E048EC52E40E948ECDDA
:1068F0000E94FBCD6F3F710519F010F06FEF70E053
:1069000070933A0460933904D8C88FEF90E0909365
:106910003A0480933904D1C88091770F9091780F11
:10692000891B8F7009F0C9C88091F50F8111C5C806
:106930000E94318A5F9A809128048E7F8093280478
:106940008A9A479A809128048D7F809328048091A9
:1069500008018095817080930601479A80912804F0
:106960008B7F80932804129AA8C883E50E9452B8AE
:10697000882319F10E946DB820E030E040E252E433
:106980000E9488C887FD0FC00E946DB820E030ECDF
:1069900049E754E40E94D8CE181644F00E946DB81E
:1069A0000E94F6CD05C068E270E002C067EE73E0B9
:1069B00070930302609302025AC3E6E7FCE08491FD
:1069C0008F01882351F0082E000C990B0E941E772E
:1069D0000F5F1F4FF8018491F4CFC0900202D09056
:1069E00003020D2C000CEE08FF08F7FE0DC06DE24F
:1069F0008EE595E101D666277727CB016C197D09D5
:106A00008E099F094AE003C04AE0C701B6010E940F
:106A100076B853C88091770F9091780F891B8F704B
:106A200009F025C380910314823009F420C3833612
:106A300009F0EBC21CC38091770F9091780F891BEE
:106A40008F7009F03AC880910314823009F435C878
:106A5000833609F0B6C331C88091770F9091780FD3
:106A6000891B8F7009F003C380910314823009F4ED
:106A7000FEC2833609F0F8C4FAC28091770F909174
:106A8000780F891B8F7009F0F2C280910314823055
:106A900009F4EDC2833609F01CC5E9C28091770F75
:106AA0009091780F891B8F7009F0E1C280910314D7
:106AB000823009F4DCC2833609F040C5D8C2809127
:106AC0003114811103C00E942377C4C18E3271F545
:106AD000809132148E3209F046C18091961188233C
:106AE00009F4B8C1815080939611882361F090E039
:106AF00001974FE1489F9001499F300D1124C90132
:106B0000805A9F4E02C082E290E12BE1FC01349654
:106B1000A5E4B0E101900D922A95E1F7FC01828194
:106B20009381909344108093431094C18C3309F067
:106B30001AC16CE173E081E394E10E9429D0892BB2
:106B400021F481E080934F1485C16BE273E081E30F
:106B500094E10E9429D0892B79F4EAEDF8E0849140
:106B60008F010F5F1F4F882321F00E947840F801AA
:106B7000F6CF87EC98E0E4C062E473E081E394E14F
:106B80000E9429D0892B79F4E3EAF8E084918F01FF
:106B90000F5F1F4F882321F00E947840F801F6CF45
:106BA00080E998E0CDC069E573E081E394E10E945B
:106BB00029D0892B79F4E5E7F8E084918F010F5F04
:106BC0001F4F882321F00E947840F801F6CF80E71C
:106BD00098E0B6C067E673E081E394E10E9429D0B3
:106BE000892B79F4E5E5F8E084918F010F5F1F4F61
:106BF000882321F00E947840F801F6CF80E598E0E4
:106C00009FC065E773E081E394E10E9429D0892B5E
:106C100079F4E5E3F8E084918F010F5F1F4F88233B
:106C200021F00E947840F801F6CF8CE298E088C00D
:106C300063E873E081E394E10E9429D0892B71F429
:106C400009E018E0F8018491882329F00F5F1F4FB5
:106C50000E947840F7CF82E098E072C069E973E063
:106C600081E394E10E9429D0892B79F4E3EEF7E0E7
:106C700084918F010F5F1F4F882321F00E9478407D
:106C8000F801F6CF8CED97E05BC06BEA73E081E32F
:106C900094E10E9429D0892B79F4E4ECF7E0849107
:106CA0008F010F5F1F4F882321F00E947840F80169
:106CB000F6CF83EB97E044C066EB73E081E394E1A9
:106CC0000E9429D0892B79F4EAE9F7E084918F01B9
:106CD0000F5F1F4F882321F00E947840F801F6CF04
:106CE00088E897E02DC062EC73E081E394E10E94B4
:106CF00029D0892B79F4EDE6F7E084918F010F5FBD
:106D00001F4F882321F00E947840F801F6CF8BE5D1
:106D100097E016C060ED73E081E394E10E9429D012
:106D2000892BA9F4E1E4F7E084918F010F5F1F4FF5
:106D3000882321F00E947840F801F6CF8FE297E097
:106D40009093680D8093670D0E94A44083C06DED01
:106D500073E081E394E10E9429D0892B09F07AC085
:106D600010924F1477C01D8218861C821B8285EEFC
:106D700092E09A83898380914810811103C062E276
:106D800070E102C061E470E16115710519F06C5F9A
:106D90007F4F02C060E070E021E041E354E1CE01AA
:106DA00005960E947C97882361F18BE1FE01359660
:106DB000A5E4B0E101900D928A95E1F72B813C8129
:106DC0003093441020934310809196118A3008F03C
:106DD0003DC091E0980F90939611FFE18F9FC00105
:106DE0001124DC01AC59BF4E4BE1E5E4F0E1019028
:106DF0000D924A95E1F7FC01E05AFF4E338322835E
:106E000025C0EFEFFAE184918F010F5F1F4F8823B8
:106E100021F00E947840F801F6CFE9E1F7E0849193
:106E20008F010F5F1F4F882321F00E947840F801E7
:106E3000F6CF01E314E1F80181918F01882319F065
:106E40000E947840F8CF8AE00E947840CE010196F7
:106E50000E944F51109231148091090180FF07C1A7
:106E6000EAEBFBE084918F01882311F40C945D2DF3
:106E7000082E000C990B0E941E770F5F1F4FF80120
:106E80008491F2CF8FE40E9452B881110C945D2D51
:106E900083E40E9452B80C945D2D83E50E9452B8A1
:106EA000811159C08FE40E9452B8882319F082E8FA
:106EB0009BE007C084E50E9452B8882349F08AE528
:106EC0009BE09093680D8093670D0E94A44043C09F
:106ED00083E40E9452B8882319F081E39BE0F1CF4C
:106EE00081E50E9452B8882319F089E09BE0E9CF40
:106EF00088E40E9452B88823C9F0E5E0FBE0849161
:106F00008F01882351F0082E000C990B0E941E77E8
:106F10000F5F1F4FF8018491F4CF8DE090E00E9445
:106F20001E778AE090E00E941E7715C08CE40E94D4
:106F300052B8882381F0E1E0FBE084918F0188233F
:106F400061F3082E000C990B0E941E770F5F1F4FF4
:106F5000F8018491F4CFE9ECFBE084918F01882360
:106F600011F40C945D2D082E000C990B0E941E77D5
:106F70000F5F1F4FF8018491F2CF8091770F8091BE
:106F8000780F0C945D2D83E50E9452B8882309F494
:106F90006EC089ED9AE09093680D8093670D0E9412
:106FA000A440E9ECFBE084918F01882311F40C9458
:106FB0005D2D082E000C990B0E941E770F5F1F4F4E
:106FC000F8018491F2CFE4EDFAE084918F018823F7
:106FD00051F0082E000C990B0E941E770F5F1F4F77
:106FE000F8018491F4CFEFECFAE084918F018823CB
:106FF00011F40C945D2D082E000C990B0E941E7745
:107000000F5F1F4FF8018491F2CF88E50E9452B8BC
:10701000811106C089E50E9452B8882309F4C3C0D3
:1070200088E50E9452B8882341F080E79CE0909365
:10703000680D8093670D0E94A44089E50E9452B8B4
:10704000882341F08AE69CE09093680D8093670D59
:107050000E94A4408AE50E9452B8882341F084E649
:107060009CE09093680D8093670D0E94A4408091EE
:10707000FC139091FD13019664E070E00E949BCF99
:107080009093FD138093FC138091F8139091F91362
:1070900001969093F9138093F813109200141092B4
:1070A000FF130C943E2C4091FC135091FD139F0153
:1070B0002F5F3F4F309300142093FF1390E6949F6F
:1070C0009001959F300D112428583D4EE20FF31F7B
:1070D00080830C943E2C00910114109102147801CD
:1070E00024E0E20EF11C6AE270E0C7010E941ED0AB
:1070F000F80124812F3221F4B8016B5F7F4F03C068
:107100002C3339F4B70181E394E10E9432D00C941E
:107110005D2D10923114009719F0FC013197108207
:10712000809101149091021440E061E004960E9465
:107130007EB68091C111882389F0EBE8FCE0849150
:107140008F01882309F425CB082E000C990B0E948F
:107150001E770F5F1F4FF8018491F3CFE7E8FCE043
:1071600084918F01882309F414CB082E000C990B0D
:107170000E941E770F5F1F4FF8018491F3CF0E948A
:107180006578E3E8FCE084918F01882311F40C9486
:107190005D2D082E000C990B0E941E770F5F1F4F6C
:1071A000F8018491F2CF8AE50E9452B8811138CF5C
:1071B00083E40E9452B8882309F459CF80E69CE00A
:1071C00050CF86E40E9452B8882309F44AC10E9435
:1071D0006DB80E94FBCD8B018CE59CE09093680D0F
:1071E0008093670DB1D788E50E9452B8882309F4CF
:1071F00050C00E946DB82B013C012DEC3CEC4CE4DE
:107200005EE30E9488C89E012F5F3F4F79011816E8
:1072100074F020E030E0A901C301B2010E94D8CE91
:1072200018162CF41F930F9381E59CE004C12DECFC
:107230003CEC4CEC5DEBC301B2010E9488C818160F
:107240007CF020E030E040E85FEBC301B2010E9437
:10725000D8CE18162CF41F930F9385E49CE0EBC056
:107260001F930F93C301B2010E94F6CD7F936F93DA
:107270008BE39CE09F938F93FF92EF920E945AC8FA
:107280000FB6F894DEBF0FBECDBFCE01019637D743
:10729000DFC089E50E9452B8882309F441C00E94EA
:1072A0006DB82B013C012DEC3CEC4CE45EE30E94FC
:1072B00088C8FE0131967F01181674F020E030E096
:1072C000A901C301B2010E94D8CE18162CF41F9355
:1072D0000F9380E39CE0AFC02DEC3CEC4CEC5DEBFD
:1072E000C301B2010E9488C818167CF020E030E08B
:1072F00040E85FEBC301B2010E94D8CE18162CF40F
:107300001F930F9384E29CE096C01F930F93C301D9
:10731000B2010E94F6CD7F936F938AE19CE0AACFE1
:107320008AE50E9452B8882309F441C00E946DB8D2
:107330002B013C012DEC3CEC4CE45EE30E9488C840
:10734000FE0131967F01181674F020E030E0A901AB
:10735000C301B2010E94D8CE18162CF41F930F93CC
:107360008FE09CE068C02DEC3CEC4CEC5DEBC30185
:10737000B2010E9488C818167CF020E030E040E896
:107380005FEBC301B2010E94D8CE18162CF41F93F4
:107390000F9383E09CE04FC01F930F93C301B20192
:1073A0000E94F6CD7F936F9389EF9BE063CF85E4D6
:1073B0000E9452B8882309F44BC00E946DB82B017B
:1073C0003C012DEC3CEC4CE45EE30E9488C8FE01DD
:1073D00031967F01181674F020E030E0A901C30156
:1073E000B2010E94D8CE18162CF41F930F938EEE84
:1073F0009BE021C02DEC3CEC4CEC5DEBC301B201F9
:107400000E9488C818167CF020E030E040E85FEB6E
:10741000C301B2010E94D8CE18162CF41F930F930B
:1074200082EE9BE008C0C301B2010E94F6CD7F93BB
:107430006F9387ED9BE09F938F93FF92EF920E9453
:107440005AC80F900F900F900F900F900F901DCF74
:1074500083ED9BE09093680D8093670D75D60C9437
:107460005D2D00E010E0B8CE20E030E040E251E4D5
:10747000609131047091320480913304909134040E
:107480000E9488C887FF07C08CEC9BE09093680D32
:107490008093670D59D682E390E090933C048093EB
:1074A0003B040E94967D88EC90E00E94BC75E9EC5C
:1074B000FBE084918F01882311F40C945D2D082E3C
:1074C000000C990B0E941E770F5F1F4FF8018491EB
:1074D000F2CF20E030E040E251E46091310470915D
:1074E000320480913304909134040E9488C887FF4D
:1074F00007C082EC9BE09093680D8093670D24D6C3
:1075000080E590E090933C0480933B040E94967D3C
:1075100080EF90E00E94BC75E9ECFBE084918F0164
:10752000882311F40C945D2D082E000C990B0E94F9
:107530001E770F5F1F4FF8018491F2CF80E090E03B
:107540000E94BC7510923C0410923B040E94967DF0
:10755000EEEBFBE084918F01882311F40C945D2DF8
:10756000082E000C990B0E941E770F5F1F4FF80129
:107570008491F2CF6F960FB6F894DEBF0FBECDBFE9
:10758000DF91CF911F910F91FF90EF90DF90CF90FF
:10759000BF90AF909F908F907F906F905F904F9033
:1075A0003F902F9008959091AD16E92FF0E0EF51A4
:1075B000F44F80839F5F943018F49093AD1602C00F
:1075C0001092AD168091AE168F5F8093AE1608951F
:1075D00080911C0B90911D0B981759F0E92FF0E04A
:1075E000E456F54F80819F5F9F7790931D0B90E04D
:1075F00008958FEF9FEF08950F931F93CF93DF931D
:10760000FC01A685B7858D0100581F4FE8018881D0
:10761000998101968F779927AD014E575F4FEA0107
:107620002881398128173907D1F3E8012881398168
:10763000A20FB31F6C93A685B785A058BF4F1196B4
:107640009C938E93A689B7892C9181E090E0078C5A
:1076500002C0880F991F0A94E2F7822B8C9381E075
:1076600081A30488F589E02D80818064808381E096
:1076700090E0DF91CF911F910F910895FC0181A1BE
:10768000882329F0A489B5898C9186FFFBCF11A2AC
:107690000895FC01A485B585FD01E058FF4F2081C8
:1076A00031813296808191812817390779F0808164
:1076B0009181A80FB91F8C91208131812F5F3F4F9D
:1076C0002F7733273183208390E008958FEF9FEF4A
:1076D0000895DC011C96ED91FC911D97DF01A058E7
:1076E000BF4F2D913C91119712968D919C911197BE
:1076F0002817390739F08D919C91E80FF91F808187
:1077000090E008958FEF9FEF0895FC012485358563
:10771000F901E058FF4F80819181329620813181BB
:1077200080589F4F821B930B60E870E00C949BCFB6
:107730000895089580E090E00895CF93FC012081A2
:107740002B33A1F02091AE16243080F4C62FBC015B
:107750008091AD16F0E68F9FC00111248A51944F9D
:107760000E9432D08C2F1FDF81E001C080E0CF91DA
:1077700008952F923F924F925F926F927F928F92D5
:107780009F92AF92BF92CF92DF92EF92FF920F93B0
:107790001F93CF93DF9300D000D0CDB7DEB79A838D
:1077A00089830E9416B6E981FA81C680D780E08479
:1077B000F184C114D104E104F10409F0ACC22485C0
:1077C000222309F469C332852150248721E0230F45
:1077D00022874585241301C01286E981FA8124E0BD
:1077E000329FE00DF11D1124C684D784E088F18812
:1077F000E981FA81C282D382E482F582DC01CB0185
:107800008C0D9D1DA11DB11D86839783A087B18717
:1078100084819581892B09F43FC3FFB7FD83F894D8
:10782000E981FA81228033802101612C712C04814D
:107830001581809139028F3121F08F3F09F068C2A4
:1078400005C0EFE1F9E124912E83DAC08FE1809346
:107850003902EFE1F9E184918E838F3F09F458C238
:10786000823009F469C030F5882309F44CC08130B6
:1078700009F0C6C0109280001092810080918100B2
:107880008860809381008091810081608093810075
:10789000EAEEF4E2E491F0E0EE0FFF1FE956FB4D53
:1078A00085919491E0E3F5E2E491E0934A04E1E00C
:1078B000EE8330C19E81943009F482C008F460C028
:1078C000953009F09DC01092200110922101809105
:1078D0002101886080932101809121018160809342
:1078E0002101EAEEF4E2E491F0E0EE0FFF1FE95629
:1078F000FB4D85919491E0E3F5E2E491E093470438
:1079000095E09E8307C114BC15BC84B5826084BD1C
:1079100085B5816085BDEAEEF4E2E491F0E0EE0F1A
:10792000FF1FE956FB4D85919491E0E3F5E2E49168
:10793000E0934B041E82ABC21092B0001092B100D3
:107940008091B00082608093B0008091B10081602E
:107950008093B100EAEEF4E2E491F0E0EE0FFF1F55
:10796000E956FB4D859194919093C60B8093C50B7E
:10797000E0E3F5E2E491E093C70BF2E0FE8387C217
:1079800010929000109291008091910088608093F5
:10799000910080919100816080939100EAEEF4E281
:1079A000E491F0E0EE0FFF1FE956FB4D85919491B5
:1079B000E0E3F5E2E491E093490423E02E83AAC0DA
:1079C0001092A0001092A1008091A1008860809385
:1079D000A1008091A10081608093A100EAEEF4E211
:1079E000E491F0E0EE0FFF1FE956FB4D8591949175
:1079F000E0E3F5E2E491E093480484E08E838AC0FA
:107A0000EE81E7FD85C161E08FE10E94DBB48E81EC
:107A10008D7F09F083C04801A12CB12C60E072E198
:107A20008AE790E0A50194010E94AECF29833A83B2
:107A30004B835C8369017A01F1E0CF1AD108E10838
:107A4000F1082FEFC216D104E104F10409F008F4A3
:107A50004EC060E472E48FE090E0A50194010E94C2
:107A6000AECF69017A0181E0C81AD108E108F108B6
:107A70009E81923009F5EFEFCE16D104E104F104B6
:107A800009F008F4CBC160E970ED83E090E0A50156
:107A900094010E94AECF69017A01F1E0CF1AD108BA
:107AA000E108F1082FEFC216D104E104F10411F04E
:107AB00008F041C183E027C08FEFC816D104E1046C
:107AC000F104B9F0B0F068E478EE81E090E0A5014F
:107AD00094010E94AECF69017A0191E0C91AD108E0
:107AE000E108F108EE81EE2309F49AC163C181E057
:107AF00001C082E09E81911106C095B5987F892BC7
:107B000085BD7AC085E09091B100987F892B8093E4
:107B1000B10072C061E08FE10E94DBB44801A12C8A
:107B2000B12C60E072E18AE790E0A50194010E9427
:107B3000AECF69017A01E1E0CE1AD108E108F1087F
:107B4000C114D104F1E0EF06F10488F068E478EEA6
:107B500081E090E0A50194010E94AECF69017A0115
:107B600081E0C81AD108E108F10883E001C081E092
:107B70009E81913071F490918100987F892B809340
:107B80008100452846284728D9F52FEF3FEFA90166
:107B900068C0EE81E33071F490919100987F892B59
:107BA0008093910045284628472851F52FEF3FEF55
:107BB000A90179C0FE81F43071F49091A100987F01
:107BC000892B8093A100452846284728C9F42FEF28
:107BD0003FEFA9017AC02E81253071F490912101E7
:107BE000987F892B8093210145284628472841F416
:107BF0002FEF3FEFA9017BC045284628472869F0B1
:107C0000D801AA0FBB1F91010E94A2CC28EE33E03D
:107C100040E050E00E9476CC03C02FEF3FEFA90177
:107C20008E81823081F12CF4882361F08130C9F09B
:107C30006FC09E81943009F448C0ACF1953009F4CE
:107C400056C066C0C7BC20935C0430935D0440936B
:107C50005E0450935F0480916E00826080936E009A
:107C600057C0D0928900C092880020935804309366
:107C7000590440935A0450935B0480916F008260D2
:107C800080936F0045C0C092B3002093C80B30931F
:107C9000C90B4093CA0B5093CB0B8091700082604C
:107CA0008093700035C0D0929900C09298002093C4
:107CB00054043093550440935604509357048091D4
:107CC000710082608093710023C0D092A900C0929D
:107CD000A8002093500430935104409352045093D1
:107CE00053048091720082608093720011C0D09220
:107CF0002901C092280120934C0430934D044093F5
:107D00004E0450934F0480917300826080937300FF
:107D1000ED81EFBFC1C0DC01CB018C199D09AE091B
:107D2000BF09B7FDB9C04698E981FA81168217826A
:107D300010861186B1C068E478EE81E090E0A5017C
:107D400094010E94AECF69017A01F1E0CF1AD10807
:107D5000E108F1082FEFC216D104E104F10441F16A
:107D600038F164E274EF80E090E0A50194010E9494
:107D7000AECF69017A01F1E0CF1AD108E108F1082C
:107D80002FEFC216D104E104F10409F008F4BACED1
:107D900062E17AE780E090E0A50194010E94AECF15
:107DA00069017A0181E0C81AD108E108F10819C017
:107DB00084E0A9CE2FEFC216D104E104F10409F04A
:107DC00008F463C062E17AE780E090E0A5019401E5
:107DD0000E94AECF69017A01F1E0CF1AD108E10823
:107DE000F1082FEFC216D104E104F104A9F0A0F0CC
:107DF00089819A81AB81BC812AE0B595A795979539
:107E000087952A95D1F76C017D01F1E0CF1AD10851
:107E1000E108F10887E077CE86E075CE82E073CE88
:107E2000EFEFCE16D104E104F10469F160F162E1F3
:107E30007AE780E090E0A50194010E94AECF69014D
:107E40007A0181E0C81AD108E108F1089FEFC9164C
:107E5000D104E104F104A9F0A0F089819A81AB81F9
:107E6000BC813AE0B595A795979587953A95D1F756
:107E70006C017D01E1E0CE1AD108E108F10885E04E
:107E80003CCE84E03ACE83E038CE84E033CE61E06D
:107E90008FE10E94DBB4BFCD26960FB6F894DEBF0B
:107EA0000FBECDBFDF91CF911F910F91FF90EF904B
:107EB000DF90CF90BF90AF909F908F907F906F900A
:107EC0005F904F903F902F9008950F931F93CF9303
:107ED000DF93CDB7DEB72C970FB6F894DEBF0FBE99
:107EE000CDBFE9E2F4E080859185A285B385448128
:107EF00055816681778100811181228133810983D7
:107F00001A832B833C834D835E836F8378878987B5
:107F10009A87AB87BC87AE01475F5F4FBE016B5F3F
:107F20007F4FCE0101960E94E8AA25E334E0AE011E
:107F3000475F5F4FBE016B5F7F4FCE0101960E948E
:107F400061BB2C960FB6F894DEBF0FBECDBFDF919C
:107F5000CF911F910F910895809118049091190469
:107F6000009731F04AE050E060E070E00C94DCC52E
:107F700060E070E0CB010895EFDF97FD0AC0ECDF11
:107F80006F3F71058105910509F02CF4E5DF862F1F
:107F9000089580E008958FEF0895809118049091DE
:107FA0001904892B31F0E8DF91E0811103C090E0E2
:107FB00001C091E0892F08950F931F93CF93809173
:107FC000180490911904009711F1FC018F01C191DF
:107FD0002C2F2F7DA9F0C53411F0C536B9F7F80163
:107FE000108260E070E080911804909119040E9462
:107FF00089C4F801C083562F472F382F292F0BC073
:1080000060E070E0CF911F910F910C9489C450E013
:1080100040E030E020E0652F742F832F922FCF9126
:108020001F910F91089581548A3108F042C0E82FC2
:10803000F0E04091D8165091D9166091DA167091FF
:10804000DB1604C076956795579547958A95D2F7C4
:10805000842F817040FF2FC0E254F94E9081992304
:1080600009F1E0919D16F0919E16E90FF11D9081A6
:1080700020ED290F2A3098F09E3211F491810CC026
:108080009D3211F09B3271F4918120ED290F2A303D
:1080900030F09E3239F4928190539A3018F42E2F9A
:1080A0009F2F02C020E090E02093180490931904C1
:1080B000089580E008950895B6DF882341F081E0B7
:1080C0002091180430911904232B09F480E00895BD
:1080D000FC01238121110C94E991089580E1E9E2EA
:1080E000F4E0A6E4BBE001900D928A95E1F70895D3
:1080F0009091C00095FFFCCF8093C6000895EF9249
:10810000FF921F93CF93DF937C0160E016DB182F63
:10811000882399F0EFEFFAE18491EF01219688230B
:1081200019F0E6DFFE01F8CFB70183E29DE00E947F
:10813000024F82E2DDDF8AE0DBDF812FDF91CF912A
:108140001F91FF90EF900895DF92EF92FF920F93AF
:108150001F93CF93DF93CDB7DEB76E970FB6F8942A
:10816000DEBF0FBECDBF6091670D7091680D6115C8
:10817000710541F14DE150E0CE0101967C010E9474
:1081800031C81E8EF7018F010E191F09D190DD2015
:1081900019F09AE0D912F7CFF701E00FF11F108222
:1081A000C701ADDF882371F0DD20A9F00F5F1F4FFD
:1081B0008091670D9091680D080F191F1093680D3D
:1081C0000093670D81E02091670D3091680D232B9E
:1081D00029F480E003C000E010E0F0CF6E960FB607
:1081E000F894DEBF0FBECDBFDF91CF911F910F91ED
:1081F000FF90EF90DF9008953F924F925F926F92C1
:108200007F928F929F92AF92BF92CF92DF92EF9226
:10821000FF920F931F93CF93DF931F92CDB7DEB7DB
:1082200093DF81116EC28091AE16843008F047C092
:10823000CFD9AC0197FF7CC142C08E3409F0D9C1BF
:108240000115110509F4D5C166E57EE0C8010E945B
:1082500040C87C01892B09F48EC16EE470E0C8012E
:1082600004960E941ED0009709F485C14AE050E0B0
:1082700060E070E001960E94DCC56093600470933A
:10828000610480936204909363048090BA16909086
:10829000BB16A090BC16B090BD162FEF821A920AA2
:1082A000A20AB20A681579058A059B0509F465C119
:1082B000EF2809F062C183E29EE00E9420B880911D
:1082C000F50F882309F41DC28091AE16811102C0FA
:1082D0001092C604EE24E39440916F1250917012F4
:1082E000609171127091721280916B1290916C1268
:1082F000A0916D12B0916E12481759076A077B075B
:1083000008F4E12C00E010E09924939480E6882E94
:108310009BE5A92E9EE0B92E2DE8322E8091AE1657
:10832000843008F0EEC1E110ECC18091C6048111E7
:10833000E8C18091C6119091C711A091C811B09168
:10834000C91180936F1290937012A0937112B09321
:10835000721241E050E0BE016F5F7F4F8EEB91E102
:108360000E947094019719F4898190E002C08FEF08
:108370009FEFF82E40906F12509070126090711223
:108380007090721240916B1250916C1260916D124C
:1083900070916E12EE24E394441655066606770635
:1083A00008F4E12C4416550666067706B0F40196EB
:1083B00009F46AC08AE0F81609F489C09DE0F9164C
:1083C00009F485C023E2F21619F08AE3F81296C088
:1083D0008091C504811192C06FC00E94D8698EEB54
:1083E00091E10E94E9918091D911882359F181503E
:1083F0008093D911389EC001112441E061E082527E
:108400009E4E0E947EB6E091D91194E0E99FF00162
:108410001124E652FE4E4081518162817381409366
:108420006F125093701260937112709372128EEBF0
:1084300091E10E94FF908091F60F8823A9F090921D
:10844000F50F12C01092F50F0E9493A60E94C57FEF
:108450000E94547F6D3371058105910528F0B0921B
:10846000680DA092670D70DE8091F50F811128C014
:10847000EEE6FEE084916F012FEFC21AD20A882344
:10848000D9F036DEF601F6CFEAEEFAE184916F011B
:108490009FEFC91AD90A882319F02ADEF601F6CF10
:1084A000EFE5FEE084916F012FEFC21AD20A882314
:1084B00019F01EDEF601F6CF83E2F81208C005C0FF
:1084C00023E2F2121BC100E010E09092C604109269
:1084D000C5040115110519F40E949A820CC08091FF
:1084E000AD16889E000D111D1124F801EA51F44FBC
:1084F000108280E058D800E010E010CF0F35110551
:1085000008F00CCF9BE3F91202C09092C504809151
:10851000C504811103CF8091AD16F801889EE00D4E
:10852000F11D1124EA51F44FF0820F5F1F4FF6CE78
:10853000982F2091B8163091B9168A3019F09D30D5
:1085400009F0AAC01092C4042115310519F40E9443
:108550009A8269CEF901EC59FB4F10821092B9163C
:108560001092B81604E614E0F8018191803209F007
:1085700064CE8F01F9CFC80179CE6AE270E0C801FC
:108580000E9456D09C01009701F1982F901BF12C6E
:10859000992339F09150F801E90FF11D8081F826F7
:1085A000F7CF4AE050E060E070E0C90101960E9418
:1085B000DCC5CF2CD12CE12CF12C6C157D058E0562
:1085C0009F0531F084E09EE078CE8AED9DE075CE87
:1085D0008091600490916104A0916204B091630461
:1085E0008093BA169093BB16A093BC16B093BD1699
:1085F0000EC08091F30F882351F064EE73E0C80140
:108600000E9429D0892B19F080EB9DE056CE8091F5
:10861000410281111FC067E470E0C8010E941ED0B2
:108620000097C1F04AE050E060E070E001960E94DF
:10863000DCC5643071058105910560F4E9E3FDE076
:1086400084917F019FEFE91AF90A882319F050DD20
:10865000F701F6CF68EE73E0C8010E9429D0892B9C
:1086600011F4109240026DEE73E0C8010E9429D00F
:10867000892B21F480E39DE00E94725162EF73E048
:10868000C8010E9429D0892B11F40E94318A61E02F
:1086900084E694E052D8C7CD2F3531050CF0C3CD18
:1086A0009C35C1F40E94E83A97FDBDCD2091C404E9
:1086B0002111B9CD2091B8163091B916A9014F5F9B
:1086C0005F4F5093B9164093B816F901EC59FB4F20
:1086D0008083A9CD9B3319F481E08093C4048091F9
:1086E000C4048111A0CDC90101969093B91680935D
:1086F000B816F901EC59FB4F408395CD1092C50493
:10870000EBCE0F90DF91CF911F910F91FF90EF90E3
:10871000DF90CF90BF90AF909F908F907F906F90A1
:108720005F904F903F9008958F929F92AF92BF922B
:10873000EF92FF920F931F93CF93DF93CDB7DEB7E6
:10874000A0970FB6F894DEBF0FBECDBF61157105BF
:108750008105910589F100E0842E912CA12CB12C8A
:10876000102FEE24E394F12CEC0EFD1EE00EF11C14
:1087700007FDFA94A50194010E9476CCF70160836D
:10878000B901CA010F5F611571058105910541F7B6
:108790001F3F21F1E1E0F0E0EC0FFD1FE10FF11DC3
:1087A00017FDFA9580818A3010F097E301C090E3BD
:1087B000890F9EDC1150ECCF80E3A0960FB6F894A1
:1087C000DEBF0FBECDBFDF91CF911F910F91FF9004
:1087D000EF90BF90AF909F908F908ACCA0960FB6ED
:1087E000F894DEBF0FBECDBFDF91CF911F910F91E7
:1087F000FF90EF90BF90AF909F908F900895CF9291
:10880000DF92EF92FF926B017C0197FF0AC08DE22D
:108810006FDCF094E094D094C094C11CD11CE11C96
:10882000F11C4AE0C701B601FF90EF90DF90CF90B6
:108830007BCF8F929F92AF92BF92CF92DF92EF92B7
:10884000FF92CF936B017C01B42E20E030E0A901B0
:108850000E9488C887FF06C08DE24ADCF7FAF094D0
:10886000F7F8F094C0E060E070E080E09FE3CB15A3
:1088700041F02DEC3CEC4CEC5DE30E94EDC8CF5F89
:10888000F6CF9B01AC01C701B6010E94B2CC6B01CF
:108890007C010E94FBCD4B015C014AE045DFCC230B
:1088A00079F1C501B4010E948CC89B01AC01C701DC
:1088B000B6010E94B1CC6B017C018EE219DC20E094
:1088C00030E040E251E4C701B6010E94EDC84B011F
:1088D0005C010E94F6CD6B01770FEE08FF08C7011F
:1088E000B6018DDFC701B6010E948EC89B01AC01A5
:1088F000C501B4010E94B1CC6B017C01C150F9F6F5
:10890000CF91FF90EF90DF90CF90BF90AF909F906E
:108910008F9008951F920F920FB60F9211240BB6ED
:108920000F922F938F939F93EF93FF9320911D0BA3
:10893000E0911C0B81E08E0F8F779091C600281775
:1089400029F0F0E0E456F54F9083E82FE0931C0BFC
:10895000FF91EF919F918F912F910F900BBE0F90F0
:108960000FBE0F901F9018959C0197FD0EC0843686
:10897000910584F064E670E00E949BCFCB016AE031
:1089800070E00E949BCF805D06C031952195310932
:108990008DE201C080E2809324042A30310564F026
:1089A000EAE0F0E0C901BF010E949BCFCB01BF010B
:1089B0000E949BCF805D01C080E280932504C901A5
:1089C0006AE070E00E949BCF805D8093260484E281
:1089D00094E008951F920F920FB60F9211240BB6D8
:1089E0000F922F933F938F939F93EF93FF93209139
:1089F000D6143091D7148091D8149091D914281797
:108A0000390731F4809131018F7D8093310114C099
:108A1000E091D814F091D914EA5AFB4E208180914C
:108A2000D8149091D91401968F7799279093D914DF
:108A30008093D81420933601FF91EF919F918F91ED
:108A40003F912F910F900BBE0F900FBE0F901F9074
:108A500018951F920F920FB60F9211240BB60F921A
:108A60002F934F935F938F939F93EF93FF938091F7
:108A7000300182FD1CC02091360180915A159091E1
:108A80005B1540915C1550915D1501968F77992784
:108A90004817590771F0E0915A15F0915B15E652AD
:108AA000FB4E208390935B1580935A1502C08091F2
:108AB0003601FF91EF919F918F915F914F912F918F
:108AC0000F900BBE0F900FBE0F901F9018958091C6
:108AD000770F9091780F891B8F7019F480E090E0E8
:108AE00008959091740F992351F0833030F48FEFF3
:108AF000890F19F08093740FF1CF1092740FE091E9
:108B0000780F88E5E89FF0011124E953FB4F80813D
:108B100080FDE4CF8091780F8F5F8F708093750F09
:108B20009091780F8091760F981304C08091750F03
:108B30008093760FCF0108950F930FB70F93009195
:108B40006E000F930B7F00936E0000916F000D7FFE
:108B500000936F000F930BB70F930CB70F921F92F8
:108B60002F933F934F935F936F937F938F939F9335
:108B7000AF93BF93EF93FF9311244AD0FF91EF91EE
:108B8000BF91AF919F918F917F916F915F914F9125
:108B90003F912F911F900F900CBF0F910BBF0F9122
:108BA0000260F89400936F000F9100936E000F9194
:108BB0000FBF0F91189580914C0A80FF03C08998D0
:108BC0008FEF02C0899A81E08093100280914C0A55
:108BD00081FF03C08F9A8FEF02C08F9881E080934E
:108BE000110280914C0A82FF09C080910B0180958F
:108BF000827080930901439A8FEF07C080910B0127
:108C0000827080930901439881E080931202089555
:108C10002F923F924F925F926F927F928F929F928C
:108C2000AF92BF92CF92DF92EF92FF920F931F937A
:108C3000CF93DF93CDB7DEB72D970FB6F894DEBF95
:108C40000FBECDBFF8948FEF9FEF90938900809374
:108C500088002AE02987212C312C44244A94542C62
:108C6000320178948091980A9091990AA0919A0A79
:108C7000B0919B0A892B8A2B8B2B09F010C2809113
:108C800084158823E1F010928415809182159091CB
:108C90008315892B09F403C210924D0A1092831593
:108CA000109282159091770F8091780F981709F4A0
:108CB000F6C18091780F8F5F8F708093780F8091CD
:108CC000821590918315892B09F4E9C1C090940A0B
:108CD000D090950AE090960AF090970A4091900AF9
:108CE0005091910A6091920A7091930A0091830ABF
:108CF00010E020E030E0DB01CA018C199D09AE09CB
:108D0000BF09081719072A073B0710F4D901C80142
:108D1000482F8C0D9D1DAE1DBF1D8093940A90930E
:108D2000950AA093960AB093970A209184003091F7
:108D30008500245E3F4FC090690AD0906A0AE09097
:108D40006B0AF0906C0A8091590A90915A0AA0918E
:108D50005B0AB0915C0A8C0D9D1DAE1DBF1D8093FA
:108D6000690A90936A0AA0936B0AB0936C0AB7FDE4
:108D70001CC0889AC0909115D0909215E0909315E0
:108D8000F090941580911002082E000C990BAA0BFC
:108D9000BB0B8C0D9D1DAE1DBF1D80939115909337
:108DA0009215A0939315B0939415C0906D0AD0902E
:108DB0006E0AE0906F0AF090700A80915D0A9091BF
:108DC0005E0AA0915F0AB091600A8C0D9D1DAE1DD8
:108DD000BF1D80936D0A90936E0AA0936F0AB093A3
:108DE000700AB7FD1CC08E9AC0909515D09096154C
:108DF000E0909715F090981580911102082E000CC4
:108E0000990BAA0BBB0B8C0D9D1DAE1DBF1D809336
:108E1000951590939615A0939715B0939815C090BB
:108E2000710AD090720AE090730AF090740A8091EF
:108E3000610A9091620AA091630AB091640A8C0D54
:108E40009D1DAE1DBF1D8093710A9093720AA09361
:108E5000730AB093740AB7FD3EC090914B0A80919B
:108E600012029923C1F09091490A92FF02C087FD36
:108E700005C09091480A992309F4BEC56091490A3A
:108E800070914A0A73FF02C087FD0CC09091470A97
:108E9000911108C006C090910B0190959870909325
:108EA0000901419AC0909915D0909A15E0909B15B0
:108EB000F0909C15082E000C990BAA0BBB0B8C0D87
:108EC0009D1DAE1DBF1D8093991590939A15A0937B
:108ED0009B15B0939C15C090750AD090760AE090CF
:108EE000770AF090780A8091650A9091660AA091BD
:108EF000670AB091680A8C0D9D1DAE1DBF1D809341
:108F0000750A9093760AA093770AB093780AB7FD12
:108F10003AC080909D1590909E15A0909F15B0909E
:108F2000A015C09013020C2C000CDD08EE08FF0801
:108F3000C80CD91CEA1CFB1CC0929D15D0929E1532
:108F4000E0929F15F092A015C090550AD090560A55
:108F5000E090570AF090580A8C199D09AE09BF0994
:108F60008093750A9093760AA093770AB093780A53
:108F700090914C0A8091810A93FF02C0815001C0F8
:108F80008F5F8093810A8091690A90916A0AA0910B
:108F90006B0AB0916C0AB7FD15C0C090550AD0900D
:108FA000560AE090570AF090580A8C199D09AE09AC
:108FB000BF098093690A90936A0AA0936B0AB093E1
:108FC0006C0A889880916D0A90916E0AA0916F0A40
:108FD000B091700AB7FD15C0C090550AD090560ADE
:108FE000E090570AF090580A8C199D09AE09BF0904
:108FF00080936D0A90936E0AA0936F0AB093700AE3
:109000008E988091710A9091720AA091730AB09122
:10901000740AB7FD3AC0C090550AD090560AE09045
:10902000570AF090580A8C199D09AE09BF09809320
:10903000710A9093720AA093730AB093740A809194
:109040004B0A8823E1F08091490A82FF04C0809195
:10905000120287FD05C08091480A882309F4D3C411
:109060008091490A90914A0A93FF04C080911202AC
:1090700087FD0BC08091470A811107C005C0809110
:109080000B018870809309014198415041F0809113
:1090900084009091850082179307C8F34CCE80918D
:1090A0001D0290911E02A0911F02B0912002892BF7
:1090B0008A2B8B2B09F08AC08091820A882309F4BD
:1090C00052C08090940A9090950AA090960AB09011
:1090D000970AC0907D0AD0907E0AE0907F0AF090B7
:1090E000800A8091810AC814D904EA04FB0488F438
:1090F00020914E0A30914F0A4091520A5091530AE2
:109100004217530730F481508093810A215031096E
:1091100015C08C149D04AE04BF04E8F420914E0ADF
:1091200030914F0A4091500A5091510A2417350747
:1091300090F48F5F8093810A2F5F3F4F30934F0AE7
:1091400020934E0A4091190250911A0260911B021D
:1091500070911C020BC04092190250921A02609248
:109160001B0270921C024FEF5FEFBA018091810ADF
:1091700087FD02C0169801C0169A20918400309194
:109180008500245E3F4F8091810A8823B9F0149AAC
:109190008091810A87FF02C08F5F01C08150809358
:1091A000810A14988091810A882369F38091840050
:1091B0009091850082179307C8F3E5CF40931D0275
:1091C00050931E0260931F02709320028091980AB0
:1091D0009091990AA0919A0AB0919B0A892B8A2BA7
:1091E0008B2B09F08FC3A0918215B0918315109736
:1091F00009F4AEC5C090940AD090950AE090960A02
:10920000F090970A4091900A5091910A6091920AC9
:109210007091930AC416D506E606F706D0F01092B0
:109220004D0A10928315109282159091770F8091BC
:10923000780F981709F48CC58091780F8F5F8F7025
:109240008093780F00ED802E07E0902EA12CB12C9A
:109250008AC140918C0A50918D0A60918E0A70915A
:109260008F0A4C155D056E057F0508F46DC04091B1
:10927000880A5091890A60918A0A70918B0AD29665
:109280000D911D912D913C91D597EE27419FF12D88
:10929000529FC001629F900D619F800D911D429F62
:1092A000F00D811D9E1F519FF00D811D9E1F609F1F
:1092B000F00D811D9E1F509FF10D8E1F9E1FF69574
:1092C0008E1F9E1F349F800D911D359F900D112480
:1092D000FD01EA5BFF4F0081118122813381080F7C
:1092E000191F211D311D0093840A1093850A2093B4
:1092F000860A3093870A3497C080D180E280F38059
:10930000C016D106E206F30640F4C092840AD09259
:10931000850AE092860AF092870AC090840AD0906B
:10932000850AE090860AF090870A82E896E121E0BB
:10933000FC0185909590A590B4908C149D04AE048A
:10934000BF0408F466C370C320917D0A30917E0A81
:1093500040917F0A5091800A29833A834B835C8332
:109360002C153D054E055F0508F070C04091790A47
:1093700050917A0A60917B0A70917C0A4A875B87D8
:109380006C877D87D2960D911D912D913C91D5973B
:10939000EE27419FF12D529FC001629F900D619F6A
:1093A000800D911D429FF00D811D9E1F519FF00D5C
:1093B000811D9E1F609FF00D811D9E1F509FF10D0E
:1093C0008E1F9E1FF6958E1F9E1F349F800D911D30
:1093D000359F900D11248C0120E030E08090840AAC
:1093E0009090850AA090860AB090870AFD01E65BFE
:1093F000FF4F081519052A053B05A0F4408151814E
:10940000628173814D835E836F837887801A910AAE
:10941000A20AB30A84169506A606B70638F44A01CE
:109420005B0104C080809180A280B38082E896E1D5
:1094300051E05D83FC01059115912591349108154A
:1094400019052A053B0508F473C380C38091810A7E
:109450008823D9F0D8964D915C91D99760E070E05F
:109460000091190210911A0220911B0230911C02E6
:10947000401751076207730741F010921D021092C6
:109480001E0210921F02109220024091150250916C
:109490001602609117027091180277FF5CC0AE5BF4
:1094A000BF4F8D919D910D90BC91A02D22E836E18A
:1094B00041E0F901C590D590E590F490C816D90621
:1094C000EA06FB0658F4B695A79597958795440F3D
:1094D0002C5F3F4F76E12E39370759F74093830AC7
:1094E00080329105A105B10520F480E290E0A0E072
:1094F000B0E08097A109B109811538E09307A10573
:10950000B10508F4DFC344E0949F900111242E5765
:109510003D4EF901329645915491EE27859FB00159
:10952000849F610D7E1F06946E1F7E1F1124CB0148
:10953000A0E0B0E0F9014591549160E070E0481B73
:10954000590B6A0B7B0B40931502509316026093E4
:109550001702709318028090150290901602A09046
:109560001702B09018028091821590918315892B73
:1095700009F0C0C1ACDA9093831580938215892BD2
:1095800009F4B8C1E0918215F0918315808183FFC1
:109590003EC085899689A789B08D80939115909357
:1095A0009215A0939315B0939415818D928DA38DF0
:1095B000B48D8093951590939615A0939715B093BD
:1095C0009815858D968DA78DB0A180939915909350
:1095D0009A15A0939B15B0939C1581A192A1A3A16C
:1095E000B4A180939D1590939E15A0939F15B09361
:1095F000A0159091770F8091780F981709F4BACF42
:109600008091780F8F5F8F708093780FB3CFC5886C
:10961000D688E788F08C81E0C114D104E104F1041C
:1096200009F480E0018D128D238D348D0115110513
:109630002105310509F08260458D568D678D70A139
:10964000411551056105710509F0846080934D0A4B
:109650001092790A10927A0A10927B0A10927C0A70
:109660001092880A1092890A10928A0A10928B0A24
:1096700085A196A1A7A1B0A58093900A9093910A85
:10968000A093920AB093930A882499245401881ACB
:10969000990AAA0ABB0A8092750A9092760AA09249
:1096A000770AB092780A8092710A9092720AA09218
:1096B000730AB092740A80926D0A90926E0AA09218
:1096C0006F0AB092700A8092690A90926A0AA09218
:1096D0006B0AB0926C0ACC0CDD1CEE1CFF1CC09215
:1096E000590AD0925A0AE0925B0AF0925C0A000F83
:1096F000111F221F331F00935D0A10935E0A2093EF
:109700005F0A3093600A440F551F661F771F40930E
:10971000610A5093620A6093630A7093640A41A1DC
:1097200052A163A174A1440F551F661F771F409378
:10973000650A5093660A6093670A7093680A880FF7
:10974000991FAA1FBB1F8093550A9093560AA09396
:10975000570AB093580A1092940A1092950A1092E0
:10976000960A1092970A82A593A5A4A5B5A5809301
:109770008C0A90938D0AA0938E0AB0938F0A86A5C7
:1097800097A5A0A9B1A980937D0A90937E0AA09382
:109790007F0AB093800A81A58093540A97A9909379
:1097A000820A992309F124AD35AD3093530A2093F1
:1097B000520A22AD33AD3093510A2093500A1092D1
:1097C0001D0210921E0210921F021092200240AD44
:1097D00051AD60E070E04093190250931A0260931B
:1097E0001B0270931C0208C04092190250921A0288
:1097F00060921B0270921C0296A920914C0A92134F
:109800000AC02091140230E0482F082E000C550B9E
:109810004217530729F090934C0A80931402CBD936
:109820008091D40B81110E94E5AB409215025092B9
:1098300016026092170270921802E0918215F09160
:109840008315EA5BFF4F80819181A281B381809370
:10985000840A9093850AA093860AB093870A22E827
:1098600036E141E0F901C590D590E590F490C81635
:10987000D906EA06FB0660F4B695A79597958795F5
:10988000440F2C5F3F4FEEE9F6E1E217F30751F783
:109890004093830A80329105A105B10520F480E24E
:1098A00090E0A0E0B0E08097A109B109811558E0EF
:1098B0009507A105B10508F428C264E0969F9001C0
:1098C00011242E573D4EF901329645915491EE27C1
:1098D000859FB001849F610D7E1F06946E1F7E1FC1
:1098E0001124F90185909490A12CB12C861A970A25
:1098F000A108B1088092980A9092990AA0929A0AB7
:10990000B0929B0A0091980A1091990A20919A0AA4
:1099100030919B0A40911D0250911E0260911F02DE
:1099200070912002F02E1983F22FE32F4017510778
:109930006207730720F4F42E5983F62FE72F8F2D3B
:109940009981AF2FBE2F0097E1E0AE07B10520F05F
:109950008FEF9FEFA0E0B0E0081B190B2A0B3B0B29
:109960000093980A1093990A20939A0A30939B0ABD
:109970004F3FFFEF5F076F077F0761F0481B590BF1
:109980006A0B7B0B40931D0250931E0260931F02D3
:1099900070932002F8942091840030918500205F1C
:1099A0003F4F498541504987442339F0280E391EDD
:1099B0002216330608F455C901C0190130928900F6
:1099C0002092880078942D960FB6F894DEBF0FBED3
:1099D000CDBFDF91CF911F910F91FF90EF90DF905E
:1099E000CF90BF90AF909F908F907F906F905F903F
:1099F0004F903F902F90089590910B019095987003
:109A0000909309013BCA80910B01887080930901F2
:109A100027CBF694E794D794C794220F0496E6E1F7
:109A20008E399E0709F084CC2093830AF0E2CF168A
:109A3000D104E104F10428F410E2C12ED12CE12C70
:109A4000F12C30E2C31AD108E108F108C11488E012
:109A5000D806E104F104F8F0E4E0DE9EC001112430
:109A60008E579D4EFC01329625913491FC2DEE27A8
:109A7000F39F8001F29F010D1E1F06940E1F1E1FF3
:109A80001124FC0185909490A12CB12C801A910A8C
:109A9000A108B10822C09701860136952795179530
:109AA0000795F801EC7F9F012E57314FF901859002
:109AB0009490F901329685919491EC2DE770E89F8E
:109AC0009001E99F300D1124F3E036952795FA9522
:109AD000E1F7821A930AA12CB12C480D591D6A1D79
:109AE0007B1D4093880A5093890A60938A0A709379
:109AF0008B0A9091820A8091810A992309F474C09B
:109B0000882309F430CDD8968D919C91D997A0E007
:109B1000B0E04091190250911A0260911B027091BD
:109B20001C0284179507A607B70709F060C01BCD74
:109B3000B694A794979487944D81440F4D830496CF
:109B40006EE976E16817790709F074CC2D812093CE
:109B5000830A30E283169104A104B10428F450E290
:109B6000852E912CA12CB12C60E2861A9108A108B7
:109B7000B108811478E09706A104B10408F440C04C
:109B8000E4E09E9EC00111248E579D4EFC0132964A
:109B900025913491F82DEE27F39F8001F29F010D5E
:109BA0001E1F06940E1F1E1F1124FC018590949009
:109BB000A12CB12C801A910AA108B1084A855B85B5
:109BC0006C857D85480D591D6A1D7B1D4093790A62
:109BD00050937A0A60937B0A70937C0A8091820A80
:109BE000811132C08091810A882309F4BCCC109283
:109BF0001D0210921E0210921F0210922002B3CC7E
:109C0000950184013695279517950795F801EC7F06
:109C10009F012E57314FF90185919491F9013296A8
:109C200005911491E82DE770E09F9001E19F300DC0
:109C3000112443E0369527954A95E1F74C01821AA5
:109C4000930AA12CB12CBACF49815A816B817C81B6
:109C50002D81420F511D611D711D4C155D056E0555
:109C60007F05C8F48091810A882309F47CCCD896BA
:109C70004D915C91D99760E070E0009119021091CC
:109C80001A0220911B0230911C02401751076207F3
:109C9000730709F468CC10921D0210921E021092F4
:109CA0001F0210922002D8968D919C91D997A0E026
:109CB000B0E08093190290931A02A0931B02B09314
:109CC0001C0251CCAC01BD0176956795579547951F
:109CD000FA01EC7F9F012E57314FF90145915491C4
:109CE000F9013296659174918770869F9001879FE4
:109CF000300D1124C901F3E096958795FA95E1F7A7
:109D0000481B590B60E070E01ECCAC01BD0176959C
:109D1000679557954795FA01EC7F9F012E57314F74
:109D2000F90185909490F90132964591549187708C
:109D3000849F9001859F300D1124C901A3E0969561
:109D40008795AA95E1F7881A990AA12CB12CD2CD52
:109D500080ED882E87E0982EA12CB12C0BCCCF92D1
:109D6000DF92EF92FF92CF93DF936A017B01FC01B8
:109D70008491EF012196882321F00E947840FE0112
:109D8000F7CF4AE0C701B601DF91CF91FF90EF9086
:109D9000DF90CF900C949443CF92DF92EF92FF929A
:109DA000CF93DF936A017B01FC018491EF0121963F
:109DB000882321F00E947840FE01F7CF42E0C701DE
:109DC000B601DF91CF91FF90EF90DF90CF900C9490
:109DD00019440F931F93CF93DF938B01FC01849160
:109DE000EF012196882321F00E947840FE01F7CFF1
:109DF000B801110F880B990BDF91CF911F910F9133
:109E00000C94FF430F931F93CF93DF938B01FC01BF
:109E10008491EF012196882321F00E947840FE0171
:109E2000F7CFE8018991882319F00E947840FACF92
:109E3000DF91CF911F910F9108950F931F93CF93AF
:109E4000DF9300D01F92CDB7DEB78C0108960E9439
:109E50006EAA69837A838B839C83B8016C5F7F4F82
:109E6000AE014F5F5F4FC8010E940DA99B01AC017D
:109E7000F80160857185828593850E94B1CCF801D7
:109E800060877187828793870F900F900F900F9054
:109E9000DF91CF911F910F91089586E40E941340A6
:109EA0008093C215882351F00E94DC3F60930C021E
:109EB00070930D0280930E0290930F0283E50E942F
:109EC0001340882351F00E94DC3F60930802709396
:109ED000090280930A0290930B0282E40E941340CD
:109EE000882351F00E94DC3F6093040270930502C6
:109EF000809306029093070208958FEF8EBD0DB4F4
:109F000007FEFDCF8EB50895CF92DF92EF92FF92BC
:109F1000CF93DF93EC01C090560BD090570BE0909D
:109F2000580BF090590BA7019601688179818A81BD
:109F30009B810E9488C887FF04C0C882D982EA82B8
:109F4000FB82C0905A0BD0905B0BE0905C0BF090C2
:109F50005D0BA70196016C817D818E819F810E949E
:109F600088C887FF04C0CC82DD82EE82FF82C09069
:109F70002702D0902802E0902902F0902A02A7013F
:109F80009601688179818A819B810E94D8CE1816BA
:109F900024F4C882D982EA82FB82C0902B02D0903E
:109FA0002C02E0902D02F0902E02A70196016C8108
:109FB0007D818E819F810E94D8CE181624F4CC8298
:109FC000DD82EE82FF82C0905E0BD0905F0BE0904E
:109FD000600BF090610BA7019601688579858A85F1
:109FE0009B850E9488C887FF04C0C886D986EA86F8
:109FF000FB86C0902F02D0903002E0903102F090AA
:10A000003202A7019601688579858A859B850E9421
:10A01000D8CE181624F4C886D986EA86FB86DF9146
:10A02000CF91FF90EF90DF90CF9008954F925F9285
:10A030006F927F928F929F92AF92BF92CF92DF9258
:10A04000EF92FF920F931F93CF93DF93D82EC82FD9
:10A05000D0E0FE01EA5FF74EC49082E0D81203C060
:10A0600081E080934B0A7E01EE0CFF1CEE0CFF1C7E
:10A07000F701E650F84E45905590659074906C2D20
:10A080000C2C000C770B880B990B0E948EC84B018F
:10A090005C0120E030E040EC5FE3C301B2010E94CC
:10A0A000EDC8A50194010E94EDC8AB01BC0100E020
:10A0B00010E098018D2D0E94929BF701E251F84E1D
:10A0C0002591359145915491C501B4010E94EDC887
:10A0D0004B015C0120E030E0A9010E9488C8882380
:10A0E00009F448C000E010E09801B501A4017058DF
:10A0F0008D2D0E94929BFE01E551F84EC491C11135
:10A1000017C0EFEFFAE18491EF012196882321F047
:10A110000E947840FE01F7CFE9ECF7E18491EF016E
:10A120002196882321F00E947840FE01F7CFCAE0F3
:10A13000F701E055FA4D45905590659074906C2F5D
:10A1400070E080E090E00E948EC89B01AC01C301EA
:10A15000B2010E948ECD2B013C01A5019401C501E5
:10A16000B4010E94B2CCAB01BC01930182018D2DE0
:10A170000E94929B82E0D81249C0409027165090CE
:10A1800028166090291670902A1620E030E0A90168
:10A19000C301B2010E94D8CE5301420187FF04C01F
:10A1A000B7FAB094B7F8B09420E030E0A901C50147
:10A1B000B4010E9488C8882349F120E030E0A90159
:10A1C000C301B2011C142CF40E94D8CE18162CF036
:10A1D00008C00E9488C887FF04C081E08093480AB5
:10A1E00003C081E08093470A1C1424F4B7FAB094AA
:10A1F000B7F8B09400E010E09801B501A40182E046
:10A200000E94929B1092480A1092470A10924B0AA1
:10A2100081E090E00D2C01C0880F0A94EAF790913C
:10A220002804982B909328049091450B892B8093B8
:10A23000450BF701E75CF44F108211821282138202
:10A240008D2D0E94F29DF701E354F84E8591959172
:10A25000A591B491E701C75DDB4F88839983AA83F9
:10A26000BB830E94653FF701EA5BF44F88819981C7
:10A27000AA81BB8180839183A283B383DF91CF9135
:10A280001F910F91FF90EF90DF90CF90BF90AF9014
:10A290009F908F907F906F905F904F90089525EEE4
:10A2A00032E0FC013183208304960C9468405F9A6D
:10A2B000809128048E7F809328048A9A479A8091FF
:10A2C00028048D7F809328048091080180958170F7
:10A2D00080930601479A809128048B7F80932804FD
:10A2E000129A0895EAEEFAE18491EF01219688230B
:10A2F00021F00E947840FE01F7CFEDE9F7E184916B
:10A30000EF012196882321F00E947840FE01F7CFCB
:10A310000E94DA7FCCDFE9E9F7E18491EF0188233D
:10A3200049F0082E000C990B0E941E772196FE0121
:10A330008491F5CF8DE090E00E941E778AE090E056
:10A340000E941E77FFEF2BE48DE1F150204080400A
:10A35000E1F700C00000F8949FEFE4E3FCE09150C7
:10A36000E040F040E1F700C000000E94DA7FA895CD
:10A37000FECF2F923F924F925F926F927F928F9279
:10A380009F92AF92BF92CF92DF92EF92FF920F9384
:10A390001F93CF93DF9300D01F92CDB7DEB70E94FB
:10A3A000342B0E9416B66B017C01109122021123FE
:10A3B00009F47BC080912B0B882309F476C040916F
:10A3C0006E0B50916F0B6091700B7091710B460189
:10A3D0005701841A950AA60AB70AB7FC78C08330D9
:10A3E00051F134F481300CF460C0EFEFFAE106C0B3
:10A3F000843009F05AC0EFEFFAE13BC084919F012D
:10A400002F5F3F4F3B832A83882329F00E947840A7
:10A41000EA81FB81F3CFE7E1F7E184919F012F5FB0
:10A420003F4F3B832A83882309F43FC00E94784032
:10A43000EA81FB81F2CFEFEFFAE184919F012F5F78
:10A440003F4F3B832A83882329F00E947840EA818A
:10A45000FB81F3CFE0E0F7E184919F012F5F3F4F55
:10A460003B832A83882309F10E947840EA81FB819B
:10A47000F3CF84919F012F5F3F4F3B832A83882333
:10A4800029F00E947840EA81FB81F3CFE8EEF6E103
:10A4900084919F012F5F3F4F3B832A83882329F0BC
:10A4A0000E947840EA81FB81F3CF212F30E0A8EEB3
:10A4B000B3E00E94A2CCC60ED71EE81EF91EC092C1
:10A4C0006E0BD0926F0BE092700BF092710B89B112
:10A4D00082FB882780F9809350149091511498172B
:10A4E0000CF049C08091521490915314A0915414CF
:10A4F000B09155140196A11DB11D883B3DE3930712
:10A50000A105B1054CF48093521490935314A09379
:10A510005414B09355143BC010925214109253141B
:10A5200010925414109255148091F50F882319F04D
:10A530000E9486781DC0E9E2F7E18491FB83EA83FB
:10A54000882371F0082E000C990B0E941E772A8137
:10A550003B812F5F3F4F3B832A83F9018491F0CFEA
:10A560008DE090E00E941E778AE090E00E941E77C6
:10A57000809150140AC0891751F010925214109211
:10A5800053141092541410925514809351148091C6
:10A59000AE16843010F40E94FC400E9416B6C090A3
:10A5A000300BD090310BE090320BF090330BC11494
:10A5B000D104E104F10481F100912C0B10912D0BD9
:10A5C00020912E0B30912F0B0C0D1D1D2E1D3F1DAC
:10A5D0004B015C01801A910AA20AB30AB7FC1CC0A5
:10A5E000EAEEFAE184919F012F5F3F4F3B832A837C
:10A5F000882329F00E947840EA81FB81F3CF6091A3
:10A600009D1670919E168FE597E1FCDB8AE00E9413
:10A61000784086E597E181C0C0902302D090240263
:10A62000E0902502F0902602C114D104E104F10467
:10A63000E9F13091770F2091780F321749F060934C
:10A640002C0B70932D0B80932E0B90932F0B2EC001
:10A6500000912C0B10912D0B20912E0B30912F0B74
:10A660000C0D1D1D2E1D3F1DDC01CB01801B910B10
:10A67000A20BB30BB7FD1AC05F9A809128048E7F9E
:10A68000809328048A9A479A809128048D7F80932A
:10A690002804809108018095817080930601479A73
:10A6A000809128048B7F80932804129A80917E0BDE
:10A6B00090917F0B909902C0019604C0181619065C
:10A6C0002CF4019790937F0B80937E0B80917E0BEF
:10A6D00090917F0B8E3E92400CF1EAEEFAE184916C
:10A6E0009F012F5F3F4F3B832A83882329F00E94DD
:10A6F0007840EA81FB81F3CFE6E3F7E184919F01A3
:10A700002F5F3F4F3B832A83882329F00E947840A4
:10A71000EA81FB81F3CF8DE297E1E4DD0E9416B67A
:10A7200000917A0B10917B0B20917C0B30917D0B6B
:10A730004B015C01801A910AA20AB30AB7FC4EC011
:10A740008B019C010C53164F2F4F3F4F00937A0BF8
:10A7500010937B0B20937C0B30937D0B4F9BA9C1F7
:10A760007A9BA7C12091060120FFA3C12091C715A4
:10A7700021119FC1379B9DC1379B9BC1029B99C1F2
:10A780000091760B1091770B2091780B3091790B1B
:10A79000011511052105310599F0DC01CB01801B64
:10A7A000910BA20BB30B80569A4EA109B1098827D1
:10A7B000B7FD83959927AA27BB27682F619501C00C
:10A7C00060E0262F30E08091020161118095807158
:10A7D00080930001B90187E00E9417B59091770F2F
:10A7E0008091780F981791F0E091780F28E5E29F1B
:10A7F000F0011124E75EFA4F60818091780F90910B
:10A80000770F981729F08F5F8F70F9CF6091390417
:10A8100070E089E00E9417B58091C215882309F481
:10A82000F8C0009108021091090280900A028C82FF
:10A8300090900B029A8260914104709142046E5F85
:10A840007F4F072E000C880B990B0E948EC8980131
:10A85000A4010E9488C887FDDCC0F090780F212CED
:10A86000312CE12C19828091770F8F1509F462C089
:10A870008F2D90E038E5A32EA89EF001A99EF00D43
:10A880001124E953FB4F458956896789708D452B03
:10A89000462B472B81F4418D528D638D748D452B52
:10A8A000462B472B41F4458D568D678D70A1452B66
:10A8B000462B472BD1F128E5B22EB89E9001B99EC8
:10A8C000300D1124C90189539B4F6C01FC0161813A
:10A8D0007281838194810E941DCF4B015C01F6013E
:10A8E00061A172A183A194A10E948CC82B013C019B
:10A8F000F60165A176A187A190A50E948CC89B0155
:10A90000AC01C301B2010E948ECDA50194010E9449
:10A91000EDC85B016C0191014E2D59810E94D8CE8A
:10A9200018161CF41501EC2CD98281E08F0D8F7064
:10A93000F82E99CF20910C0230910D0240910E0219
:10A9400050910F02B1018E2D99810E94EDC898019E
:10A950004C815A810E94B2CC6B017C019B01AC01FD
:10A96000B8018C819A810E94D8CE1816ACF0009163
:10A97000040210910502809006028C8290900702DA
:10A980009A829801A401B601C7010E94D8CE181678
:10A990001CF08601EC82FA82C090720BD090730B8F
:10A9A000E090740BF090750B98014C815A81C701AF
:10A9B000B6010E94D8CE1816D4F420E037ED43EA51
:10A9C0005CE3B8018C819A810E94EDC84B015C0167
:10A9D00028E431EE4AE75FE3C701B6010E94EDC803
:10A9E000A50194010E94B2CC8B018C839A83C8018B
:10A9F000AC81BA818093720B9093730BA093740B0C
:10AA0000B093750BB801CD010E94F6CDCB010E9429
:10AA1000BC750E949A8285ED9FE00E94B93BA09090
:10AA2000380BA982AA2009F44DC00E9416B60091E5
:10AA3000340B1091350B2091360B3091370BDC0124
:10AA4000CB01801B910BA20BB30BB7FD3BC00E9447
:10AA500016B66B017C01B9802B2D30E0A8EEB3E077
:10AA60000E94A2CCC60ED71EE81EF91EC092340B5F
:10AA7000D092350BE092360BF092370B0E94DC7CC3
:10AA80008AE00F900F900F900F90DF91CF911F9160
:10AA90000F91FF90EF90DF90CF90BF90AF909F907D
:10AAA0008F907F906F905F904F903F902F900C947D
:10AAB00078406093760B7093770B8093780B90932C
:10AAC000790B5ECE0F900F900F900F90DF91CF918A
:10AAD0001F910F91FF90EF90DF90CF90BF90AF90BC
:10AAE0009F908F907F906F905F904F903F902F90AE
:10AAF00008952F923F924F925F926F927F928F9222
:10AB00009F92AF92BF92CF92DF92EF92FF920F93FC
:10AB10001F93CF93DF93CDB7DEB7CC54D1090FB6D7
:10AB2000F894DEBF0FBECDBF80912102882319F0BB
:10AB300086E49BE0E9D98091BD0B83FDA9C0C0905C
:10AB4000520BD090530BE090540BF090550B20918A
:10AB50003504309136044091370450913804C701D0
:10AB6000B6010E9488C8882309F492C08091BC0B6A
:10AB7000811133C060914304709144048091450475
:10AB8000909146040E94F6CD209137023091380210
:10AB90006217730714F5C0923504D0923604E09220
:10ABA0003704F0923804EFEFFAE184917F019FEFD0
:10ABB000E91AF90A882321F00E947840F701F5CFBD
:10ABC000EDECF6E184917F01AFEFEA1AFA0A8823EF
:10ABD00021F00E947840F701F5CF8090520B9090C1
:10ABE000530BA090540BB090550B2091350430912D
:10ABF00036044091370450913804C501B4010E94D5
:10AC0000B1CC6B017C0120E030E0A9010E94D8CEDC
:10AC100087FF04C0F7FAF094F7F8F094E0912A0B5C
:10AC2000B4E0EB9FF0011124ED5CFD4F20813181F8
:10AC300042815381C701B6010E94EDC820E030E097
:10AC400048E453E40E94D8CE181614F580923504D7
:10AC500090923604A0923704B0923804EFEFFAE1F4
:10AC600084917F019FEFE91AF90A882321F00E945D
:10AC70007840F701F5CFEEEAF6E184917F01AFEF7E
:10AC8000EA1AFA0A882321F00E947840F701F5CFEA
:10AC90008091A7166090020270900302C090460B4C
:10ACA000D090470BE090480BF090490B80904A0BF6
:10ACB00090904B0BA0904C0BB0904D0B882309F457
:10ACC00081C22090A8163090A9164090AA165090E4
:10ACD000AB1620E030E0A901C201B1010E9488C892
:10ACE000882379F020914E0B30914F0B4091500BFF
:10ACF0005091510BC201B1010E94D8CE18160CF030
:10AD000061C2B301770C880B990B0E948EC8209109
:10AD10004B0230914C0240914D0250914E020E94E4
:10AD2000EDC82AE037ED43E25CE30E94EDC86DA771
:10AD30007EA78FA798AB2091290430912A044091D7
:10AD40002B0450912C04C701B6010E94B1CC2B01F9
:10AD50003C0120912D0430912E0440912F045091FC
:10AD60003004C501B4010E94B1CC25966CAF7DAF13
:10AD70008EAF9FAF259720E030E0A901C301B2015B
:10AD80000E9488C8811141C020E030E0A9012596C9
:10AD90006CAD7DAD8EAD9FAD25970E9488C88111A9
:10ADA00034C070902A0B19AA1AAA1BAA1CAAC9821D
:10ADB000DA82EB82FC828D829E82AF82B88680919D
:10ADC0004E0B90914F0BA091500BB091510B898776
:10ADD0009A87AB87BC87AE01475F5F4FBE016B5F51
:10ADE0007F4FCE0101960E94E8AAFE01F1966F0105
:10ADF000E72C8E01035D1F4F22E53BE0AE01475F6C
:10AE00005F4FBE016B5F7F4F2AC2209131043091AA
:10AE10003204409133045091340460914E0B709190
:10AE20004F0B8091500B9091510B0E94B1CC299601
:10AE30006CAF7DAF8EAF9FAF2997209135043091D5
:10AE4000360440913704509138046091520B709150
:10AE5000530B8091540B9091550B0E94B1CC2196CD
:10AE60006CAF7DAF8EAF9FAF2197A3019201C3015D
:10AE7000B2010E94EDC86B017C0125962CAD3DAD61
:10AE80004EAD5FAD2597CA01B9010E94EDC89B0187
:10AE9000AC01C701B6010E94B2CC6B017C012996BE
:10AEA0002CAD3DAD4EAD5FAD2997CA01B9010E94F1
:10AEB000EDC89B01AC01C701B6010E94B2CC0E9453
:10AEC0001DCF6B017C012DEB37E346E855E30E9473
:10AED00088C887FF17C020E030E0A90121966CAD3B
:10AEE0007DAD8EAD9FAD21970E94D8CE2196CCAC82
:10AEF000DDACEEACFFAC219787FF04C0F7FAF0940D
:10AF0000F7F8F0942DEB37E346E855E3C701B601B7
:10AF10000E9488C887FDA6C120E030E040EA50E4E6
:10AF2000C701B6010E948ECD0E94FBCD1B01672B8D
:10AF300019F422242394312CB10180E090E00E9486
:10AF40008CC89B01AC0160E070E080E89FE30E9448
:10AF50008ECD4B015C019B01AC01C701B6010E9483
:10AF6000EDC82D966CAF7DAF8EAF9FAF2D97A5012D
:10AF70009401C301B2010E94EDC8698B7A8B8B8B5F
:10AF80009C8BA501940125966CAD7DAD8EAD9FADDA
:10AF900025970E94EDC86D8B7E8B8F8B988FA501B6
:10AFA000940129966CAD7DAD8EAD9FAD29970E9421
:10AFB000EDC8698F7A8F8B8F9C8FA50194012196A4
:10AFC0006CAD7DAD8EAD9FAD21970E94EDC86D8FAC
:10AFD0007E8F8F8F98A380E1E9E2F4E0DE01119685
:10AFE00001900D928A95E1F799249394F1E02F1A3C
:10AFF000310809F04BC0E0902A0B2D968CAD9DAD29
:10B00000AEADBFAD2D9789AF9AAFABAFBCAF80915E
:10B01000460B9091470BA091480BB091490B89A327
:10B020009AA3ABA3BCA380914A0B90914B0BA09128
:10B030004C0BB0914D0B8DA39EA3AFA3B8A78091ED
:10B040004E0B90914F0BA091500BB091510B89A7D3
:10B050009AA7ABA7BCA7AE01475D5F4FBE016B5D72
:10B060007F4FCE0181960E94E8AADE01D9966D013C
:10B070008E01035D1F4F22E53BE0AE01475D5F4F50
:10B08000BE016B5D7F4FCE018196EBC08091660B58
:10B09000811112C00E9416B6DC01CB0188539F4F6C
:10B0A000AF4FBF4F8093620B9093630BA093640BE1
:10B0B000B093650B9092660B0E949A820E9416B61E
:10B0C000C090620BD090630BE090640BF090650B26
:10B0D000DC01CB018C199D09AE09BF09B7FD11C078
:10B0E0000E9416B6DC01CB0188539F4FAF4FBF4F74
:10B0F0008093620B9093630BA093640BB093650BEA
:10B1000038D96E01B1E1CB0ED11CFE0131967F0121
:10B110005601D6012D913D914D915D916D01F70143
:10B1200060817181828193810E94B2CCD7016D933D
:10B130007D938D939D937D01AA16BB0651F7E090F8
:10B140002A0B2D968CAD9DADAEADBFAD2D978DABC1
:10B150009EABAFABB8AF89819A81AB81BC8189A32B
:10B160009AA3ABA3BCA38D819E81AF81B8858DA32B
:10B170009EA3AFA3B8A789859A85AB85BC8589A70F
:10B180009AA7ABA7BCA7AE01475D5F4FBE016B5D41
:10B190007F4FCE0181960E94E8AADE01D5966D010F
:10B1A0008E01035D1F4F9E01235F3F4FAE01475D40
:10B1B0005F4FBE016B5D7F4FCE018196D6D081116E
:10B1C00015CF19CFB301770C880B990B0E948EC84D
:10B1D00020914B0230914C0240914D0250914E0211
:10B1E0000E94EDC82AE037ED43E25CE30E94EDC81F
:10B1F00069AB7AAB8BAB9CAB70902A0B80914E0BFA
:10B2000090914F0BA091500BB091510BC982DA82F3
:10B21000EB82FC82898A9A8AAB8ABC8A89A39AA328
:10B22000ABA3BCA31DA61EA61FA618AAAE014F5D08
:10B230005F4FBE016F5E7F4FCE0101960E94E8AA6C
:10B24000FE01BD966F01E72C8E010F5C1F4F22E5BA
:10B250003BE0AE014F5D5F4FBE016F5E7F4FCE01A1
:10B26000019683D080E1E6E4FBE0A9E2B4E001903E
:10B270000D928A95E1F7C45BDF4F0FB6F894DEBFFD
:10B280000FBECDBFDF91CF911F910F91FF90EF9037
:10B29000DF90CF90BF90AF909F908F907F906F90F6
:10B2A0005F904F903F902F900895CF93DF9380E071
:10B2B0000E9466A6CEE1DBE0688379838A839B8364
:10B2C00081E00E9466A66C837D838E839F8382E0EB
:10B2D0000E9466A6688779878A879B87DF91CF91CE
:10B2E0000895CF93DF93E091AC16F0E0EF51F44F67
:10B2F0008081882381F0EBEAF6E18491EF012196C9
:10B30000882321F00E947840FE01F7CF8AE0DF9188
:10B31000CF910C947840DF91CF910895CF93DF9334
:10B3200080911C0B80931D0BE2EAF6E18491EF0102
:10B330002196882321F00E947840FE01F7CF80916A
:10B34000BA169091BB16A091BC16B091BD16BC0167
:10B35000CD016F5F7F4F8F4F9F4F0E94FF438AE069
:10B360000E947840DF91CF91BCCF2F923F924F92B5
:10B370005F926F927F928F929F92AF92BF92CF9285
:10B38000DF92EF92FF920F931F93CF93DF93CDB78E
:10B39000DEB7C857D1090FB6F894DEBF0FBECDBFD8
:10B3A000E091C415F091C515EF2B11F00C947E625D
:10B3B0002896DFAECEAE28976E2C79016A015B012C
:10B3C000FC0120813181428153816C962CAF3DAFCD
:10B3D0004EAF5FAF6C9720911517309116174091C3
:10B3E0001717509118176C966CAD7DAD8EAD9FAD53
:10B3F0006C970E94EDC80E94E3CEE0966CAF7DAFE3
:10B400008EAF9FAFE097D5018D919D910D90BC912E
:10B41000A02DA0968CAF9DAFAEAFBFAFA0972091EF
:10B42000191730911A1740911B1750911C17BC0126
:10B43000CD010E94EDC80E94E3CEE4966CAF7DAFD3
:10B440008EAF9FAFE497D6012D913D914D915C91C8
:10B45000A4962CAF3DAF4EAF5FAFA49720911D17C0
:10B4600030911E1740911F1750912017A4966CAD74
:10B470007DAD8EAD9FADA4970E94EDC80E94E3CE36
:10B48000E8966CAF7DAF8EAF9FAFE897D7012D9157
:10B490003D914D915C9122962CAF3DAF4EAF5FAF89
:10B4A0002297209121173091221740912317509114
:10B4B000241722966CAD7DAD8EAD9FAD22970E9474
:10B4C000EDC80E94E3CE60966CAF7DAF8EAF9FAFAC
:10B4D00060978091BD0B83FF1CC060962CAD3DAD85
:10B4E0004EAD5FAD60972093A90F3093AA0F4093A4
:10B4F000AB0F5093AC0F22968CAD9DADAEADBFADF2
:10B5000022978093990F90939A0FA0939B0FB093DB
:10B510009C0FD801BC91BDA3F801F181F9ABD80112
:10B520001296BC91BEABF801F381FAAF8091770F10
:10B530009091780F891B8F708F3019F40E94B95148
:10B54000F5CF0091770FE9960FAFE9978091770FCC
:10B55000082F10E01CA30BA380919D0F90919E0FCC
:10B56000A0919F0FB091A00FE0968CAC9DACAEACBB
:10B57000BFACE097881A990AAA0ABB0A8091A10F6A
:10B580009091A20FA091A30FB091A40FE4962CACC0
:10B590003DAC4EAC5FACE497281A390A4A0A5B0A04
:10B5A0008091A50F9091A60FA091A70FB091A80F21
:10B5B000E8962CAD3DAD4EAD5FADE897281B390B3D
:10B5C0004A0B5B0B2DA73EA74FA758AB8091A90F45
:10B5D0009091AA0FA091AB0FB091AC0F60960CADFB
:10B5E0001DAD2EAD3FAD6097081B190B2A0B3B0B11
:10B5F00009A71AA72BA73CA7012B022B032B09F4A1
:10B60000BCC08091BC0B81114BC060914304709110
:10B61000440480914504909146040E94F6CD209107
:10B62000370230913802621773070CF039C0609608
:10B630002CAD3DAD4EAD5FAD60972093A90F30931B
:10B64000AA0F4093AB0F5093AC0F22968CAD9DADDB
:10B65000AEADBFAD22978093990F90939A0FA093B0
:10B660009B0FB0939C0FEFEFFAE184918F010F5F76
:10B670001F4F811103C0E8E2F8E104C00E94784046
:10B68000F801F3CF84918F010F5F1F4F882321F0C2
:10B690000E947840F801F6CF19A61AA61BA61CA690
:10B6A00094E0699E800111240D5C1D4F69A57AA567
:10B6B0008BA59CA50E948EC8D8012D913D914D91DE
:10B6C0005C910E94EDC86B017C0120E030E0A90193
:10B6D0000E94D8CE87FF04C0F7FAF094F7F8F094F0
:10B6E0006091211770912217809123179091241750
:10B6F0000E94F6CD9B01AC01A8ECB0E00E9498CC72
:10B700000E948EC8A70196010E9488C887FF39C091
:10B7100060960CAD1DAD2EAD3FAD60970093A90FA7
:10B720001093AA0F2093AB0F3093AC0F22962CAD41
:10B730003DAD4EAD5FAD22972093990F30939A0F98
:10B7400040939B0F50939C0FEFEFFAE184918F0190
:10B750000F5F1F4F811103C0E9E0F8E104C00E94B0
:10B760007840F801F3CF84918F010F5F1F4F88233A
:10B7700021F00E947840F801F6CF19A61AA61BA660
:10B780001CA6D501C4018827B7FD83959927AA2750
:10B79000BB27782E57FE03C0382F3260732E8DA53D
:10B7A0009EA5AFA5B8A9B7FF03C0972D9460792EC9
:10B7B00009A51AA52BA53CA537FF03C0172D1860B6
:10B7C000712E24E0629E800111240D5C1D4F69A53D
:10B7D0007AA58BA59CA50E948EC8D8012D913D917C
:10B7E0004D915C910E94EDC86B017C0120E030E03E
:10B7F000A9010E94D8CE87FF04C0C701B6019058A6
:10B8000002C0C701B60120E030E040E05FE30E94E3
:10B81000B2CC0E94FBCD6AAB7BAB8CAB9DAB88E519
:10B820000BA11CA1809FF001819FF00D1124E95311
:10B83000FB4F108276AAB501A401B7FE07C04427CA
:10B840005527BA01481959096A097B0988E50BA1EE
:10B850001CA1809FF001819FF00D1124E953FB4F43
:10B86000458B568B678B708F2C962CAE3DAE4EAEB3
:10B870005FAE2C9757FE0DC088279927DC018219EF
:10B880009309A409B5092C968CAF9DAFAEAFBFAF9D
:10B890002C9728E50BA11CA1209FF001219FF00D02
:10B8A0001124E953FB4F2C968CAD9DADAEADBFADD1
:10B8B0002C97818F928FA38FB48F0DA51EA52FA5D6
:10B8C00038A937FF07C030952095109501951F4F77
:10B8D0002F4F3F4FE8E57E2EABA1BCA17A9EF00131
:10B8E0007B9EF00D1124E953FB4F058F168F278F98
:10B8F00030A38AA99BA9ACA9BDA981A392A3A3A3A4
:10B90000B4A323964FAF2397752EF62FE72F2C96CF
:10B910008CAD9DADAEADBFAD2C97481759076A07EA
:10B920007B0778F429969FAD299723969FAF23979D
:10B930002A967FAC2A972B96FFAD2B972C96EFADCE
:10B940002C9723968FAD2397972DAF2FBE2F80175F
:10B950009107A207B30710F4D901C8010AA91BA9CE
:10B960002CA93DA980179107A207B30710F4D901AC
:10B97000C80128E50BA11CA1209FF001219FF00D1B
:10B980001124E953FB4F85A396A3A7A3B0A706975D
:10B99000A105B10508F4ABC5DF01AE5ABF4F8091D8
:10B9A000390490913A048D939C9361A6452B462BC4
:10B9B000472B09F05F9888E50BA11CA1809FF0013F
:10B9C000819FF00D1124E953FB4F818D928DA38D42
:10B9D000B48D892B8A2B8B2B11F08A98479888E598
:10B9E0000BA11CA1809FF001819FF00D1124E95350
:10B9F000FB4F858D968DA78DB0A1892B8A2B8B2B24
:10BA000031F08091080181708093060147982AA93E
:10BA10003BA94CA95DA9232B242B252B09F470C528
:10BA20008091C20B882319F081508093C20B611062
:10BA300004C0129880E28093C20B6090B80B7090A3
:10BA4000B90B0091BA0B1091BB0B9301A8016DA12A
:10BA500079A98EA99AAD0E9488C887FF04C06DA2FB
:10BA600079AA0EAB1AAFC501B4010E948EC820910D
:10BA700005173091061740910717509108170E943B
:10BA8000EDC826966CAF7DAF8EAF9FAF2697698BC2
:10BA90007A8B8B8B9C8BC201B1010E948EC8209146
:10BAA000091730910A1740910B1750910C170E94FB
:10BAB000EDC82B013C016D8B7E8B8F8B988F6DA514
:10BAC0007EA58FA598A90E948EC820910D17309150
:10BAD0000E1740910F17509110170E94EDC84B019F
:10BAE0005C01698F7A8F8B8F9C8F20911117309119
:10BAF00012174091131750911417C701B6010E94F5
:10BB0000EDC86B017C016D8F7E8F8F8F98A388E5C8
:10BB10000BA11CA1809FF001819FF00D1124E9531E
:10BB2000FB4F258936894789508D2DA73EA74FA702
:10BB300058AB263031054105510508F4EAC4289672
:10BB4000AEADBFAD2897CD90DD90ED90FC9020E09C
:10BB500030E0A901C701B6010E9488C88111F8C46C
:10BB600026962CAD3DAD4EAD5FAD2697CA01B9010D
:10BB70000E94EDC86B017C01A3019201C301B201D7
:10BB80000E94EDC89B01AC01C701B6010E94B2CC76
:10BB90006B017C01A5019401C501B4010E94EDC8AF
:10BBA0009B01AC01C701B6010E94B2CC0E941DCF1F
:10BBB00028E50BA11CA1209FF001219FF00D11246D
:10BBC000E953FB4F658776878787908B88E50BA1C4
:10BBD0001CA1809FF001819FF00D1124E953FB4FC0
:10BBE0004584568467847088A301920160E070E008
:10BBF00080E89FE30E948ECD64966CAF7DAF8EAFE0
:10BC00009FAF64972DA139A94EA95AAD0E94EDC8E6
:10BC10004B015C018091770F9091750F891B8F709C
:10BC200027968FAF2797A501940160E074E284E71F
:10BC300099E40E948ECD0E94E3CE6B017C01279691
:10BC40008FAD27978250863008F491C4A5019401E6
:10BC5000C301B2010E94EDC89B01AC010E94EDC876
:10BC600068966CAF7DAF8EAF9FAF689788E5ABA14C
:10BC7000BCA18A9F80018B9F100D112409531B4F7B
:10BC800068962CAD3DAD4EAD5FAD6897D80111966D
:10BC90002D933D934D935C93149795962D913D91E3
:10BCA0004D915C9198972EAB3FAB48AF59AFCA010D
:10BCB000B9010E948CC86AAF7BAF8CAF9DAF9B016E
:10BCC000AC01C501B4010E94EDC80E9478CD0E946C
:10BCD000FBCDA8966CAF7DAF8EAF9FAFA897F80154
:10BCE000EE5BFF4F60837183828393838E010F5ECF
:10BCF0001F4F2A961FAF0EAF2A97005111092496A5
:10BD00001FAF0EAF249700EA1BE0AC961FAF0EAF3B
:10BD1000AC978E010F5D1F4F1AA309A324960EAD99
:10BD20001FAD2497AA961FAF0EAFAA97312C212CD6
:10BD300010E81DA30FE309AB2A96AEADBFAD2A975D
:10BD40002D913D914D915D912A96BFAFAEAF2A974F
:10BD5000C501B4010E94EDC86B017C01AA96EEAD4D
:10BD6000FFADAA976193719381939193AA96FFAFC8
:10BD7000EEAFAA9720E030E0A9010E94D8CE87FF5D
:10BD800004C0F7FAF094F7F8F094AC96AEADBFADFE
:10BD9000AC974D905D906D907D90AC96BFAFAEAF7F
:10BDA000AC97A7019601C301B2010E9488C887FD24
:10BDB00018C409A11AA12A962EAD3FAD2A970217E1
:10BDC000130709F0B9CF20E030E040E85FE3632DCE
:10BDD000722D8DA199A90E9488C887FF58C07E0145
:10BDE00031E1E30EF11C24960EAD1FAD2497232DF7
:10BDF000322D4DA159A9D8016D917D918D919C91C4
:10BE00000E94EDC8F80161937193819391938F0122
:10BE1000EE16FF0661F728E50BA11CA1209FC001CB
:10BE2000219F900D11249C0129533B4F79018901D9
:10BE30000E5B1F4FA8966CAD7DAD8EAD9FADA897E4
:10BE40000E948CC8232D322D4DA159A90E94EDC806
:10BE50000E94FBCDD8016D937D938D939C93139796
:10BE6000232D322D4DA159A9632D722D8DA199A994
:10BE70000E94EDC868962CAD3DAD4EAD5FAD6897A4
:10BE80000E94EDC8F70161837283838394832AAD96
:10BE90003BAD4CAD5DAD64966CAD7DAD8EAD9FADF3
:10BEA00064970E94EDC86DA37EA38FA398A70DA5EC
:10BEB0001EA52FA538A9012B022B032B09F0A9C31E
:10BEC00088E52BA13CA1829F8001839F100D112446
:10BED00009531B4FF801818D928DA38DB48D892B51
:10BEE0008A2B8B2B09F095C3858D968DA78DB0A1DC
:10BEF000892B8A2B8B2B09F08CC320919C0B3091C2
:10BF00009D0B40919E0B50919F0B6DA17EA18FA127
:10BF100098A50E94EDC80E9478CD0E94FBCD2B0110
:10BF20003C01D801D7961C9288E52BA13CA1829FA9
:10BF30008001839F100D112409531B4FF801E25B10
:10BF4000FF4F4082518262827382C301B2010E941C
:10BF50008CC86B017C012DA13EA14FA158A50E9468
:10BF60008ECD6AAF7BAF8CAF9DAFD80151966D93EC
:10BF70007D938D939C9354972DEB37E346E051E4EA
:10BF8000C701B6010E94EDC80E94FBCDF80162AB6B
:10BF900073AB84AB95AB87A9882371F1FE96209192
:10BFA000900B3091910B4091920B5091930B6081CB
:10BFB0007181828193810E94EDC82AAD3BAD4CAD69
:10BFC0005DAD0E94EDC8209121173091221740915C
:10BFD0002317509124170E94EDC89B01AC0160E02B
:10BFE00074E284EF99E40E948ECD0E94FBCDD801CB
:10BFF000D9967C936E93D89788E50BA11CA1809F5E
:10C00000F001819FF00D1124E953FB4F2181328112
:10C01000438154812C962CAF3DAF4EAF5FAF2C9730
:10C02000CA01B9010E941DCF362E272E8C0140E88F
:10C030005BE062965FAF4EAF62973E0151E1650EE5
:10C04000711C80E89BE09FAB8EAB24964EAC5FAC3E
:10C05000249739A62DA60DA319AB1AAAD201CD900B
:10C06000DD90ED90FD902D0120E030E0A901C701A9
:10C07000B6010E94D8CE87FF04C0F7FAF094F7F813
:10C08000F094EEA9FFA981909190A190B190FFAB9F
:10C09000EEABA7019601C501B4010E9488C887FDD7
:10C0A000D4C564147504D1F627965FAD2797552340
:10C0B00009F444C6C090790FD0907A0FE0907B0FBE
:10C0C000F0907C0F2DEB37E346E855E3C701B6014E
:10C0D0000E9488C887FD32C6C701B6010E941DCFE5
:10C0E0006B017C019B01AC01632D722DC8010E9484
:10C0F00088C887FD03C03C2C2D2C87019601A70121
:10C10000632D722DC8010E948ECD68966CAF7DAFF5
:10C110008EAF9FAF68978DE79FE028969FAF8EAF59
:10C12000289720E030E040E85FE32AAB3BAB4CAB24
:10C130005DAB1EAA2896AEADBFAD28972D913D915F
:10C140004D915D912896BFAFAEAF289768966CADC4
:10C150007DAD8EAD9FAD68970E94EDC84B015C012F
:10C160002496EEADFFAD2497C190D190E190F1906F
:10C170002496FFAFEEAF2497FEA9FF2391F02AA9E2
:10C180003BA94CA95DA90E94EDC84B015C012AA9FD
:10C190003BA94CA95DA9C701B6010E94EDC86B017E
:10C1A0007C01A7019601C501B4010E94D8CE20E010
:10C1B00030E0A90118160CF08EC5C701B6010E9427
:10C1C000D8CE18160CF482C520E030E0A901C501D4
:10C1D000B4010E9488C887FD79C52601370177FA26
:10C1E000709477F87094A3019201C501B4010E9484
:10C1F000D8CE181614F4240135016296AEADBFAD49
:10C200006297CD90DD90ED90FD906296BFAFAEAF9E
:10C210006297A3019201C701B6010E9488C887FFF7
:10C2200015C0A3019201C701B6010E948ECD9B01EA
:10C23000AC016AA97BA98CA99DA90E94EDC86AAB33
:10C240007BAB8CAB9DABBEA9BF5FBEABEDE8FFE0A7
:10C2500028962EAD3FAD2897E217F30709F06ACF75
:10C260003EA9332361F02AA93BA94CA95DA9632DFE
:10C27000722DC8010E94EDC8362E272E8C0124EAAB
:10C2800030E74DE75FE3632D722DC8010E94EDC8D2
:10C290006B017C012091BE0B3091BF0B4091C00B14
:10C2A0005091C10B0E9488C887FD3EC589A59DA5F8
:10C2B000ADA1B9A98093BE0B9093BF0BA093C00B07
:10C2C000B093C10B28E54BA15CA1249FC001259F21
:10C2D000900D1124DC01A953BB4F7D01232D322D7C
:10C2E000A801632D722DC8010E94EDC8F701618776
:10C2F0007287838794876AAD7BAD8CAD9DAD905876
:10C300009B01AC010E94B2CCD7011D962D913D91AD
:10C310004D915C9150970E94EDC89B01AC016BE080
:10C3200077ED83E29BE30E94B1CC9B01AC018BE0F3
:10C3300097EDA3E2BBE3F70185839683A783B087DC
:10C3400010812C966CAD7DAD8EAD9FAD2C970E946B
:10C3500088C818160CF4F7C483E0182B88E52BA1C5
:10C360003CA1829FF001839FF00D1124E953FB4F04
:10C37000108380E1FE013196ADE7BFE001900D92A0
:10C380008A95E1F72C968CAD9DADAEADBFAD2C97E7
:10C390008093790F90937A0FA0937B0FB0937C0FCB
:10C3A000E0960CAD1DAD2EAD3FADE09700939D0F17
:10C3B00010939E0F20939F0F3093A00FE4962CAD07
:10C3C0003DAD4EAD5FADE4972093A10F3093A20F2A
:10C3D0004093A30F5093A40FE8968CAD9DADAEADE6
:10C3E000BFADE8978093A50F9093A60FA093A70FDA
:10C3F000B093A80F60960CAD1DAD2EAD3FAD60970C
:10C400000093A90F1093AA0F2093AB0F3093AC0F9A
:10C410006C962CAD3DAD4EAD5FAD6C9720938D0FFE
:10C4200030938E0F40938F0F5093900FA0968CAD4A
:10C430009DADAEADBFADA0978093910F9093920F3D
:10C44000A093930FB093940FA4960CAD1DAD2EAD99
:10C450003FADA4970093950F1093960F2093970FDD
:10C460003093980F22962CAD3DAD4EAD5FAD229727
:10C470002093990F30939A0F40939B0F50939C0FEA
:10C480009091770F8091780F981303C084E6809382
:10C49000740FE9968FADE9978F5F8F708093770F58
:10C4A0008091770F9091760F81508F7089134DC4D2
:10C4B0001091780F1BA30091770F09A728E51BA106
:10C4C00009A51013CDC4812C912CA12CB12C1DA633
:10C4D0001DA219AA1EAE212C312C00E010E029A5C6
:10C4E0003BA12313CAC42114310409F079C58091FA
:10C4F0006F00826080936F0081E0E2C680E0E0C65A
:10C500006090B40B7090B50B0091B60B1091B70B07
:10C510009CCA818D928DA38DB48D0697A105B1051E
:10C5200008F00DCB858D968DA78DB0A10697A1053E
:10C53000B10508F004CB20E030E0A901C701B60145
:10C540000E94D8CE87FF04C0F7FAF094F7F8F09471
:10C5500088E50BA11CA1809FF001819FF00D1124A3
:10C56000E953FB4FC586D686E786F08A2FCB8091AC
:10C57000B00B9091B10BA091B20BB091B30BC81658
:10C58000D906EA06FB0608F061CB8C199D09AE09B5
:10C59000BF09BC01CD01660F771F881F991F279621
:10C5A0004FAD2797042F10E020E030E0A90198015B
:10C5B0000E9476CCCA01B9010E948CC80E94E3CEC9
:10C5C0006C0D7D1D8E1D9F1D0E948CC89B01AC01B2
:10C5D00060E074E284E799E40E948ECD4B015C0137
:10C5E00035CBA7019601C301B2010E948ECD7B011C
:10C5F0008C019B01AC01632D722D8DA199A90E9424
:10C60000D8CE18160CF0D5CB3E2C2F2C0DA319AB81
:10C61000D0CB0AA91BA92CA93DA9012B022B032BC6
:10C6200049F02091980B3091990B40919A0B5091C1
:10C630009B0B08C02091940B3091950B4091960B69
:10C640005091970B6DA17EA18FA198A50E94EDC876
:10C650000E9478CD0E94FBCD2B013C012AA93BA969
:10C660004CA95DA9232B242B252BC9F020E030E019
:10C67000A9016091900B7091910B8091920B909118
:10C68000930B0E9488C8882351F081E009A51AA560
:10C690002BA53CA510161106120613060CF080E01F
:10C6A00098E52BA13CA1929F8001939F100D11242E
:10C6B00009531B4FD801D7968C93882309F4B2C035
:10C6C00020918D0F30918E0F40918F0F5091900FD0
:10C6D0006C966CAD7DAD8EAD9FAD6C970E94B1CC6C
:10C6E00069A77AA78BA79CA72091910F3091920FF1
:10C6F0004091930F5091940FA0966CAD7DAD8EAD8F
:10C700009FADA0970E94B1CC4B015C012091950F89
:10C710003091960F4091970F5091980FA4966CAD61
:10C720007DAD8EAD9FADA4970E94B1CC6B017C0115
:10C7300029A53AA54BA55CA5CA01B9010E94EDC87F
:10C7400069A77AA78BA79CA7A5019401C501B4018D
:10C750000E94EDC89B01AC0169A57AA58BA59CA59B
:10C760000E94B2CC4B015C01A7019601C701B60142
:10C770000E94EDC89B01AC01C501B4010E94B2CC7E
:10C780000E941DCF6B017C012091990F30919A0F6F
:10C7900040919B0F50919C0F22966CAD7DAD8EAD5C
:10C7A0009FAD22970E94B1CCA70196010E948ECD29
:10C7B0006B017C01F801FE96608371838283938311
:10C7C00020E030E040E450E40E94D8CE18161CF47B
:10C7D000F80117AA27C02091900B3091910B40913E
:10C7E000920B5091930BC701B6010E94EDC89B01BB
:10C7F000AC0160918C0B70918D0B80918E0B9091A0
:10C800008F0B0E948ECD2DA13EA14FA158A50E9455
:10C81000EDC80E94FBCD641575058605970510F4DB
:10C820002B013C018091E1169091E216A091E31654
:10C83000B091E4160EA91FA928AD39AD8017910754
:10C84000A207B30708F4DFC02DA53EA54FA558A940
:10C85000232B242B252B41F16091E5167091E616D0
:10C860008091E7169091E816641575058605970581
:10C87000D8F42EA93FA948AD59AD0E9467CC6B01F1
:10C880007C012DA53EA54FA558A9C301B2010E9468
:10C8900067CCC616D706E806F90630F4C701B6011C
:10C8A0000E9476CC29013A0188E50BA11CA1809F4A
:10C8B000F001819FF00D1124E953FB4FC18CD28C04
:10C8C000E38CF48CC114D104E104F10431F16091E2
:10C8D000E9167091EA168091EB169091EC166415AA
:10C8E000750586059705C8F42EA93FA948AD59AD31
:10C8F0000E9467CC4B015C01A7019601C301B20104
:10C900000E9467CC86169706A806B90630F4C501C2
:10C91000B4010E9476CC29013A0188E50BA11CA143
:10C92000809FF001819FF00D1124E953FB4FC58CCE
:10C93000D68CE78CF0A0C114D104E104F10431F1EC
:10C940006091ED167091EE168091EF169091F016B1
:10C950006415750586059705C8F42EA93FA948AD4D
:10C9600059AD0E9467CC4B015C01A7019601C30140
:10C97000B2010E9467CC86169706A806B90630F465
:10C98000C501B4010E9476CC29013A0188E50BA1CA
:10C990001CA1809FF001819FF00D1124E953FB4FF2
:10C9A000C1A0D2A0E3A0F4A0C114D104E104F10419
:10C9B00009F4BACA6091F1167091F2168091F316DB
:10C9C0009091F416641575058605970508F0ACCAB4
:10C9D0002EA93FA948AD59AD0E9467CC4B015C011F
:10C9E000A7019601C301B2010E9467CC8616970683
:10C9F000A806B90608F098CAC501B4010E9476CC11
:10CA000029013A0191CA2DA53EA54FA558A9232B6E
:10CA1000242B252BC9F16091E5167091E6168091C3
:10CA2000E7169091E816641575058605970560F57B
:10CA30000E948CC82AAD3BAD4CAD5DAD0E94EDC8E7
:10CA40006B017C016DA57EA58FA598A90E948CC85D
:10CA50004B015C01C301B2010E948CC8A501940185
:10CA60000E94EDC89B01AC01C701B6010E9488C8B5
:10CA700087FF0AC0A5019401C701B6010E948ECDAF
:10CA80000E94FBCD2B013C0188E50BA11CA1809FDE
:10CA9000F001819FF00D1124E953FB4F818C928CA2
:10CAA000A38CB48C81149104A104B104B9F16091F8
:10CAB000E9167091EA168091EB169091EC166415C8
:10CAC00075058605970550F50E948CC82AAD3BADCB
:10CAD0004CAD5DAD0E94EDC86B017C01C501B40198
:10CAE0000E948CC84B015C01C301B2010E948CC83A
:10CAF000A50194010E94EDC89B01AC01C701B601DC
:10CB00000E9488C887FF0AC0A5019401C701B60129
:10CB10000E948ECD0E94FBCD2B013C0188E50BA12C
:10CB20001CA1809FF001819FF00D1124E953FB4F60
:10CB3000858C968CA78CB0A081149104A104B104BB
:10CB4000B9F16091ED167091EE168091EF1690910B
:10CB5000F016641575058605970550F50E948CC87A
:10CB60002AAD3BAD4CAD5DAD0E94EDC86B017C01C3
:10CB7000C501B4010E948CC84B015C01C301B20124
:10CB80000E948CC8A50194010E94EDC89B01AC01D4
:10CB9000C701B6010E9488C887FF0AC0A501940199
:10CBA000C701B6010E948ECD0E94FBCD2B013C0136
:10CBB00088E50BA11CA1809FF001819FF00D11243D
:10CBC000E953FB4FC1A0D2A0E3A0F4A0C114D1044B
:10CBD000E104F10409F4A8C96091F1167091F2160C
:10CBE0008091F3169091F4166415750586059705E6
:10CBF00008F09AC90E948CC82AAD3BAD4CAD5DAD22
:10CC00000E94EDC84B015C01C701B6010E948CC8AF
:10CC10006B017C01C301B2010E948CC8A70196017F
:10CC20000E94EDC89B01AC01C501B4010E9488C8F7
:10CC300087FF7AC9A7019601C501B4010E948ECD74
:10CC40000E94FBCD2B013C016FC9FAA9FF2331F1F2
:10CC5000A5019401632D722DC8010E94EDC84B01FE
:10CC60005C0129A53DA54DA159A9C701B6010E94A6
:10CC7000EDC89B01AC01C501B4010E9488C887FFC3
:10CC800022C0A7019601C501B4010E948ECD69A7FB
:10CC90007DA78DA399AB21E02AAB03CAA70196011A
:10CCA000C501B4010E948ECD9B01AC0169A57DA593
:10CCB0008DA199A90E94EDC869A77DA78DA399AB05
:10CCC00031E03AABEEC941E04AABEBC9A7019601AE
:10CCD000C501B40113C0C701B6010E9488C887FD11
:10CCE00009C020E030E0A901C501B4010E94D8CEFE
:10CCF00018164CF4A5019401C701B6010E94B1CCED
:10CD00002B013C017ACA2401350177FA709477F837
:10CD10007094A3019201C701B6010E9488C887FDE3
:10CD20006CCA2601370169CA29A53DA54DA159A99B
:10CD3000C701B6010E9488C887FFB8CA39A42DA4CC
:10CD40000DA119A9B3CA81E008CBF090770F8FEF3E
:10CD50008F0D8F708BA3B090760F8091770FB816E0
:10CD600009F454C0C12CD12C0BA10B1509F44EC0F1
:10CD7000602E712C28E5269D8001279D100D112421
:10CD800009531B4FD8018C9183FD2BC00EAF1AABFA
:10CD90000115110541F11996BC91B9A7F801F28569
:10CDA000FDA7D8011B96BC91BDA3F801F485F9AB92
:10CDB000D80115962D903D904D905C901897A2014A
:10CDC000910169A57DA58DA19F2F0E9488C8811121
:10CDD00080C1C114D10439F0F601808180FD79C190
:10CDE00002C0CEAEDAAA8BA181508F708BA3809146
:10CDF000760F8B1103C0CEACDAA8B6CF0BA10B1502
:10CE000029F081E08B0D8F70B82EF1CF1091760F45
:10CE10001BA3C12CD12C8091770F0BA1801709F493
:10CE200047CB802E912C28E5289D8001299D100D4F
:10CE3000112409531B4FD8018C9183FD0AC058015E
:10CE4000C114D10439F0C6010E941286811102C0BA
:10CE5000BFC156018BA18F5F8F708BA36501DBCFA4
:10CE6000802F81508F70289FF0011124E953FB4FD0
:10CE7000908193FF28CB89A722CB48E5439FC0012F
:10CE80001124DC01A953BB4F1D018C9183FD19C0F6
:10CE900015966D917D918D919C9118970E941DCF53
:10CEA000F62EE72ED82EC92E0115110509F48AC0D9
:10CEB000F801808180FD0AC0D1018C9180FD06C0FF
:10CEC00081C0FDA4EDA0D9A8CEAC81C0F8018081BD
:10CED00081608083C8010E94128681116FC0F801B1
:10CEE00061817281838194810E941DCF2B013C015D
:10CEF0009B01AC0160E070E080E89FE30E948ECD72
:10CF00004B015C019B01AC016F2D7E2D8D2D9C2D65
:10CF10000E94EDC869837A838B839C832DA53DA1F4
:10CF200049A95EADC501B4010E94EDC8698B7A8B39
:10CF30008B8B9C8BAE014F5F5F4FBE016F5E7F4F4F
:10CF4000C8010E9436A7D801D7968C918823B1F1E9
:10CF50002091900B3091910B4091920B5091930B3B
:10CF6000F801FE9660817181828193810E94EDC8F3
:10CF700020912117309122174091231750912417A7
:10CF80000E94EDC84B015C019B01AC01C301B201E1
:10CF90000E94EDC80E94FBCDF80173AF62AFA501FE
:10CFA00094016F2D7E2D8D2D9C2D0E94EDC80E9429
:10CFB000FBCDD801DD967C936E93DC97F8018081E0
:10CFC0008E7F80838F2C9E2CAD2CBC2C81018BA15D
:10CFD0008F5F8F708BA3FDA6EDA2D9AACEAE7FCABC
:10CFE000D1018C9181608C93C8010E9412868111BD
:10CFF0006BC0F10161817281838194810E941DCF98
:10D000006B017C019B01AC0160E070E080E89FE374
:10D010000E948ECD2B013C012DEC3CEC4CE45DE3F9
:10D020000E94EDC869837A838B839C839401A50158
:10D03000C301B2010E94EDC8698B7A8B8B8B9C8BEC
:10D04000AE014F5F5F4FBE016F5E7F4FC1010E9417
:10D0500036A7D101D7968C918823B1F12091900BFE
:10D060003091910B4091920B5091930BF101FE96F0
:10D0700060817181828193810E94EDC82091211786
:10D080003091221740912317509124170E94EDC828
:10D090004B015C019B01AC01C701B6010E94EDC8C8
:10D0A0000E94FBCDF10173AF62AF2DEC3CEC4CE480
:10D0B0005DE3C501B4010E94EDC80E94FBCDD10122
:10D0C000DD967C936E93DC97F10180818E7F808367
:10D0D0000ECA28E5269DF001279DF00D1124E95385
:10D0E000FB4F808181FD43C0C114D10441F0D601C2
:10D0F0001596CD90DD90ED90FC90189708C08BE0D0
:10D10000C82E87EDD82E83E2E82E8BE3F82EB8E503
:10D11000B69DF001B79DF00D1124E953FB4F8189B5
:10D120009289A389B489BC01CD0190589B01AC01BF
:10D130000E94B2CCF80125853685478550890E942A
:10D14000EDC89B01AC01C701B6010E94B1CCE62E2F
:10D15000872E982EA92E262F372F482F592F69A5B5
:10D160007DA58DA199A90E9488C887FF04C0E9A464
:10D170008DA49DA0A9A82E2D382D492D5A2DC20170
:10D18000B1010E9488C8882309F42DCEF8E5F69DE8
:10D19000C001F79D900D11249C0129533B4F69015B
:10D1A000D9018C9181608C93C8010E9412868823DA
:10D1B00029F0F60180818E7F808315CE8E2D982DEB
:10D1C000A92DBA2DF60185839683A783B0870BCE50
:10D1D000D6018C9181FD52C0D60115962D913D91BD
:10D1E0004D915C91189729A73AA74BA75CA7150109
:10D1F000B5E02B0E311CF8014580568067807084A5
:10D20000A301920169A57AA58BA59CA50E9488C857
:10D2100087FF34C0F60181899289A389B489BC0152
:10D22000CD0190589B01AC010E94B2CCD6011D9655
:10D230002D913D914D915C9150970E94EDC89B01BD
:10D24000AC0169A57AA58BA59CA50E94B1CC6B0108
:10D250007C019B01AC01C301B2010E94D8CE18161B
:10D260006CF4D8018C9181608C93C5010E94128668
:10D270008823E1F0F80180818E7F808318E5189D76
:10D28000F001199DF00D1124E953FB4F21853285E2
:10D290004385548565817681878190850E9488C801
:10D2A0008111D8CD0BA10093760FD4CDD101CD92B1
:10D2B000DD92ED92FC9213970BA10093760FDECFD7
:10D2C000C858DF4F0FB6F894DEBF0FBECDBFDF9159
:10D2D000CF911F910F91FF90EF90DF90CF90BF9073
:10D2E000AF909F908F907F906F905F904F903F9006
:10D2F0002F9008958091770F9091780F891B8F70F0
:10D300008F3019F40E94B951F5CF8091770F8F5F5C
:10D310008F70E091770F98E59E9FF0011124E953FB
:10D32000FB4FDF011D929A95E9F798E090834091B9
:10D330009D0F50919E0F60919F0F7091A00F458B94
:10D34000568B678B708F4091A10F5091A20F609107
:10D35000A30F7091A40F418F528F638F748F4091F0
:10D36000A50F5091A60F6091A70F7091A80F458F40
:10D37000568F678F70A34091A90F5091AA0F6091AB
:10D38000AB0F7091AC0F41A352A363A374A3209180
:10D39000770F9091780F291303C094E69093740F40
:10D3A0008093770F80916F00826080936F00089563
:10D3B0009091770F8091780F981306C08091C415D3
:10D3C0009091C515892B19F00E94B951F1CF08959C
:10D3D000CF93DF938B3D9240B1F0EAEEFAE1849176
:10D3E000EF012196882321F00E947840FE01F7CFBB
:10D3F000E3E4F8E18491EF012196882331F00E9463
:10D400007840FE01F7CF80E001C081E0DF91CF914D
:10D4100008952F923F924F925F926F927F928F92D8
:10D420009F92AF92BF92CF92DF92EF92FF920F93B3
:10D430001F93CF93DF93CDB7DEB7C757D1090FB690
:10D44000F894DEBF0FBECDBF2DB63EB6A7961FAE79
:10D450001EAEA79784E690E0A9969FAF8EAFA997DE
:10D4600001E09E012B593F4F44E050E0BE01655A58
:10D470007F4FCE0189599F4F0E94A2AC9E012B592C
:10D480003F4F42E050E0BE0167597F4FCE018959BE
:10D490009F4F0E94A2AC43E050E0BE01655A7F4F0F
:10D4A00087ED92E00E9439D0892B09F43FC06F9636
:10D4B0008FAD6F97882339F08FE36C968FAF6C97A1
:10D4C0006D961FAE6D97EFEFFAE184917F012FEF1C
:10D4D000E21AF20A811103C0E6E0F9E104C00E94F9
:10D4E0007840F701F2CF84917F013FEFE31AF30A0E
:10D4F000882321F00E947840F701F5CFBE01655ADC
:10D500007F4F8DEF98E10E94024FEFEEF8E184919A
:10D510007F019FEFE91AF90A882321F00E947840E1
:10D52000F701F5CF81E08093C30B54C5EDB7FEB78B
:10D53000E696FFAFEEAFE6976B961CAE1DAE1EAE45
:10D540001FAE6B97A7961FAE1EAEA79701E09E0178
:10D550002B593F4F41E050E0BE0160597F4FCE0153
:10D5600089599F4F0E94A2AC80E1E3E5F2E0DE0121
:10D57000919601900D928A95E1F780E1E3E6F2E061
:10D58000DE01519601900D928A95E1F780E1E3E783
:10D59000F2E0DE01119601900D928A95E1F7E19695
:10D5A0004FADE19750E04D5F5F4F440F551F440F63
:10D5B000551F2DB73EB7241B350B0FB6F8943EBF51
:10D5C0000FBE2DBF8DB79EB701967C0100E09E0176
:10D5D0002B593F4FBC01CE0189599F4F0E94A2ACED
:10D5E0009E012B593F4F44E050E060EB7BE0CE01C1
:10D5F00089599F4F0E94A2ACE1968FACE197912C84
:10D6000093E0890E911C880C991C880C991CEDB72D
:10D61000FEB7E819F9090FB6F894FEBF0FBEEDBFCB
:10D620002DB73EB72F5F3F4F69018DB79EB7881961
:10D6300099090FB6F8949EBF0FBE8DBFEDB7FEB728
:10D6400031965F019E012B593F4FA401B601CE01D7
:10D6500089599F4F0E94A2AC9E012B593F4FA401B4
:10D66000B501CE0189599F4F0E94A2AC1091C40B05
:10D67000112309F4A7C000E09E012B593F4F44E05D
:10D6800050E068E97BE0CE0189599F4F0E94A2AC2F
:10D690009E012B593F4F44E050E06CE97BE0CE0106
:10D6A00089599F4F0E94A2AC9E012B593F4F44E0E5
:10D6B00050E064E97BE0CE0189599F4F0E94A2AC03
:10D6C0009E012B593F4F44E050E068EB7BE0CE01D8
:10D6D00089599F4F0E94A2AC9E012B593F4F44E0B5
:10D6E00050E064EB7BE0CE0189599F4F0E94A2ACD1
:10D6F0009E012B593F4F40E150E060E87BE0CE01B6
:10D7000089599F4F0E94A2AC9E012B593F4F44E084
:10D7100050E0BE01695A7F4FCE0189599F4F0E9448
:10D72000A2AC9E012B593F4F4CE050E065ED7BE0F1
:10D73000CE0189599F4F0E94A2AC9E012B593F4FA9
:10D7400044E050E063E276E1CE0189599F4F0E94A8
:10D75000A2AC9E012B593F4F44E050E0BE01695AF4
:10D760007F4FCE0189599F4F0E94A2AC01E09E01DC
:10D770002B593F4F41E050E0BE0161597F4FCE0130
:10D7800089599F4F0E94A2AC9E012B593F4F41E007
:10D7900050E0BE0162597F4FCE0189599F4F0E94D0
:10D7A000A2AC11118AC06B968CAD9DADAEADBFAD74
:10D7B0006B9780932B1690932C16A0932D16B093F5
:10D7C0002E167BC0E1968FADE19790E0029620EA9D
:10D7D0003BE0E4963FAF2EAFE497B501DE01119632
:10D7E000E5E18E2EE7E19E2EAE014F5E5F4FF5EF35
:10D7F000AF2EF6E1BF2EE896FFAEEEAEE8977E01C3
:10D8000031E2E30EF11C20E030E0821793072CF0A8
:10D81000E896EEADFFADE89701C0F701408051807A
:10D8200062807380F50141925192619271925F0121
:10D830008217930714F0F60101C0FA01408051806D
:10D8400062807380F40141925192619271924F0112
:10D850008217930734F0FB0140805180628073800F
:10D8600005C04D905D906D907C901397E496EEAD61
:10D87000FFADE4974192519261927192E496FFAFAD
:10D88000EEAFE4972F5F3F4F6C5F7F4F1496F4E04D
:10D89000CF0ED11C4C5F5F4FE896EEADFFADE89721
:10D8A0003496E896FFAFEEAFE897F4E0EF0EF11C88
:10D8B0002430310509F0A9CFDECEE0968FADE09798
:10D8C000853099F4AF968FADAF97853071F400E055
:10D8D0009E012B593F4F44E650E06FE276E1CE01C6
:10D8E00089599F4F0E94A2AC24C0111102C00E940E
:10D8F000D5ABE0968FADE097AF96CFACAF978C9D50
:10D9000060011124E12CF12CEC14FD0491F000E0F5
:10D910009E012B593F4F44E050E0BE01695A7F4FB2
:10D92000CE0189599F4F0E94A2AC2FEFE21AF20A52
:10D93000EBCF00E09E012B593F4F44E050E0BE0189
:10D940006D5A7F4FCE0189599F4F0E94A2AC1AE0B9
:10D95000115079F000E09E012B593F4F44E050E018
:10D96000BE01695A7F4FCE0189599F4F0E94A2ACD8
:10D97000EFCF01E09E012B593F4F41E050E0BE0147
:10D9800063597F4FCE0189599F4F0E94A2AC9E01DF
:10D990002B593F4F41E050E0BE0164597F4FCE010B
:10D9A00089599F4F0E94A2AC00E09E012B593F4F26
:10D9B00044E050E0BE01635C7F4FCE0189599F4F28
:10D9C0000E94A2AC9E012B593F4F44E050E0BE01A3
:10D9D0006F5C7F4FCE0189599F4F0E94A2ACAE96DB
:10D9E0008FADAE97AD96CFACAD978C9D60011124F5
:10D9F000E12CF12C00E09E012B593F4FCE14DF04A7
:10DA000071F044E050E0BE01695A7F4FCE01895960
:10DA10009F4F0E94A2AC3FEFE31AF30AEBCF41E025
:10DA200050E0BE016F587F4FCE0189599F4F0E9431
:10DA3000A2AC9E012B593F4F41E050E0BE01655919
:10DA40007F4FCE0189599F4F0E94A2AC9E012B5956
:10DA50003F4F44E050E0BE01695A7F4FCE018959E3
:10DA60009F4F0E94A2AC9E012B593F4F44E050E0D3
:10DA7000BE01695A7F4FCE0189599F4F0E94A2ACC7
:10DA80009E012B593F4F44E050E067E276E1CE0122
:10DA900089599F4F0E94A2AC9E012B593F4F44E0F1
:10DAA00050E0BE01615B7F4FCE0189599F4F0E94BC
:10DAB000A2AC9E012B593F4F44E050E0BE01655B94
:10DAC0007F4FCE0189599F4F0E94A2AC9E012B59D6
:10DAD0003F4F44E050E0BE01695B7F4FCE01895962
:10DAE0009F4F0E94A2AC10E000E09E012B593F4FD7
:10DAF00044E050E0BE01695A7F4FCE0189599F4FE3
:10DB00000E94A2AC111110C06B96CCACDDACEEAC97
:10DB1000FFAC6B9720E030E84BE355E4C701B6015A
:10DB20000E9488C8811103C054E0F52E33C0809153
:10DB3000C40B811108C0C092B615D092B715E092FF
:10DB4000B815F092B91500E09E012B593F4F44E003
:10DB500050E062EB75E1CE0189599F4F0E94A2AC63
:10DB60009E012B593F4F44E050E06AEB75E1CE0136
:10DB700089599F4F0E94A2AC9E012B593F4F44E010
:10DB800050E0BE01695A7F4FCE0189599F4F0E94D4
:10DB9000A2AC12C0FA94FF2079F000E09E012B594C
:10DBA0003F4F44E050E0BE01695A7F4FCE01895992
:10DBB0009F4F0E94A2ACEECF1F5F153009F094CFAB
:10DBC00000E09E012B593F4F42E050E0BE016D59ED
:10DBD0007F4FCE0189599F4F0E94A2AC9E012B59C5
:10DBE0003F4F44E050E0BE01695A7F4FCE01895952
:10DBF0009F4F0E94A2AC6B96CCACDDACEEACFFAC00
:10DC00006B9720E030E84BE355E4C701B6010E9472
:10DC100088C8882329F18091C40B811108C0C09263
:10DC2000AE15D092AF15E092B015F092B11500E0AC
:10DC30009E012B593F4F44E050E06AEA75E1CE0166
:10DC400089599F4F0E94A2AC9E012B593F4F44E03F
:10DC500050E066EA75E1CE0189599F4F0E94A2AC5F
:10DC600000E09E012B593F4F42E050E0BE016F594A
:10DC70007F4FCE0189599F4F0E94A2AC9E012B5924
:10DC80003F4F41E050E0BE016F587F4FCE018959B0
:10DC90009F4F0E94A2AC19E0115000E09E012B5949
:10DCA0003F4F112359F044E050E0BE01695A7F4FC5
:10DCB000CE0189599F4F0E94A2ACEECF41E050E0C7
:10DCC00063E976E1CE0189599F4F0E94A2ACF12C05
:10DCD00000E09E012B593F4F44E050E0BE01695ADD
:10DCE0007F4FCE0189599F4F0E94A2AC1091C40B67
:10DCF000111110C0F1100EC06B968CAD9DADAEAD84
:10DD0000BFAD6B978093981690939916A0939A162F
:10DD1000B0939B16F39485E0F812DACF111102C08C
:10DD20000E94DB454CE0F42EFA94F11003C03CE075
:10DD3000F32E0FC000E09E012B593F4F42E050E010
:10DD4000BE01615A7F4FCE0189599F4F0E94A2ACFC
:10DD5000EBCFFA9400E09E012B593F4FFF2059F082
:10DD600044E050E0BE016D5B7F4FCE0189599F4F6B
:10DD70000E94A2ACEECF46E050E0BE01635C7F4F54
:10DD8000CE0189599F4F0E94A2AC9E012B593F4F53
:10DD900044E050E060E97BE0CE0189599F4F0E944A
:10DDA000A2AC9E012B593F4F4CE050E0BE016F5C8E
:10DDB0007F4FCE0189599F4F0E94A2AC2CE1F22ED9
:10DDC000FA94F11003C094E0F92E1DC000E09E010A
:10DDD0002B593F4F44E050E0BE01695A7F4FCE01BE
:10DDE00089599F4F0E94A2ACEBCF00E09E012B59B6
:10DDF0003F4F44E050E0BE01695A7F4FCE01895940
:10DE00009F4F0E94A2ACFA94F110EFCF8BE0F82E56
:10DE1000FA94FF2079F000E09E012B593F4F44E037
:10DE200050E0BE01695A7F4FCE0189599F4F0E9431
:10DE3000A2ACEECFA9968EAD9FADA997845691095D
:10DE4000C7DA8093C30B882309F1EFEFFAE18491DD
:10DE50007F019FEFE91AF90A882321F00E94784098
:10DE6000F701F5CFA9966EAD7FADA99764567109FC
:10DE700087EE98E10E94E94E6BED72E08FED98E13C
:10DE80000E94E94E8AE00E94784099C0A7962EAD84
:10DE90003FADA797AB968EAD9FADAB9728173907CF
:10DEA00009F44BC081E08093C30BEAEEFAE1849160
:10DEB0007F012FEFE21AF20A811103C0EFEBF8E1C4
:10DEC00004C00E947840F701F2CF84917F013FEFB8
:10DED000E31AF30A882321F00E947840F701F5CF76
:10DEE000AB966EAD7FADAB9780E090E04AE00E94CC
:10DEF0009443EAEBF8E184917F019FEFE91AF90A74
:10DF0000882321F00E947840F701F5CFA7966EADE7
:10DF10007FADA79780E090E04AE00E949443EAEA50
:10DF2000F8E184917F012FEFE21AF20A882309F4C5
:10DF300046C00E947840F701F4CF111142C0EFEFC4
:10DF4000FAE184917F013FEFE31AF30A811103C0E4
:10DF500007ED12E004C00E947840F701F2CFF8010B
:10DF600081918F01882319F00E947840F8CFA996FB
:10DF70006EAD7FADA997645671098DE898E10E9456
:10DF8000E94EA7964EAD5FADA79760E070E080E8E0
:10DF900098E10E94AF4EEDE7F8E184917F012FEF09
:10DFA000E21AF20A811107C08091C30B811109C0E6
:10DFB0000E9461AD06C00E947840F701EECF1123A8
:10DFC00099F3E6968EAD9FADE6970FB6F8949EBF97
:10DFD0000FBE8DBF8091C40B811102C00E9471A041
:10DFE0009091C30B81E089270FB6F8943EBE0FBE17
:10DFF0002DBEC958DF4F0FB6F894DEBF0FBECDBFA0
:10E00000DF91CF911F910F91FF90EF90DF90CF9014
:10E01000BF90AF909F908F907F906F905F904F9048
:10E020003F902F90089581E08093C40BF2D9109215
:10E03000C40B8111EEC90E9405A581E008958F925D
:10E040009F92AF92BF92CF92DF92EF92FF920F9387
:10E050001F93CF93DF93CDB7DEB7CA5AD1090FB65E
:10E06000F894DEBF0FBECDBFE9961CAE1DAE1EAE4E
:10E070001FAEE9978091F7039091F803A091F903FF
:10E08000B091FA03ED968CAF9DAFAEAFBFAFED97F9
:10E09000C556DF4F19821882CB59D04084E690E0F4
:10E0A000C356DF4F99838883CD59D0401092C30B5C
:10E0B0009E0125563F4F44E050E0BE0167587F4F18
:10E0C000CE0183569F4F0E94EEACC356DF4F88812E
:10E0D0009981CD59D0400296C356DF4F99838883EA
:10E0E000CD59D040C556DF4F19821882CB59D04048
:10E0F00081E0CD55DF4F8883C35AD0409E0125561D
:10E100003F4F41E050E0BE016D557F4FCE01835639
:10E110009F4F0E94EEAC9E0125563F4F40E150E0DC
:10E1200065EF76E1CE0183569F4F0E94EEAC9E01D3
:10E1300025563F4F44E050E060EB7BE0CE01835634
:10E140009F4F0E94EEAC9E0125563F4F40E150E0AC
:10E1500065E177E1CE0183569F4F0E94EEAC9E01B0
:10E1600025563F4F40E150E060EA7BE0CE01835608
:10E170009F4F0E94EEAC9E0125563F4F44E050E079
:10E1800068E97BE0CE0183569F4F0E94EEAC9E0172
:10E1900025563F4F44E050E06CE97BE0CE018356CA
:10E1A0009F4F0E94EEAC9E0125563F4F44E050E049
:10E1B00064E97BE0CE0183569F4F0E94EEAC9E0146
:10E1C00025563F4F44E050E068EB7BE0CE0183569C
:10E1D0009F4F0E94EEAC9E0125563F4F44E050E019
:10E1E00064EB7BE0CE0183569F4F0E94EEAC9E0114
:10E1F00025563F4F40E150E060E87BE0CE0183567A
:10E200009F4F0E94EEAC8AE097EDA3EABCE3E9964B
:10E210008CAF9DAFAEAFBFAFE9979E0125563F4F84
:10E2200044E050E0BE016B587F4FCE0183569F4FB4
:10E230000E94EEAC9E0125563F4F4CE050E065ED4C
:10E240007BE0CE0183569F4F0E94EEAC8091A816D2
:10E250009091A916A091AA16B091AB16C358DF4FA2
:10E2600088839983AA83BB83CD57D0409E012556CE
:10E270003F4F44E050E0BE0163587F4FCE018356CC
:10E280009F4F0E94EEAC85E0CC55DF4F8883C45A87
:10E29000D040CB55DF4F8883C55AD0409E012556CC
:10E2A0003F4F44E050E06BE276E1CE0183569F4F52
:10E2B0000E94EEAC9E0125563F4F41E050E0BE016A
:10E2C0006C557F4FCE0183569F4F0E94EEAC9E014E
:10E2D00025563F4F41E050E0BE016B557F4FCE01C8
:10E2E00083569F4F0E94EEAC9E0125563F4F44E659
:10E2F00050E06FE276E1CE0183569F4F0E94EEAC74
:10E30000CF57DF4F188219821A821B82C158D04022
:10E310009E0125563F4F44E050E0BE016F577F4FAE
:10E32000CE0183569F4F0E94EEACE9961CAE1DAE07
:10E330001EAE1FAEE9971AE0115071F09E012556EE
:10E340003F4F44E050E0BE016B587F4FCE018356F3
:10E350009F4F0E94EEACF0CF83E0CA55DF4F888319
:10E36000C65AD040C955DF4F8883C75AD040CB57D3
:10E37000DF4F188219821A821B82C558D040C757B6
:10E38000DF4F188219821A821B82C958D040E99641
:10E390001CAE1DAE1EAE1FAEE9979E0125563F4F27
:10E3A00041E050E0BE016A557F4FCE0183569F4F3A
:10E3B0000E94EEAC9E0125563F4F41E050E0BE0169
:10E3C00069557F4FCE0183569F4F0E94EEAC9E0150
:10E3D00025563F4F44E050E0BE0167577F4FCE01C6
:10E3E00083569F4F0E94EEAC9E0125563F4F44E05E
:10E3F00050E0BE016B577F4FCE0183569F4F0E9466
:10E40000EEAC0AE010E00150110971F09E012556B2
:10E410003F4F44E050E0BE016B587F4FCE01835622
:10E420009F4F0E94EEACEFCFC855DF4F1882C85AFD
:10E43000D0408FEFC755DF4F8883C95AD0409E0127
:10E4400025563F4F41E050E0BE0168557F4FCE0159
:10E4500083569F4F0E94EEAC9E0125563F4F41E0F0
:10E4600050E0BE0167557F4FCE0183569F4F0E94FB
:10E47000EEACE9961CAE1DAE1EAE1FAEE9979E0136
:10E4800025563F4F44E050E0BE016B587F4FCE0110
:10E4900083569F4F0E94EEAC9E0125563F4F44E0AD
:10E4A00050E0BE016B587F4FCE0183569F4F0E94B4
:10E4B000EEAC9E0125563F4F44E050E067E276E126
:10E4C000CE0183569F4F0E94EEAC809183029091C3
:10E4D0008402A0918502B0918602C357DF4F8883E2
:10E4E0009983AA83BB83CD58D040809187029091B5
:10E4F0008802A0918902B0918A02CF56DF4F8883AB
:10E500009983AA83BB83C159D040CB56DF4F198270
:10E510001882C559D040C956DF4F19821882C75991
:10E52000D0409E0125563F4F44E050E0BE01635766
:10E530007F4FCE0183569F4F0E94EEAC9E01255621
:10E540003F4F44E050E0BE016F567F4FCE018356EF
:10E550009F4F0E94EEAC9E0125563F4F44E050E095
:10E56000BE016B567F4FCE0183569F4F0E94EEAC8B
:10E5700010E0C12C80E8D82E8BE3E82E85E4F82E3D
:10E58000812C912C90E8A92E9FE3B92E111138C04F
:10E590009E0125563F4F44E050E066EB75E1CE0109
:10E5A00083569F4F0E94EEAC9E0125563F4F44E09C
:10E5B00050E062EB75E1CE0183569F4F0E94EEACB6
:10E5C0009E0125563F4F44E050E06AEB75E1CE01D5
:10E5D00083569F4F0E94EEACE9968CAE9DAEAEAED8
:10E5E000BFAEE9979E0125563F4F44E050E0BE0183
:10E5F0006B587F4FCE0183569F4F0E94EEAC2AC0CE
:10E60000E996CCAEDDAEEEAEFFAEE9979E012556A3
:10E610003F4F44E050E0BE016B587F4FCE01835620
:10E620009F4F0E94EEACE9961CAE1DAE1EAE1FAE13
:10E63000E99704E0015071F09E0125563F4F44E0F8
:10E6400050E0BE016B587F4FCE0183569F4F0E9412
:10E65000EEACF0CF1F5F153009F098CF84E190E069
:10E66000C156DF4F99838883CF59D0409E012556EC
:10E670003F4F42E050E0BE0161567F4FCE018356CE
:10E680009F4F0E94EEAC9E0125563F4F44E050E064
:10E690006EEA75E1CE0183569F4F0E94EEAC9E015B
:10E6A00025563F4F44E050E06AEA75E1CE018356BB
:10E6B0009F4F0E94EEAC9E0125563F4F44E050E034
:10E6C00066EA75E1CE0183569F4F0E94EEAC80E270
:10E6D00090E0CF55DF4F99838883C15AD0409E0187
:10E6E00025563F4F42E050E0BE016F557F4FCE01AF
:10E6F00083569F4F0E94EEACC655DF4F1882CA5A10
:10E70000D04080E2EBE8F2E0DE019D9601900D92B0
:10E710008A95E1F79E0125563F4F41E050E0BE014A
:10E7200066557F4FCE0183569F4F0E94EEAC9E01EF
:10E7300025563F4F40E250E0BE01635D7F4FCE0162
:10E7400083569F4F0E94EEAC9E0125563F4F41E0FD
:10E7500050E063E976E1CE0183569F4F0E94EEAC14
:10E7600010E011110EC08091981690919916A09109
:10E770009A16B0919B16E9968CAF9DAFAEAFBFAF26
:10E78000E9979E0125563F4F44E050E0BE016B588B
:10E790007F4FCE0183569F4F0E94EEAC1F5F153016
:10E7A00001F7BE01635B7F4F86E1FB0111928A9501
:10E7B000E9F79E0125563F4F46E150E0CE018356D2
:10E7C0009F4F0E94EEAC8CE2EBEAF2E0DE01119684
:10E7D00001900D928A95E1F79E0125563F4F4CE23C
:10E7E00050E0BE016F5F7F4FCE0183569F4F0E9466
:10E7F000EEACBE0161597F4F86E0FB0111928A9514
:10E80000E9F79E0125563F4F46E050E0CE01835682
:10E810009F4F0E94EEAC9E0125563F4F44E050E0D2
:10E8200060E97BE0CE0183569F4F0E94EEACBE01B3
:10E830006D597F4F8CE0FB0111928A95E9F79E019B
:10E8400025563F4F4CE050E0CE0183569F4F0E942B
:10E85000EEACE9961CAE1DAE1EAE1FAEE9971CE1F4
:10E86000115071F09E0125563F4F44E050E0BE012B
:10E870006B587F4FCE0183569F4F0E94EEACF0CF76
:10E88000E9961CAE1DAE1EAE1FAEE99714E0115006
:10E8900071F09E0125563F4F44E050E0BE016B5899
:10E8A0007F4FCE0183569F4F0E94EEACF0CFE9968A
:10E8B0001CAE1DAE1EAE1FAEE9971BE0115071F0ED
:10E8C0009E0125563F4F44E050E0BE016B587F4FFC
:10E8D000CE0183569F4F0E94EEACF0CF8091C30BC8
:10E8E000811167C0C356DF4FE880F980CD59D04011
:10E8F000F4E6EF1AF108C556DF4F88819981CB59AC
:10E90000D040C756DF4F99838883C959D04084E6E9
:10E9100090E0C356DF4F99838883CD59D0409E0144
:10E9200025563F4F44E050E067ED72E0CE0183563C
:10E930009F4F0E94EEAC9E0125563F4F42E050E0B3
:10E94000BE0167567F4FCE0183569F4F0E94EEACAB
:10E95000EFEFFAE184918F010F5F1F4F882321F0C1
:10E960000E947840F801F6CFB7018BE698E10E944B
:10E97000E94EC756DF4F48815981C959D04060E000
:10E9800070E08EE598E10E94AF4EEBE5F8E18491EE
:10E990008F010F5F1F4F882321F00E947840F801FC
:10E9A000F6CFC7010E94E8699091C30B892B809331
:10E9B000C30B9091C30B81E08927C655DF4F0FB67B
:10E9C000F894DEBF0FBECDBFDF91CF911F910F91A5
:10E9D000FF90EF90DF90CF90BF90AF909F908F907F
:10E9E0000895CF92DF92EF92FF920F931F93CF93F0
:10E9F000DF936C017A018B01C0E0D0E0CE15DF051A
:10EA000081F0D8016D918D01D601ED91FC910190BD
:10EA1000F081E02DC6011995892B11F02196EECFDA
:10EA20007E01C701DF91CF911F910F91FF90EF9071
:10EA3000DF90CF9008950E94DECF1F920F920FB605
:10EA40000F9211240BB60F922F933F934F935F9326
:10EA50006F937F938F939F93AF93BF93EF93FF93A6
:10EA60008091C80B9091C90BA091CA0BB091CB0BB0
:10EA7000892B8A2B8B2B59F19091C70BE091C50BF9
:10EA8000F091C60B8081892780838091C80B90917B
:10EA9000C90BA091CA0BB091CB0B181619061A0618
:10EAA0001B060CF056C08091C80B9091C90BA09129
:10EAB000CA0BB091CB0B0197A109B1098093C80B88
:10EAC0009093C90BA093CA0BB093CB0B42C080911B
:10EAD0003902EFE1F9E1E4919FEF90933902E230DE
:10EAE000C9F050F4EE2399F0E13081F590916F0078
:10EAF0009D7F90936F002AC0E43019F1E0F0E5307B
:10EB000029F5909173009D7F909373001FC0109220
:10EB10006E001CC0909170009D7F9093700091E0FA
:10EB20009093B0009091B100987F94609093B10061
:10EB30001092B3000BC0909171009D7F9093710073
:10EB400005C0909172009D7F9093720060E00E94DA
:10EB5000ADB4FF91EF91BF91AF919F918F917F9154
:10EB60006F915F914F913F912F910F900BBE0F903E
:10EB70000FBE0F901F90189590934204809341040C
:10EB800080E00C94E27D8F929F92AF92BF92CF92E1
:10EB9000DF92EF92FF921F93CF93DF93C82F87E905
:10EBA00091E19093730F8093720F1092B31182E0F2
:10EBB00090E0A0E0B0E080939C1190939D11A09311
:10EBC0009E11B0939F111092710F10926D0F1092C1
:10EBD0006E0F10926F0F1092700F8FEF9FEFDC018E
:10EBE0008093690F90936A0FA0936B0FB0936C0F93
:10EBF000CC2379F1C53008F0F8C040E060E070E067
:10EC0000CB010E9448AE882309F4EFC020E1C29FE7
:10EC1000C0011124875A924FFC01E254FE4F20811B
:10EC20002F7709F0E2C03C96408151816281738167
:10EC3000443651056105710508F4D7C03497C0808A
:10EC4000D180E280F380C114D104E104F10421F405
:10EC5000CCC0C12CD12C760140E0C701B6010E9486
:10EC600048AE182F882309F4C0C08091740D90918C
:10EC7000750D8115924009F0B8C0A091790DAA23B5
:10EC800009F4B3C06091770D7091780D611571052D
:10EC900009F4ABC02091760D222309F4A6C0A093FD
:10ECA000AE112093A01180E030E041E050E0C82F89
:10ECB000FA01082E02C0EE0FFF1F0A94E2F72E178A
:10ECC0003F0739F08F5FC83091F789E08093A91131
:10ECD0008CC08093A91120917F0D3091800D21155A
:10ECE000310519F040E050E008C020918D0D3091C1
:10ECF0008E0D40918F0D5091900D2093A111309366
:10ED0000A2114093A3115093A41146015701860EFE
:10ED1000971EA11CB11C8092AF119092B011A092CD
:10ED2000B111B092B211E0917A0DF0917B0DF09398
:10ED3000B511E093B411B0E00E9498CC860E971EF6
:10ED4000A81EB91E8092B6119092B711A092B81168
:10ED5000B092B91185E0EE0FFF1F8A95E1F7E150FF
:10ED6000FE4FEF2FFF27E6958E0E9F1EA11CB11CB4
:10ED70008092AA119092AB11A092AC11B092AD11F9
:10ED800020917C0D30917D0D2115310521F0A901D7
:10ED900060E070E008C04091890D50918A0D60914B
:10EDA0008B0D70918C0DD701C60188199909AA099C
:10EDB000BB09840F951FA61FB71F04C0B695A79562
:10EDC00097958795CA95D2F78093A5119093A61130
:10EDD000A093A711B093A811853F2FE09207A1053A
:10EDE000B10528F48CE08093B31110E01AC0853F80
:10EDF0009F4FA105B10510F480E111C08091950DE0
:10EE00009091960DA091970DB091980D8093B611A9
:10EE10009093B711A093B811B093B91180E2809389
:10EE2000B311812FDF91CF911F91FF90EF90DF9071
:10EE3000CF90BF90AF909F908F900895682F8EE5F0
:10EE400095E10C94FC3ACF92DF92EF92FF921F93E0
:10EE5000CF93DF931092F60F80912910882321F031
:10EE600086E290E10E94E99110929B111092981114
:10EE700085E3809397110E9416B6EB01A89561E097
:10EE8000809197110E94DBB487E991E10E944A9337
:10EE90002398229A219A209A289A85E080939911A2
:10EEA00082E58CBD1DBC1AE08FEF0E944F9311507C
:10EEB000D9F720E030E0A90160E087E991E10E9404
:10EEC0005493182F80939A11813049F00E9416B6FE
:10EED0006C1B7D0B613D774060F381E054C02AEAF2
:10EEE00031E040E050E068E087E991E10E9454930E
:10EEF00082FF03C010939B110EC014E00E947D4F4F
:10EF000080939A111150D1F78A3A11F082E03BC0F8
:10EF100082E080939B1180919B11823021F0C12C63
:10EF2000D12C760105C0C12CD12CE12C80E4F82E27
:10EF300020E030E0A90167E387E991E10E94549362
:10EF4000A701960169E287E991E10E9454938093B9
:10EF50009A11882349F00E9416B66C1B7D0B613D07
:10EF6000774030F38AE00FC080919B11823011F519
:10EF700020E030E0A9016AE387E991E10E9454931F
:10EF8000882351F088E08093981187E991E10E94ED
:10EF90004A93EFEFFAE119C00E947D4F807C803CDC
:10EFA00019F483E080939B110E947D4F0E947D4F56
:10EFB0000E947D4F87E991E10E944A931092991136
:10EFC00081E0E1DD811131C015C08491EF0121960E
:10EFD000882321F00E947840FE01F7CFE1EFFAE1AB
:10EFE0008491EF012196882309F456C00E9478404D
:10EFF000FE01F6CF80E0C7DD811117C0EAEEFAE12D
:10F000008491EF012196882321F00E947840FE012F
:10F01000F7CFE6EDFAE18491EF012196882309F418
:10F020003BC00E947840FE01F6CF6CE971E186E2B8
:10F0300090E10E949691811116C0EAEEFAE1849166
:10F04000EF012196882321F00E947840FE01F7CF3E
:10F05000E5ECFAE18491EF0121968823E9F00E9422
:10F060007840FE01F7CF81E08093F60FEFEFFAE1F1
:10F070008491EF012196882321F00E947840FE01BF
:10F08000F7CFE9EBFAE18491EF012196882321F093
:10F090000E947840FE01F7CF8BE1E6E2F0E1A5E4C3
:10F0A000B0E101900D928A95E1F780912410909142
:10F0B00025109093441080934310DF91CF911F91BE
:10F0C000FF90EF90DF90CF900895809103148230ED
:10F0D00041F484EA9AE19093680D8093670D0E9451
:10F0E000A4400E9416B6609307147093081480938E
:10F0F000091490930A148091F60F882319F081E087
:10F100008093F50F81E0809303140895CF93DF93EC
:10F110001092F50F83E0809303148091501488239C
:10F12000B1F0ECE9FAE18491EF01882341F0082E77
:10F13000000C990B83DE2196FE018491F6CF8DE0C1
:10F1400090E07CDE8AE090E0DF91CF9177CEE0EA3C
:10F15000FAE18491EF01882391F3082E000C990BBA
:10F160006DDE2196FE018491F6CF8F929F92AF9231
:10F17000BF92CF92DF92EF92FF920F931F93CF93A4
:10F18000DF9300D01F92CDB7DEB7FC0183818130C1
:10F1900079F5818181FF2CC081899289A389B48905
:10F1A000892B8A2B8B2B09F448C07F0140E050E06B
:10F1B000BA01CF010E94FF908823D1F0F701858822
:10F1C0009688A788B08CC18CD28C82E090E0A0E0B9
:10F1D000B0E0F60180839183A283B3839E012F5F09
:10F1E0003F4FB501A401C6010E9411AF811102C0B9
:10F1F00080E03CC000E010E09801B501A401C60128
:10F200000E9480AE8823A1F389809A80AB80BC8065
:10F21000F6018789803141F4F8EF8F16FFEF9F06E2
:10F22000A104B10460F4DACF88EF88168FEF980656
:10F23000A8068FE0B80618F4D1CF81E017C0F70117
:10F24000158A168A178A108E118A128A138A148ACE
:10F25000818180688183C7010E945FB0882341F269
:10F2600040E050E0BA01C7010E94FF900F900F905C
:10F270000F900F90DF91CF911F910F91FF90EF9022
:10F28000DF90CF90BF90AF909F908F900895109295
:10F29000F80F1092F50F8091C111882321F08EEBA9
:10F2A00091E10C94E99108952F923F924F925F92D1
:10F2B0006F927F928F929F92AF92BF92CF92DF9286
:10F2C000EF92FF920F931F93CF93DF93CDB7DEB7EB
:10F2D000C257D1090FB6F894DEBF0FBECDBF8C0167
:10F2E0003B014A014DB75EB7E1965FAF4EAFE19784
:10F2F000AD961FAEAD971B0154E0250E311C7E016B
:10F300008FE5E80EF11C95EE492E92E0592EE0E4CF
:10F31000F0E0EC0FFD1F3496E396FFAFEEAFE397FE
:10F32000F3018781823008F462C184859585A685C2
:10F33000B7858F719927AA27BB27892B8A2B8B2BFF
:10F3400009F055C11092061046E050E1BE016F5F12
:10F350007F4FC1010E94F7AF18160CF048C18C8591
:10F36000982F9871903129F42091731221502230F6
:10F3700078F42981222309F43AC1253E89F22E32FC
:10F3800079F2209106102E3259F28A7049F6B8C0EF
:10F390004DB75EB7AF965FAF4EAFAF97BE016F5F31
:10F3A0007F4FC7010E94F2AD0115110521F0F80150
:10F3B000808181119BC021E081E090E0F701019004
:10F3C0000020E9F73197EE19FF098E0F9F1F029673
:10F3D0004DB75EB7481B590B0FB6F8945EBF0FBE12
:10F3E0004DBF8DB79EB701965C01211102C0B801D7
:10F3F00002C06AE173E0C5010E9432D0B701C501C5
:10F400000E9413D06AE173E0C5010E9413D02596D3
:10F410001FAE259728961FAE289724961FAE1EAEC6
:10F42000249722965FAE4EAE229721E0A701B1014C
:10F43000E3968EAD9FADE3970E947C9781112AC021
:10F4400080917312811126C0EFEFFAE184916F0170
:10F450009FEFC91AD90A882321F00E947840F6014B
:10F46000F5CFE8E8FAE184916F012FEFC21AD20AD2
:10F47000882321F00E947840F601F5CF6701F6015C
:10F4800081916F01882319F00E947840F8CF8AE0BB
:10F490000E9478408BE1FE01EC5BFF4FDE01959608
:10F4A00001900D928A95E1F724968EAD9FAD249739
:10F4B0009CA38BA35AA249A240E050E0BE016F5D1D
:10F4C0007F4FC501F1DECE0181960E944F51CE01E2
:10F4D000805C9F4F0E944F51AF964EAD5FADAF978E
:10F4E0000FB6F8945EBF0FBE4DBF1ACFF801019062
:10F4F0000020E9F73197CF01801B910B20E05ECF10
:10F5000081E0903109F080E08093F70F903141F075
:10F510008985873409F004CF8A858E3709F400CFB6
:10F5200080917312813029F08230D9F18111F8CEA7
:10F530000AC0809174129091751201969093751281
:10F5400080937412EDCEBE016F5F7F4F89EF9FE015
:10F550000E94F2AD0115110529F489EFC82E8FE044
:10F56000D82E09C06801F60181916F018823A9F3A3
:10F570000E947840F8CFF60181916F01882319F03D
:10F580000E947840F8CF80E20E9478406D8D7E8D99
:10F590008F8D98A14AE00E9494438AE00E947840AF
:10F5A000BFCEBE016F5F7F4F89EF9FE00E94F2AD3B
:10F5B0008114910441F069EF7FE0C4010E9400D002
:10F5C000892B69F414C0AD96FFADAD978F2F90E0F5
:10F5D00020918015309181158217930741F0AD96E7
:10F5E0002FADAD972F5FAD962FAFAD9799CEE1962A
:10F5F0008EAD9FADE1970FB6F8949EBF0FBE8DBF45
:10F60000CE58DF4F0FB6F894DEBF0FBECDBFDF91EF
:10F61000CF911F910F91FF90EF90DF90CF90BF900F
:10F62000AF909F908F907F906F905F904F903F90A2
:10F630002F9008950F931F93CF93DF93CDB7DEB72D
:10F640006F970FB6F894DEBF0FBECDBF8B0122E0DF
:10F6500020937312909381158093801585E490E137
:10F660000E9446938BE1E5E4F0E1DE0115960190FE
:10F670000D928A95E1F780914310909144109C83FC
:10F680008B8385EE92E09A838983A801BE016F5F28
:10F690007F4F80E090E008DECE0101960E944F513E
:10F6A0006F960FB6F894DEBF0FBECDBFDF91CF913E
:10F6B0001F910F9108952F923F924F925F926F92F8
:10F6C0007F928F929F92AF92BF92CF92DF92EF92F2
:10F6D000FF920F931F93CF93DF93CDB7DEB76F9752
:10F6E0000FB6F894DEBF0FBECDBF6C012DB63EB68F
:10F6F0001D8218861C821B8285EE92E09A83898384
:10F70000FB0180819E012F5F3F4F39018F3241F015
:10F7100081E490E1F60191838083F62E172F64C077
:10F7200082E290E1F601918380838B010F5F1F4F8E
:10F730000115110509F456C04DB65EB66FE270E0D2
:10F74000C8010E941ED04C010817190708F048C0D4
:10F750007C01E01AF10AFF24C70101962DB73EB7DC
:10F76000281B390B0FB6F8943EBF0FBE2DBF8DB7C7
:10F770009EB701965C01A701B8010E9447D0F50130
:10F78000EE0DFF1D1082F60160817181611571051A
:10F7900011F06C5F7F4F21E0A501CE0105960E941C
:10F7A0007C97811111C0B50184E79AE10E94024F54
:10F7B0008EE20E9478408AE00E9478400FB6F8946A
:10F7C0005EBE0FBE4DBE0EC0F60171826082840126
:10F7D0000F5F1F4F0FB6F8945EBE0FBE4DBEA8CF91
:10F7E000F02E02C0F12C10E0C3010E944F518F2D6A
:10F7F000912F0FB6F8943EBE0FBE2DBE6F960FB67A
:10F80000F894DEBF0FBECDBFDF91CF911F910F9156
:10F81000FF90EF90DF90CF90BF90AF909F908F9030
:10F820007F906F905F904F903F902F900895FF9240
:10F830000F931F93CF93DF938C01EB01F42E80E2A3
:10F840000E9478408FEFF81611F084E501C082E441
:10F850000E9478408AE30E947840F80160817181BB
:10F860008281938142E00E941944488159816A81D2
:10F870007B8180EA9DE10E94CC4E62E070E080E0F6
:10F8800090E0DF91CF911F910F91FF900C94DEB526
:10F890008F929F92AF92BF92CF92DF92EF92FF92A0
:10F8A0000F931F93CF93DF93F0E2FF2EE12CAE2D49
:10F8B000B0E0BD016F0D711D759567956E1511F066
:10F8C000F6120BC0E3E8FBE165917491072E000C82
:10F8D000880B990B0E948EC862C09B012150310990
:10F8E000220F331F220F331FF901EB5FF44E0591F6
:10F8F0001491AB01440F551F440F551FFA01EB5FE4
:10F90000F44EC591D4918017910714F4F62ED1CFFF
:10F91000C817D90714F4E62ECACFF901E95FF44EEF
:10F92000E590F490FA01E95FF44EC590D490BC01E3
:10F93000601B710B072E000C880B990B0E948EC860
:10F940004B015C01B6016E197F09072E000C880B74
:10F95000990B0E948EC89B01AC01C501B4010E94A5
:10F96000EDC84B015C01C01BD10BBE01DD0F880B44
:10F97000990B0E948EC89B01AC01C501B4010E9485
:10F980008ECD4B015C01B701FF0C880B990B0E94D7
:10F990008EC89B01AC01C501B4010E94B2CCDF91BD
:10F9A000CF911F910F91FF90EF90DF90CF90BF907C
:10F9B000AF909F908F9008950F931F93CF93DF93F5
:10F9C000CDB7DEB728970FB6F894DEBF0FBECDBF18
:10F9D0006091410470914204072E000C880B990B32
:10F9E0000E948EC86D837E838F83988780914304A5
:10F9F00090914404A0914504B091460489839A8370
:10FA0000AB83BC834DEFBE016B5F7F4FCE01019690
:10FA10000EDF60913B0470913C04072E000C880BB4
:10FA2000990B0E948EC86D837E838F839887809107
:10FA30003D0490913E04A0913F04B091400489831D
:10FA40009A83AB83BC834FEFBE016B5F7F4FCE01C8
:10FA50000196EDDEE8EAFDE184918F010F5F1F4F13
:10FA6000882321F00E947840F801F6CFE091C81574
:10FA7000F0E0EA53FA4E608170E080E090E00E948E
:10FA8000FF43E3EAFDE184918F010F5F1F4F88235D
:10FA900021F00E947840F801F6CF6091C71570E020
:10FAA00080E090E00E94FF4328960FB6F894DEBFF6
:10FAB0000FBECDBFDF91CF911F910F9108950F938E
:10FAC0000FB70F9300916E000B7F00936E00789438
:10FAD0000F930BB70F930CB70F921F922F933F9377
:10FAE0004F935F936F937F938F939F93AF93BF9346
:10FAF000EF93FF931124DAD2FF91EF91BF91AF9171
:10FB00009F918F917F916F915F914F913F912F9135
:10FB10001F900F900CBF0F910BBF0F910460F894D2
:10FB200000936E000F910FBF0F911895CF92DF9247
:10FB3000EF92FF92C0903D04D0903E04E0903F04CD
:10FB4000F090400460913B0470913C046650710950
:10FB5000072E000C880B990B0E948EC89B01AC01EC
:10FB6000C701B6010E9488C887FF1FC020E030E0AF
:10FB700040E050E4C701B6010E94B2CC0E94FBCD28
:10FB8000709300166093FF150E9416B6DC01CB013E
:10FB9000805A9541AF4FBF4F8093FB159093FC1552
:10FBA000A093FD15B093FE1508C01092FB1510929E
:10FBB000FC151092FD151092FE15FF90EF90DF904E
:10FBC000CF900895CF92DF92EF92FF92C0904304BE
:10FBD000D0904404E0904504F090460460914104C4
:10FBE0007091420469507109072E000C880B990B23
:10FBF0000E948EC89B01AC01C701B6010E9488C853
:10FC000087FF1FC020E030E040EA50E4C701B601A2
:10FC10000E94B2CC0E94FBCD7093FA156093F91547
:10FC20000E9416B6DC01CB0188549747AF4FBF4FF7
:10FC30008093F5159093F615A093F715B093F815EA
:10FC400008C01092F5151092F6151092F715109243
:10FC5000F815FF90EF90DF90CF9008958F929F92CC
:10FC6000AF92BF92CF92DF92EF92FF920F931F93CA
:10FC7000CF93DF93F0E4FF2EE12CAE2DB0E0BD0179
:10FC80006F0D711D759567956E1511F0F6120BC00D
:10FC9000E5EFFCE165917491072E000C880B990B40
:10FCA0000E948EC862C09B0121503109220F331F70
:10FCB000220F331FF901E950F44E05911491AB0165
:10FCC000440F551F440F551FFA01E950F44EC591DA
:10FCD000D4918017910714F4F62ED1CFC817D90705
:10FCE00014F4E62ECACFF901E750F44EE590F490F3
:10FCF000FA01E750F44EC590D490BC01601B710B23
:10FD0000072E000C880B990B0E948EC84B015C01DA
:10FD1000B6016E197F09072E000C880B990B0E9403
:10FD20008EC89B01AC01C501B4010E94EDC84B0116
:10FD30005C01C01BD10BBE01DD0F880B990B0E942B
:10FD40008EC89B01AC01C501B4010E948ECD4B0150
:10FD50005C01B701FF0C880B990B0E948EC89B01B8
:10FD6000AC01C501B4010E94B2CCDF91CF911F91CB
:10FD70000F91FF90EF90DF90CF90BF90AF909F904A
:10FD80008F90089560E080910B1690910C1680DDA5
:10FD90006093430470934404809345049093460415
:10FDA0008091091690910A1659DF60933D04709373
:10FDB0003E0480933F0490934004A8951092C3158D
:10FDC00008957F928F929F92AF92BF92CF92DF92CF
:10FDD000EF92FF920F931F93CF93DF9320E030E0D9
:10FDE00048E452E4609143047091440480914504D6
:10FDF000909146040E94D8CE18164CF4EBE8FBE133
:10FE0000E491C1E001C0CC0FEA95EAF701C0C0E07F
:10FE100085E8E82E8BE1F82E0BE81BE196E0A92E91
:10FE2000912CD0E0CC24C394D12CF7017490F8012C
:10FE3000849077FC23C0892D90E0082C02C0959512
:10FE400087950A94E2F780FD19C0BE01082C02C014
:10FE5000759567950A94E2F76170B62EB1946B2D93
:10FE6000872D0E94ADB46B2D70E0872D0E9417B5D1
:10FE7000C60101C0880F8A94EAF7982AAA94FFEF76
:10FE8000EF1AFF0A0F5F1F4FA110CFCFDF91CF9165
:10FE90001F910F91FF90EF90DF90CF90BF90AF90A8
:10FEA0009F908F907F9008950F931F938091A51539
:10FEB000813019F40E9416B608C06091A1157091A6
:10FEC000A2158091A3159091A4150091CD151091C4
:10FED000CE152091CF153091D015601B710B820B80
:10FEE000930B28EE33E040E050E00E9476CC809106
:10FEF000C9159091CA15A091CB15B091CC15BC0134
:10FF0000CD01620F731F841F951F1F910F910895DC
:10FF10001092A5151092CD151092CE151092CF15F6
:10FF20001092D0151092A1151092A2151092A3153F
:10FF30001092A4151092C9151092CA151092CB15E3
:10FF40001092CC1508958091A5158130E1F0823092
:10FF500051F4AADF6093C9157093CA158093CB152D
:10FF60009093CC1501C0D4DF81E08093A5150E9449
:10FF700016B66093CD157093CE158093CF159093E0
:10FF8000D01581E0089580E008958091A5158150F5
:10FF9000823010F080E008951092A5150E9416B6E8
:10FFA0006093A1157093A2158093A3159093A41547
:10FFB00081E008951092C21580E090E00E94BC7527
:10FFC00010923C0410923B04B1DDDFDF80E090E052
:10FFD0000E94BC751092C6152C9810923C04109289
:10FFE0003B041092C715809102018072809300013A
:10FFF0000895DF92EF92FF920F931F93CF93DF93B9
:020000021000EC
:10000000F82ED62EE72E8A0180914102882309F42A
:1000100039C0EAEEFAE18491EF012196882321F0BC
:100020000E947840FE01F7CFED2DFE2D8491EF0167
:100030002196882321F00E947840FE01F7CFE6E95F
:10004000FBE18491EF012196882321F00E94784002
:10005000FE01F7CFF7FC0BC06F2DFF0C770B880B61
:10006000990B0E94FF438AE00E9478400BC0E1E9AF
:10007000FBE18491EF012196882321F00E947840D2
:10008000FE01F7CF8091D115811108C01092410275
:1000900081E08093D115C8010E947251DF91CF9108
:1000A0001F910F91FF90EF90DF9084CFEF92FF921E
:1000B0000F931F93CF93DF93809144028F37A0F06B
:1000C0008F579091C61590931C16992311F02C9A76
:1000D00001C02C982091C71520931B169091020106
:1000E000222369F090950BC090911C16891708F097
:1000F0002C9890911B16891728F09091020190720C
:10010000909300018F5F8093440290911A1681E0D2
:10011000892780931A168091430285301CF4C1E030
:10012000C80F01C0C0E0823009F4B4C054F4882381
:1001300001F1813009F0E3C088E080937B0085E421
:10014000C0C0843009F4C5C00CF4B7C0853009F0D4
:10015000D6C090911916911102C080931916809102
:100160001916815080931916882309F4C8C0C5E078
:10017000C6C0809142028F5F80311CF4809342029E
:10018000BEC0109242028091C315811113C08091AC
:100190000F169091101690930C1680930B16809169
:1001A0000D1690910E1690930A168093091681E011
:1001B0008093C3158AE0EFE0F6E1DF011D928A9596
:1001C000E9F710920E1610920D1600910B16109171
:1001D0000C161195019511098091410490914204EA
:1001E000D1E0181619062CF08091C615811101C0B6
:1001F000D0E08091CF0B9091D00B91958195910992
:100200008017910734F44EE25DE16FE47DE180E018
:10021000F0DE80913C0290913D029195819591098B
:100220000817190744F4DD2331F041E65DE162E887
:100230007DE180E0DEDE80913B0490913C0411E0A2
:10024000181619062CF08091C715811101C010E015
:10025000E0900916F0900A168091CD0B9091CE0B8C
:100260008E159F0534F04EE35DE16FE47DE18FEF85
:10027000C0DE80913A0290913B02E816F9060CF438
:100280003EC01123E1F141E75DE162E87DE18FEFDE
:10029000B0DE35C080917A0086FD2EC08091780056
:1002A0009091790020910F1630911016820F931FB4
:1002B0009093101680930F1622C088E080937B00E5
:1002C00086E480937C0080917A00806480937A0039
:1002D00016C080917A0086FD11C0809178009091BF
:1002E000790020910D1630910E16820F931F909376
:1002F0000E1680930D1603C0C2E001C0C4E0C09387
:1003000043028091D40B81110E94E5AB8091C4150A
:100310009091C5150097A9F001979093C51580930A
:10032000C415892B71F484E99DE19093680D809345
:10033000670DDF91CF911F910F91FF90EF900C947B
:10034000A440DF91CF911F910F91FF90EF900895FE
:100350002F923F924F925F926F927F928F929F92D5
:10036000AF92BF92CF92DF92EF92FF920F931F93C3
:10037000CF93DF9300D01F92CDB7DEB75C017A83B5
:1003800069834A01170107FD07C0802F002E000C6A
:10039000990B9C838B8304C0E1E0F0E0FC83EB834A
:1003A000F90140805180628073808B819C81880F2D
:1003B000991F880F991F9C838B838F5F994E7C01B7
:1003C000A3019201FC0160817181828193810E946D
:1003D00088C8882391F0F70140825182628273823B
:1003E00011E020E030E0A901C301B2010E94D8CEA3
:1003F00018160CF010E0F5011083F50180818230B1
:10040000D1F0833009F45EC0813009F07CC0EB810B
:10041000FC81EF5FF94E2081318142815381F401EB
:1004200060817181828193810E9488C887FD6BC041
:1004300082E0F50180838B819C818F5F994E9C8344
:100440008B83B60180E090E00E948CC89B01AC01D8
:10045000EB81FC8160817181828193810E94B1CCAA
:100460009B01AC01F40160817181828193810E94C2
:10047000D8CE87FD14C00E9416B66B017C01910195
:10048000A8EEB3E00E94A2CCC60ED71EE81EF91E4D
:10049000E981FA81C082D182E282F38234C00E9473
:1004A00016B6E981FA81C080D180E280F380DC0158
:1004B000CB018C199D09AE09BF09B7FD24C083E0AB
:1004C000F50180830F3F19F047EF5CE102C04AE07D
:1004D0005DE16EE17DE1802F0F900F900F900F9006
:1004E000DF91CF911F910F91FF90EF90DF90CF9010
:1004F000BF90AF909F908F907F906F905F904F9044
:100500003F902F9076CD0F900F900F900F90DF912E
:10051000CF911F910F91FF90EF90DF90CF90BF9000
:10052000AF909F908F907F906F905F904F903F9093
:100530002F9008954F925F926F927F928F929F9229
:10054000AF92BF92CF92DF92EF92FF920F931F93E1
:10055000CF93DF93CDB7DEB760970FB6F894DEBFC9
:100560000FBECDBF8091C315811117C060960FB625
:10057000F894DEBF0FBECDBFDF91CF911F910F91D9
:10058000FF90EF90DF90CF90BF90AF909F908F90B3
:100590007F906F905F904F900895F4DB0E9416B6A5
:1005A0004B015C016091410470914204072E000CE4
:1005B000880B990B0E948EC869837A838B839C83F6
:1005C00044E1C42ED12C5CE3E52EF12C00E09E0129
:1005D0002F5F3F4F43E454E061EF75E180EF95E119
:1005E000B7DEC0904304D0904404E0904504F090FE
:1005F00046046091D10B7091D20B072E000C880B32
:10060000990B0E948EC89B01AC01C701B6010E94E4
:10061000D8CE18160CF009C160913E0270913F02CD
:10062000072E000C880B990B0E948EC89B01AC0111
:10063000C701B6010E9488C887FFF7C00091410436
:1006400010914204B801012E000C880B990B0E94F6
:100650008EC8A70196010E94B1CC2B013C0120ED70
:100660003CEC4CE45DE36091BA157091BB15809150
:10067000BC159091BD150E94EDC86D837E838F835C
:1006800098872091E7153091E8154091E915509130
:10069000EA15C701B6010E94B1CC9B01AC016D8186
:1006A0007E818F8198850E94EDC86D837E838F83C4
:1006B000988723E333E343E75FE36091E3157091A9
:1006C000E4158091E5159091E6150E94EDC89B0117
:1006D000AC016D817E818F8198850E94B2CC6D8343
:1006E0007E838F8398876093E3157093E4158093DE
:1006F000E5159093E615C092E715D092E815E092C3
:10070000E915F092EA1520E030E040E251E4C3013F
:10071000B2010E94D8CE18160CF431C220E030E0AD
:1007200040E251ECC301B2010E9488C887FD2FC28C
:10073000012B09F42CC28091E21581112CC2209169
:10074000DE153091DF154091E0155091E1152987B4
:100750003A874B875C872091B6153091B715409149
:10076000B8155091B915C301B2010E94EDC86B01D3
:100770007C01A301920169857A858B859C850E9405
:10078000B2CC69877A878B879C876093DE157093DC
:10079000DF158093E0159093E1152091B21530910B
:1007A000B3154091B4155091B5150E94EDC8A7013D
:1007B00096010E94B2CC2D813E814F8158850E94C6
:1007C000B1CC6B017C0120E030E04FE753E40E94A4
:1007D000D8CE20E030E0A90118160CF4E3C1C7011F
:1007E000B6010E9488C887FD07C0C701B6010E94F4
:1007F000F6CD759567951AC020E030E0A901C301D8
:10080000B2010E9488C887FF10C0A30192016985C8
:100810007A858B859C850E94B1CC6093DE157093A0
:10082000DF158093E0159093E11560E06093C615A5
:100830008091F5159091F615A091F715B091F815E6
:100840000097A105B10521F1A5019401281B390BE1
:100850004A0B5B0B57FD1CC06091F9157091FA159E
:1008600080E090E00E948CC89B01AC016091430441
:100870007091440480914504909146040E9488C878
:1008800087FF82C146ED5BE168EE7BE180E0B1DB92
:100890008091BE159091BF15A091C015B091C11562
:1008A000A5019401281B390B4A0B5B0B57FD0FC0A8
:1008B00088DAD501C4018C53964FAF4FBF4F809358
:1008C000BE159093BF15A093C015B093C11580912C
:1008D000FB159091FC15A091FD15B091FE150097A8
:1008E000A105B10511F1881A990AAA0ABB0AB7FC39
:1008F0001CC06091FF157091001680E090E00E948E
:100900008CC89B01AC0160913D0470913E048091C4
:100910003F04909140040E9488C887FF20C144EBA7
:100920005BE167EC7BE18FEF64DB60913B047091EE
:100930003C04072E000C880B990B0E948EC869831B
:100940007A838B839C8395E0C92ED12C24E1E22EFF
:10095000F12C0FEF9E012F5F3F4F4DE354E06BEE04
:1009600075E18FEE95E1F4DCC0903D04D0903E043B
:10097000E0903F04F090400420E030E040EA50E492
:10098000C701B6010E94D8CE87FDE5C020E030E067
:100990004CED52E4C701B6010E9488C818160CF449
:1009A000DAC060913B0470913C04072E000C880B68
:1009B000990B0E948EC8A70196010E94B1CC4B01F1
:1009C0005C012091AE153091AF154091B01550915A
:1009D000B1150E94EDC869877A878B879C87209123
:1009E000DA153091DB154091DC155091DD15C5010C
:1009F000B4010E94B2CC6D837E838F83988760930D
:100A0000DA157093DB158093DC159093DD1520913A
:100A1000AA153091AB154091AC155091AD150E94BF
:100A2000EDC86D877E878F87988B20ED3CEC4CE47A
:100A30005DE36091A6157091A7158091A81590911E
:100A4000A9150E94EDC82B013C012091D6153091CB
:100A5000D7154091D8155091D915C701B6010E94FC
:100A6000B1CC9B01AC01C301B2010E94EDC82B01C6
:100A70003C0123E333E343E75FE36091D2157091D8
:100A8000D3158091D4159091D5150E94EDC89B0186
:100A9000AC01C301B2010E94B2CC2B013C016093B6
:100AA000D2157093D3158093D4159093D515C09219
:100AB000D615D092D715E092D815F092D9152D857C
:100AC0003E854F85588969857A858B859C850E94EE
:100AD000B2CCA30192010E94B1CC6B017C0120E059
:100AE00030E04FE753E40E94D8CE20E030E0A90187
:100AF0001816C4F5C501B4010E94D8CE181684F4A6
:100B0000A50194016D817E818F8198850E94B1CC71
:100B10006093DA157093DB158093DC159093DD15E7
:100B20006FE71AC020E030E0A901C501B4010E94BE
:100B300088C887FF10C0A50194016D817E818F81D7
:100B400098850E94B1CC6093DA157093DB15809381
:100B5000DC159093DD1560E06093C71507CD0E940A
:100B6000967DE3CEC701B6010E9488C887FDDACF23
:100B7000C701B6010E94F6CD75956795EDCF81E06E
:100B80008093E2156FE752CE80E01CD881CE81E0E1
:100B90008093E2154ACE1092E21519861A861B86BA
:100BA0001C86D9CDC301B2010E94D8CE181654F7C5
:100BB000A301920169857A858B859C850E94B1CCC1
:100BC0006093DE157093DF158093E0159093E11527
:100BD0006FE72CCE90916F00292F227091FF05C0F6
:100BE00090916F009D7F90936F0034E0839FC001D0
:100BF0001124FC01EF56FA4E4081518162817381CC
:100C0000FC01EB57FA4E408351836283738381E08A
:100C100080938415222329F080916F008260809355
:100C20006F000895BC012091821530918315409189
:100C30008215509183152417350711F09A01F7CFCB
:100C400081E02617370709F080E008952F923F9240
:100C50004F925F926F927F928F929F92AF92BF92CC
:100C6000CF92DF92EF92FF920F931F93CF93DF9378
:100C7000CDB7DEB762970FB6F894DEBF0FBECDBF1B
:100C80008091450B982F9270E92EE82FE470FE2E8C
:100C9000F82FF170DF2E80FF04C0992311F0E111CD
:100CA00052C0EFEFFAE184918F010F5F1F4F811166
:100CB00003C0E4E6F0E204C00E947840F801F3CFFC
:100CC00084918F010F5F1F4F882321F00E9478408D
:100CD000F801F6CFD1100CC0E2E6F0E284918F016A
:100CE0000F5F1F4F882321F00E947840F801F6CF54
:100CF000E1100CC0E0E6F0E284918F010F5F1F4F1E
:100D0000882321F00E947840F801F6CFF11003C04B
:100D1000EEE5F0E203C0E6E5F0E20AC084918F015F
:100D20000F5F1F4F8823B9F30E947840F801F6CF78
:100D300084918F010F5F1F4F882309F4C7C00E9461
:100D40007840F801F5CF0DEB17E189E294E09A8B3A
:100D5000898BFE0131965F0196E0892E98E1992EEC
:100D60001F01F8016591759185919491E989FA893E
:100D7000C190D190E190F190FA8BE98BA701960197
:100D80000E94B1CC2B013C01F1016083718382830D
:100D9000938320E030E040EA51EC0E94D8CE87FDFA
:100DA0000AC020E030E040EA51E4C301B2010E94F1
:100DB00088C818162CF4F401849118160CF47CC021
:100DC000F101C190D190E190F1901F0120E030E05D
:100DD00040EA51ECC701B6010E94D8CE87FD0AC097
:100DE00020E030E040EA51E4C701B6010E9488C823
:100DF000181614F5EAEEFAE184918F010F5F1F4F88
:100E0000811103C0EAE6F0E204C00E947840F801D4
:100E1000F3CF84918F010F5F1F4F882321F00E9431
:100E20007840F801F6CF88E290E0988B8F8788ECC5
:100E300090E09E878D8738C00C5F1F4FFFEF8F1AA1
:100E40009F0A87E1093C180709F08BCF85EDE82E52
:100E50008BE0F82E10E0F50181919191A191B19173
:100E60005F01F70181939193A193B1937F01812F4A
:100E70000E94F29D1F5F133071F70E94699883E909
:100E800092E0988B8F8704E610E01E870D87BE01E5
:100E9000615F7F4FCE010D960E9434B48AEB92E0E1
:100EA000988B8F871E870D87BE01615F7F4FCE01B4
:100EB0000D960E9434B40AC0F7FAF094F7F8F09453
:100EC000F101C082D182E282F3827ACF62960FB6BC
:100ED000F894DEBF0FBECDBFDF91CF911F910F9170
:100EE000FF90EF90DF90CF90BF90AF909F908F904A
:100EF0007F906F905F904F903F902F900895CF928A
:100F0000DF92EF92FF920F931F93CF93DF9388E5C9
:100F10000E941340D82E89E40E941340C82E8823D3
:100F200019F00E94AC3F1CC0DD20C1F00E94DC3FE4
:100F300020E030E040E251E40E94B1CC20E030E01B
:100F40004CEB51E40E94B2CC21E43CE44EEA5CE379
:100F50000E94EDC80E94F6CD653010F01FEF01C071
:100F6000162F89E50E941340082F8AE40E9413403F
:100F7000C82F882319F00E94AC3F1CC00023C1F089
:100F80000E94DC3F20E030E040E251E40E94B1CC1E
:100F900020E030E04CEB51E40E94B2CC21E43CE490
:100FA0004EEA5CE30E94EDC80E94F6CD653010F079
:100FB000DFEF01C0D62F8AE50E941340E82E811191
:100FC00005C081E50E941340F82E01C0F12CC1102C
:100FD00001C0C0E02C2F30E0D11001C000E0200F94
:100FE000311D2130310521F4E1101AC0F11018C073
:100FF000EAEEFAE18491EF012196811103C0E6E364
:10100000F0E204C00E947840FE01F4CF8491EF0129
:101010002196882309F455C00E947840FE01F6CF3E
:1010200017FD02C0D7FF17C0EAEEFAE18491EF0185
:101030002196811103C0E7E1F0E204C00E947840EC
:10104000FE01F4CF8491EF0121968823D1F10E9413
:101050007840FE01F7CF0E94DC3F9B01AC01012FDD
:10106000110F110BAD2FDD0FBB0BFF2099F085E0A9
:10107000809FF001819FF00D1124EA0FFB1FEE0FFE
:10108000FF1FEE0FFF1FE15DF94E608171818281CC
:10109000938103C060E070E0CB01E5E0E09FE001F8
:1010A000E19FD00D1124CA0FDB1FCC0FDD1FCC0F29
:1010B000DD1FC15DD94E0E94B2CC688379838A83DB
:1010C0009B83DF91CF911F910F91FF90EF90DF9065
:1010D000CF9008952F923F924F925F926F927F929E
:1010E0008F929F92AF92BF92CF92DF92EF92FF9238
:1010F0000F931F93CF93DF93CDB7DEB761970FB6F2
:10110000F894DEBF0FBECDBF83E50E941340882355
:1011100049F00E94CD3F182F811106C080E00E9447
:101120008E9C02C01091A7168091290490912A04E8
:10113000A0912B04B0912C0489839A83AB83BC8348
:1011400080912D0490912E04A0912F04B091300431
:101150008D839E83AF83B887809131049091320450
:10116000A0913304B091340489879A87AB87BC87F8
:101170000E94619C882309F49AC083E40E94134072
:10118000882309F494C00E94DC3F1B012C0105E078
:10119000612C712C38EC388B82EC898BA12CB12C12
:1011A00098EC9E87E2E4EF87015080F125E02D87DF
:1011B000209F400111243D8531503D873F3FA1F3E1
:1011C000F401E30FF11DEE0FFF1FEE0FFF1FE15DB6
:1011D000F94EC080D180E280F3809601A701B5016D
:1011E0008E859F850E94D8CE18161CF45601EE8677
:1011F000FF869601A701B301888999890E9488C852
:1012000087FFD9CF3601E88AF98AD5CF930148897B
:101210005989B5018E859F850E94B2CC20E030E0CF
:1012200040E05FE30E94EDC8A20191010E94B2CCB0
:101230002B013C012DEB37E346E855EB0E94D8CE5D
:1012400087FD0AC02DEB37E346E855E3C301B20141
:101250000E9488C818165CF580E00E948E9C35E0DC
:10126000D32E45E0C42EDA949FEFD91601F105E0A4
:10127000CD9C500111240150B0F37501E00EF11C1A
:10128000C701880F991F880F991FFC01E15DF94E76
:101290007F01A301920160817181828193810E940B
:1012A000B1CCF7016083718382839383E4CF86E5B9
:1012B0000E941340882399F00E94619C882379F052
:1012C000E1E0F0E284917F012FEFE21AF20A882335
:1012D00021F00E947840F701F5CF0E9422AB8AE509
:1012E0000E941340882321F00E94DC3F0E949FB39C
:1012F000812F0E948E9C111103C0EFEFFAE11CC0F8
:101300008091A7168111F9CFEAEEFAE184918F015D
:101310000F5F1F4F882321F00E947840F801F6CF1D
:10132000E2EEFFE184918F010F5F1F4F882329F3C5
:101330000E947840F801F6CF84918F010F5F1F4F14
:10134000882321F00E947840F801F6CF8091A716FB
:10135000811103C06FE073E002C06BE073E084EDC5
:101360009FE10E94024F8AE00E947840EFEFFAE18D
:1013700084918F010F5F1F4F882321F00E947840D6
:10138000F801F6CFE7ECFFE184918F010F5F1F4F6B
:10139000882321F00E947840F801F6CFC090A8166B
:1013A000D090A916E090AA16F090AB1620E030E09D
:1013B000A901C701B6010E94D8CE18164CF442E02C
:1013C000C701B6010E9419448AE00E9478400CC00F
:1013D000E2ECFFE184918F010F5F1F4F882321F022
:1013E0000E947840F801F6CF4CE050E069E274E0EA
:1013F000CE0101960E94EACF892BD1F061960FB6FB
:10140000F894DEBF0FBECDBFDF91CF911F910F913A
:10141000FF90EF90DF90CF90BF90AF909F908F9014
:101420007F906F905F904F903F902F900C946998B1
:1014300061960FB6F894DEBF0FBECDBFDF91CF919E
:101440001F910F91FF90EF90DF90CF90BF90AF90E2
:101450009F908F907F906F905F904F903F902F90D4
:10146000089580916F00982F927081FF05C0809140
:101470006F008D7F80936F008091780F8093770F3E
:101480008093760F8093750F84E68093740F28EE17
:1014900033E03093C5152093C415992329F080912A
:1014A0006F00826080936F0081E0809384150E94BA
:1014B000D8690E9455598091A716882321F08EE1A2
:1014C0009BE00E941D4F8CE0EEE1FBE0A9E2B4E05E
:1014D00001900D928A95E1F70C94653F2F923F920F
:1014E0004F925F926F927F928F929F92AF92BF9234
:1014F000CF92DF92EF92FF920F931F93CF93DF93E0
:10150000CDB7DEB7CD54D1090FB6F894DEBF0FBE0C
:10151000CDBF85E40E945C40882321F00E94AC3F4F
:101520007B0102C0E12CF12C83E40E945C40882303
:1015300021F00E94AC3F6AA302C005E00AA385E542
:101540000E945C40882319F00E94CD3F03C085E5CE
:101550000E9413408CA7F7FC07C0812C912C16E148
:10156000A12E13E4B12E06C0812C912CBCE8AB2E29
:10157000B2E4BB2E83E50E945C40882321F00E94E8
:10158000DC3F4B015C01E114F10411F41092C81529
:1015900010922B0BED820E9416B62B013C011D818F
:1015A00017FF05C00CE310E022E0298304C003E22A
:1015B00010E035E03983D301C2018C53964FAF4F11
:1015C000BF4F8093BE159093BF15A093C015B093E5
:1015D000C11561E06E0D623080F0E4E8FFE18491B6
:1015E0008F010F5F1F4F1A830983882309F45FC39C
:1015F0000E947840E981FA81F2CFEEEAFFE184911E
:101600007F012FEFE21AF20A882321F00E9478402E
:10161000F701F5CF0E94DA7F3D8137FF04C08FE7E5
:101620008093C71508C04D81E42F440FFF0BEA5388
:10163000FA4E8FE78083C501B4010E94F6CD072ED4
:10164000000C880B990B0E948EC86A877B878C8759
:101650009D878981482F50E09801A8EEB3E00E9451
:10166000A2CC6DA77EA78FA798AB8B019C01040D20
:10167000151D261D371D0AAF1BAF2CAF3DAF81E0F6
:10168000809340021D811F3F39F40EEE1EE11FAF13
:101690000EAF08EB1EE106C00CED1EE11FAF0EAF52
:1016A00005EA1EE122961FAF0EAF22974CA25DA263
:1016B0006EA27FA249AA5AAA6BAA7CAA1DAA1EAA38
:1016C0001FAA18AE19AE188E10E4198F0CE10A8FFC
:1016D00016E41B8F1C8E1D8E1E8E1F8E1C8A1D8A6B
:1016E0001E8A1F8A188A198A1A8A1B8A19821A82E4
:1016F0001B821C828FE790E0A0E0B0E08E839F8386
:10170000A887B987FFE7CF2ED12CE12CF12C18A6A2
:1017100019A61AA61BA611E01F861E862D961FAEBF
:101720002D97212C312C2E961FAE2E970D81802FB8
:10173000000F990B9C012A533A4E24963FAF2EAFCF
:101740002497880F991F880F991FDC01AD5BBB4F51
:10175000B9A3A8A3CA01052E000CAA0BBB0B28969F
:101760008CAF9DAFAEAFBFAF28974C5F5F4FCA0144
:10177000550FAA0BBB0B2C968CAF9DAFAEAFBFAF76
:101780002C97AAA10A2E000CBB0BBBA3AAA3809185
:101790004002882309F489C20E9416B64B015C01FD
:1017A0008091C315882309F4D4C00E94C27E0D81A4
:1017B00007FD0CC0A8A1B9A1BC912D96BFAF2D9774
:1017C000E8A1F9A12180328003810BC000913D0482
:1017D0002D960FAF2D9720903E0430903F0400913E
:1017E00040042E960FAF2E972D962FAD2D97322DAC
:1017F000432D2E965FAD2E976C8D7D8D8E8D9F8D9A
:101800000E9488C887FF0AC02D960FAD2D970C8FB8
:101810002D8E3E8E2E960FAD2E970F8F288D398DE3
:101820004A8D5B8D2D966FAD2D97722D832D2E9643
:101830009FAD2E970E9488C887FF0AC02D960FADD6
:101840002D97088F298E3A8E2E960FAD2E970B8FDF
:101850008091BE159091BF15A091C015B091C11592
:10186000A5019401281B390B4A0B5B0B57FD10C0D7
:101870000E94E17ED501C4018C53964FAF4FBF4FFC
:101880008093BE159093BF15A093C015B093C1155A
:101890002D962FAD2D97322D432D2E965FAD2E9781
:1018A0006A857B858C859D851123E9F10E9488C816
:1018B00087FF4FC0B501A40144195509660977098E
:1018C000DB01CA0188589341A109B109B7FD41C0A4
:1018D000D701C6010E811F8128853985801B910B98
:1018E000A20BB30B1D81B595A7959795879517FF0B
:1018F00003C08093C71505C02496EEADFFAD2497B5
:10190000808348A759A76AA77BA70A850C8F1B85E8
:101910001D8F0C850E8F1D851F8F8CA29DA2AEA2E0
:10192000BFA210E016C00E94D8CE181694F4D501BC
:10193000C4012CA13DA14EA15FA1821B930BA40B5E
:10194000B50BAC01BD01485853416109710977FFDE
:10195000CBC120E030E040EA51E46A857B858C858C
:101960009D850E94B2CC2D962FAD2D97322D432D03
:101970002E965FAD2E970E9488C887FF10C0E0E1C9
:10198000FFE184918F010F5F1F4F1A830983882322
:1019900009F48BC10E947840E981FA81F2CFD50128
:1019A000C40129A93AA94BA95CA9821B930BA40BDA
:1019B000B50BB7FD96C00E94DC7C8AE00E9478409F
:1019C000D501C4018053984FAF4FBF4F89AB9AAB3D
:1019D000ABABBCAB0DA9011163C02EA93FA948ADAB
:1019E00059AD2D966FAD2D97722D832D2E969FADEF
:1019F0002E970E94D8CE18160CF041C028966CADD8
:101A00007DAD8EAD9FAD28970E948EC82D962FADCF
:101A10002D97322D432D2E965FAD2E970E94B2CC7E
:101A20006EAB7FAB88AF99AF2DA53EA54FA558A94A
:101A3000280D391D4A1D5B1D2AAF3BAF4CAF5DAF72
:101A40002C966CAD7DAD8EAD9FAD2C970E948EC84F
:101A50009B01AC016A857B858C859D850E94B1CCFC
:101A60002D962FAD2D97322D432D2E965FAD2E97AF
:101A70000E9488C8881F8827881F8DAB32C0D50177
:101A8000C4012AAD3BAD4CAD5DAD821B930BA40BE5
:101A9000B50BB7FD26C04EAD5FAD61E07FE11EC066
:101AA00020E030E040EA51E46A857B858C859D85A5
:101AB0000E94B1CC9B01AC012D966FAD2D97722D7C
:101AC000832D2E969FAD2E970E9488C887FF09C050
:101AD00022964EAD5FAD22976CEC7EE18D810E9427
:101AE000F97FD501C401880F991FAA1FBB1F2CA124
:101AF0003DA14EA15FA1821B930BA40BB50B8419D2
:101B00009509A609B70981389F44A241B10580F023
:101B1000E7E8FEE184918F010F5F1F4F1A8309836D
:101B2000882309F4C2C00E947840E981FA81F2CF8B
:101B30002AA13BA14E855F85241735070CF027CEDF
:101B4000EAE2FEE184918F010F5F1F4F1F830E8336
:101B5000882329F00E947840EE81FF81F3CF1D8118
:101B600017FD03C00EE013E002C00BEF13E01F836C
:101B70000E836E817F8189E19EE10E94024F49813F
:101B80005A816B817C8185E19EE10E94CC4E8AE086
:101B90000E9478406E817F8184E09EE10E94024F26
:101BA000488959896A897B8980E09EE10E94CC4EF0
:101BB0008AE00E9478406E817F818FEE9DE10E94D5
:101BC000024F4C895D896E897F898BEE9DE10E9471
:101BD000CC4E8AE00E9478401CA5112309F467C00E
:101BE0000D8107FF31C029813A814B815C812093AF
:101BF000AE153093AF154093B0155093B1152CEA44
:101C000035EC47E25EE3688979898A899B890E947D
